:100000000C94F6540C9427550C9427550C942755B2
:100010000C9427550C9416890C9427550C9427554D
:100020000C9497880C9427550C9427550C9479E9D7
:100030000C9427550D9485D40C9427550C94275572
:100040000C9427550D94933D0C9427550C942755EB
:100050000C9427550C9427550D94A6530D94B6CCAB
:100060000C9427550C94E3600C9427550C94275559
:100070000C9427550C9427550C9427550C94275510
:100080000C9427550C9427550C9427550C94275500
:100090000C9427550C9427550C9427550C942755F0
:1000A0000C9427550C9427550C9427550C942755E0
:1000B0000C9427550C9427550C9427550C942755D0
:1000C0000C9427550C9427550C9427550C942361B8
:1000D0000C9427550C9427550C9427550C942755B0
:1000E0000C94275571013D01FB0193014D01DD0188
:1000F000B101950131018F018D019901F301A70132
:1001000051015501D1019701390173014901B9012B
:100110000902A901F701570135016F0147019F014C
:10012000E901E101650191018B01EF01C1012F019D
:10013000A501A501A5018901890189010502A10186
:1001400089012D015901F101EB01530167013F01C3
:10015000C5017701AD017901FF019B014301D50183
:100160003F01CD01CF016D01F901AB017B01AF0171
:1001700075015D01D301B5014F01CB01FD01DF0127
:10018000C90181015D010B02D901D701084AD73BA2
:100190003BCE016E84BCBFFDC12F3D6C74319ABD56
:1001A00056833DDA3D00C77F11BED9E4BB4C3E917A
:1001B0006BAAAABE000000803F05A84CCDB2D44E69
:1001C000B93836A9020C50B9918688083CA6AAAA6B
:1001D0002ABE000000803F07634236B79BD8A71AAB
:1001E00039685618AEBAAB558C1D3CB7CC5763BDB9
:1001F0006DEDFD753EF6177231BF000000803F08BF
:10020000000000BE922449123EABAAAA2ABECDCC61
:10021000CC4C3E00000080BEABAAAAAA3E00000063
:1002200000BF000000803F0000000000084178D3BC
:10023000BB4387D1133D190E3CC3BD4282AD2B3E5B
:1002400068EC8276BED98FE1A93E4C80EFFFBE01FB
:10025000C4FF7F3F0000000000000D94969D0D94A8
:100260007C9D0D94AB540D949F910D94B99B0D946E
:1002700097B10D9476850D94BE7B0D9439540D94F1
:100280008ECE0D9475620D945CCE0D94047A0D940F
:10029000E29B0D94AF850D9443800D947D540D9495
:1002A000C1CE0D9407550D940BCE0D9420850D9461
:1002B000A29B0D94F7CD0D94AF810D94EACE0D94D1
:1002C000F1B90D9400770D947FB00D94FA9C0D94C4
:1002D00015CE0D9477760D9450B50D9484CE0D9473
:1002E000CE9B0D942B540D94A5850D94ACCE0D94FE
:1002F00027CE0D9439CE0D94A2CE0D9418C20D9434
:100300000A8C0D94D7CE0D94A7840D94B8810D94CA
:10031000196A0D94AA9D0D94289D0D94B1540D94C5
:10032000AF540D940B9D0D9463540D94A9540D94EA
:1003300057850D94BF540D944DCE0D94D71A0D943E
:10034000F69B0D94BA9D0D94C1810D94849D0D94DE
:10035000E7540D94ED850D94B3CE0D942FCE0D94EE
:10036000A6CE0D94A5540D9404670D94BBCE0D94A8
:100370001B730D94B9850D94F7600D9419BD0D9400
:100380001A640D94749D0D948D650D941FCE0D947B
:10039000A0830D94D3CE0D94C5CE0D9470CE0D9444
:1003A0007ACE0D943A850D94B7CE0D9466CE0D9409
:1003B000E5CE0D94E1CE0D94CA810D948B540D942D
:1003C000CFCE0D94DB9C0D94A9A90D94A3640D943C
:1003D00072700D94139C0D9401CE0D94B8640D941D
:1003E0004B9D0D94FCCD0D94D9540D9481CF0D945B
:1003F0008A9B0D94B0CE0D9455540D94C9CE0D9496
:1004000043CE0D9474820D94D2880D948C9D0D94DE
:10041000B2640D94D3850D94DDCE0D947540486182
:100420007264636F6465642044656661756C7420F2
:1004300053657474696E6773204C6F616465640002
:1004400053746F7265642073657474696E6773208A
:1004500072657472696576656400202020452F44BA
:10046000203D20002020204D393030204B004C69A9
:100470006E65617220616476616E63652073657478
:1004800074696E67733A0046696C616D656E7420BD
:1004900073657474696E67733A2044697361626C42
:1004A0006564002020204D32303020440046696CC5
:1004B000616D656E742073657474696E67733A005C
:1004C0002020204D3230392053004175746F2D5259
:1004D0006574726163743A20533D3020746F2064F8
:1004E000697361626C652C203120746F20696E74B1
:1004F00065727072657420657874727564652D6FAD
:100500006E6C79206D6F76657320617320726574EF
:100510007261637473206F72207265636F766572A7
:10052000696573002046002020204D32303820536A
:10053000005265636F7665723A20533D4578747258
:1005400061206C656E67746820286D6D2920463ABD
:10055000537065656420286D6D2F6D2900205A0049
:100560002046002020204D32303720530052657441
:10057000726163743A20533D4C656E67746820283D
:100580006D6D2920463A537065656420286D6D2F86
:100590006D29205A3A205A4C69667420286D6D29BD
:1005A000002044002049002020204D3330342050CA
:1005B0000050494420686561746265642073657405
:1005C00074696E67733A002044002049002020209F
:1005D0004D333031205000504944207365747469A4
:1005E0006E67733A00205A0020590020204D3230A7
:1005F00036205800486F6D65206F666673657420FD
:10060000286D6D293A00204500205A00205900200D
:10061000580020420020540020204D323035205315
:1006200000416476616E636564207661726961621F
:100630006C65733A20533D4D696E20666565647242
:1006400061746520286D6D2F73292C20543D4D69F0
:100650006E2074726176656C206665656472617483
:100660006520286D6D2F73292C20423D6D696E69C0
:100670006D756D207365676D656E742074696D6549
:1006800020286D73292C20583D6D6178696D756D3A
:10069000205859206A65726B20286D6D2F73292CA4
:1006A00020205A3D6D6178696D756D205A206A650C
:1006B000726B20286D6D2F73292C2020453D6D61B4
:1006C00078696D756D2045206A65726B20286D6DA7
:1006D0002F73290020540020204D32303420530045
:1006E000416363656C65726174696F6E3A20533D56
:1006F000616363656C65726174696F6E2C20543D33
:100700007265747261637420616363656C657261A4
:1007100074696F6E00204500205A00205900202087
:100720004D3230312058004D6178696D756D204132
:100730006363656C65726174696F6E20286D6D2FDF
:100740007332293A00204500205A00205900202009
:100750004D3230332058004D6178696D756D2066DB
:10076000656564726174657320286D6D2F73293A15
:1007700000204500205A0020590020204D39322009
:10078000580053746570732070657220756E6974BB
:100790003A0053657474696E67732053746F7265A1
:1007A0006400454550524F4D204572726F720000F3
:1007B00020006D65736820626564206C6576656CE9
:1007C000696E673A200029002C20002C20007068F8
:1007D00079736963616C20636F6F7264696E6174B1
:1007E00065733A20280029002C20002C2000776F08
:1007F000726C6420636F6F7264696E617465733AC2
:100800002028002046002045004731205A004D3264
:1008100034004D32362053256C75004D3130362072
:10082000530047312046256400473120453120469A
:10083000343830004731205A002046323030300002
:1008400020590047312058004D383300506F7369EC
:1008500074696F6E20726561642066726F6D2065C9
:100860006570726F6D3A004D3233202573002E672C
:10087000636F0046656564726174653A0072656312
:100880006F7665725F6D616368696E655F737461D1
:1008900074655F61667465725F706F7765725F70B3
:1008A000616E69632C20696E697469616C200072E5
:1008B00065636F7665725F6D616368696E655F73AE
:1008C000746174655F61667465725F706F7765727D
:1008D0005F70616E69632C20696E697469616C2058
:1008E000007265636F7665725F6D616368696E65DE
:1008F0005F73746174655F61667465725F706F7752
:1009000065725F70616E69632C20696E69746961DC
:100910006C200063757272656E745F706F736974BA
:10092000696F6E5B5A5F415849535D3A0043757277
:1009300072656E7420706F736974696F6E20595F91
:10094000415849533A0043757272656E7420706F56
:10095000736974696F6E20585F415849533A00417A
:10096000667465722077616974696E6720666F725C
:100970002074656D703A00473120452D3120463492
:1009800038300047312045352046313230004D386F
:1009900033004D31393020532564004D313039203A
:1009A0005325640047323820582059004731205AD7
:1009B00032352046383030004D31343020532564F4
:1009C000004D3130342053256400494E54340055D5
:1009D000564C4F202D20656E640073747073005563
:1009E000564C4F0020423A0020453A00543A005AF3
:1009F000206C6976652061646A757374206F757404
:100A0000206F662072616E67652E2053657474696D
:100A10006E6720746F20302E20436C69636B2074E6
:100A20006F20636F6E74696E75652E005A206C6955
:100A300076652061646A757374206F7574206F66C3
:100A40002072616E67652E2053657474696E67202D
:100A5000746F20300020573A0020453A00543A0085
:100A60004B494C4C3A20004175746F0020452F448F
:100A70003D00416476616E6365204B3D0022283263
:100A800029005400496E76616C6964205420636FBC
:100A900064652E00496E76616C6964204D20636F39
:100AA00064652E004D3232302053256900203A20F3
:100AB00000004C414E472053454C20464F52434581
:100AC0004400222831290020453A00205A3A0020CB
:100AD000593A0020453A00205A3A0020593A005825
:100AE0003A004D31313320530020002E0020423A8D
:100AF0000020453A00543A0020413A0020503A0084
:100B00002042403A0020403A00202F003A00205472
:100B100000202F0020423A00202F006F6B20543A13
:100B2000002569206D696E2C20256920736563009E
:100B3000496E76616C6964204D20636F6465004D79
:100B400065736820626564206C6576656C696E67A4
:100B5000206E6F74206163746976652E000A002030
:100B600020000A4D6561737572656420706F696E4F
:100B700074733A000A5A207365617263682068656D
:100B8000696768743A20002C004E756D20582C5906
:100B90003A2000476F20686F6D652066696E697343
:100BA000686564004D65736820626564206C6576D5
:100BB000656C696E67206163746976617465640051
:100BC000557073616D706C652066696E69736865D8
:100BD0006400426564206C6576656C696E672063AD
:100BE0006F7272656374696F6E2066696E6973688F
:100BF000656400206D6963726F6E7300457863658C
:100C0000737369766520626564206C6576656C69CE
:100C10006E6720636F7272656374696F6E3A20004D
:100C20006261627973746570206170706C6965646B
:100C300000636C65616E2075702066696E6973680B
:100C40006564200000206F66667365743A20006D4D
:100C500065736820626564206C6576656C696E6793
:100C60003A2000473238205730003A200054656D52
:100C700070657261747572652063616C696272611E
:100C800074696F6E20646F6E652E20436F6E746999
:100C90006E75652077697468207072657373696E0C
:100CA0006720746865206B6E6F622E0000205A20EA
:100CB000736869667420286D6D293A0050494E4466
:100CC000412074656D70657261747572653A2000BB
:100CD000002F3600537465703A200000205A2073AC
:100CE0006869667420286D6D293A0050494E444168
:100CF0002074656D70657261747572653A20002F9D
:100D0000362028736B6970706564290053746570B0
:100D10003A2000005A45524F3A2000007374617225
:100D2000742074656D70657261747572653A200027
:100D300050494E44412070726F62652063616C6956
:100D400062726174696F6E207374617274004732ED
:100D500038205730000A00205A3A200020593A2003
:100D60000020583A20004732382C2066696E616CAA
:100D700020004732382C2066696E616C20004732B3
:100D8000382C2066696E616C20004732382C20694F
:100D90006E697469616C20004732382C20696E6975
:100DA0007469616C200044393939004D3239006270
:100DB0007573793A2070617573656420666F72206F
:100DC000696E70757400627573793A20706175731D
:100DD000656420666F722075736572006275737941
:100DE0003A2070726F63657373696E670020557087
:100DF0006C6F616420696E2070726F6772657373C7
:100E000000696E697469616C207A7374657073200F
:100E100061667465722072657365743A2000696E4C
:100E2000697469616C207A7374657073206F6E20C9
:100E3000706F7765722075703A2000466163746F39
:100E400072792052455345540020202020334420FD
:100E5000205072696E74657273202020200020205B
:100E6000204F726967696E616C20507275736120E2
:100E70002020004E6F76203136203230313700434B
:100E80006F6D70696C65643A2000286E6F6E652C1A
:100E90002064656661756C7420636F6E666967298E
:100EA000004E6F7620313620323031372032313AE1
:100EB00035393A3135007374617274002020202076
:100EC000334420205072696E746572732020202094
:100ED000002020204F726967696E616C2050727526
:100EE00073612020200025002020202020200020C9
:100EF00020202020200045524153494E4720616C5C
:100F00006C206461746100466163746F7279205271
:100F10004553455400FFFFFF0000A0400000A040E3
:100F20000000004000007F4300005E439AD9514317
:100F300000000000000040C19A99193E00007F4364
:100F4000000052430000524300000000000040C176
:100F50009A99193E6563686F3A004572726F723AEA
:100F60000000002110422063308440A550C660E795
:100F700070088129914AA16BB18CC1ADD1CEE1EF4E
:100F8000F13112100273325222B5529442F772D6E6
:100F900062399318837BB35AA3BDD39CC3FFF3DE9E
:100FA000E36224433420040114E664C774A4448536
:100FB000546AA54BB528850995EEE5CFF5ACC58DEE
:100FC000D55336722611163006D776F6669556B486
:100FD000465BB77AA719973887DFF7FEE79DD7BC3E
:100FE000C7C448E5588668A77840086118022823D6
:100FF00038CCC9EDD98EE9AFF9488969990AA92B8E
:10100000B9F55AD44AB77A966A711A500A333A1225
:101010002AFDDBDCCBBFFB9EEB799B588B3BBB1ADD
:10102000ABA66C877CE44CC55C222C033C600C4175
:101030001CAEED8FFDECCDCDDD2AAD0BBD688D492D
:101040009D977EB66ED55EF44E133E322E511E70C5
:101050000E9FFFBEEFDDDFFCCF1BBF3AAF599F787D
:101060008F8891A981CAB1EBA10CD12DC14EF16F2E
:10107000E18010A100C230E3200450254046706793
:1010800060B9839893FBA3DAB33DC31CD37FE35EBF
:10109000F3B1029012F322D23235421452776256E3
:1010A00072EAB5CBA5A89589856EF54FE52CD50DCF
:1010B000C5E234C324A01481046674476424540533
:1010C00044DBA7FAB79987B8975FE77EF71DC73C5F
:1010D000D7D326F2369106B0165766767615463483
:1010E000564CD96DC90EF92FE9C899E9898AB9AB6F
:1010F000A94458654806782768C018E1088238A3D3
:10110000287DCB5CDB3FEB1EFBF98BD89BBBAB9AFE
:10111000BB754A545A376A167AF10AD01AB32A9222
:101120003A2EFD0FED6CDD4DCDAABD8BADE89DC90E
:101130008D267C076C645C454CA23C832CE01CC172
:101140000C1FEF3EFF5DCF7CDF9BAFBABFD98FF89E
:101150009F176E367E554E745E932EB23ED10EF0C2
:101160001E7C3C3E5E2B3D3F2F5B5D3B2C2A225C70
:10117000004D383420582059205A2045004D323433
:10118000004D3233202573006175746F25692E6719
:10119000000A002F000A002E0044656C6574696F18
:1011A0006E206661696C65642C2046696C653A2026
:1011B0000046696C652064656C657465643A002E50
:1011C000002E002E002E004E6F7720667265736829
:1011D0002066696C653A20004E6F7720646F696EF7
:1011E000672066696C653A20002220706F730022C8
:1011F00020706172656E743A2200535542524F5509
:1012000054494E452043414C4C20746172676574CB
:101210003A2200747279696E6720746F2063616C82
:101220006C207375622D67636F64652066696C65F9
:1012300073207769746820746F6F206D616E7920F8
:101240006C6576656C732E204D4158206C65766513
:101250006C2069733A00256920686F7572732025C8
:1012600069206D696E757465730054494D454F551D
:10127000543A004D3131300046756C6C2052582084
:101280004275666665720022206661696C65643A23
:10129000204275666665722066756C6C2100456E2D
:1012A000717565696E6720746F2074686520667259
:1012B0006F6E743A2022002200456E717565696E6A
:1012C0006720746F207468652066726F6E743A20B0
:1012D000220022206661696C65643A204275666668
:1012E00065722066756C6C210022004D363030002E
:1012F0005072757361206933204D4B3320626572E3
:101300006569742E005072757361206933204D4BEE
:101310003320676F746F7761005072757361206955
:1013200033204D4B3320707265702E0050727573F0
:1013300061206933204D4B332070726F6E74612EC3
:10134000005072757361206933204D4B33206F6BF1
:10135000005072757361206933204D4B33207265E4
:101360006164792E007A5F6D696E3A20007A5F6D54
:1013700061783A20005A204F666673657400795F81
:101380006D696E3A2000795F6D61783A20005920CE
:10139000456E746665726E756E6720766F6D206D32
:1013A000696E004F646C65676C6F73632059206FC2
:1013B00064206D696E2E3A0044697374616E7A61BF
:1013C0002059206461206D696E3A005920767A6454
:1013D000616C656E6F7374206F64206D696E3A0086
:1013E000592064697374616E63652066726F6D2045
:1013F0006D696E3A004A610054616B005369005395
:101400006900416E6F0059657300785F6D696E3ACF
:101410002000785F6D61783A200058595A204B615E
:101420006C2E2044657461696C7300537A637A652D
:10143000676F6C79206B616C2E58595A0058595A55
:101440002043616C2E206465747461676C6900448C
:10145000657461696C792058595A206B616C2E0053
:1014600058595A2063616C2E2064657461696C73ED
:1014700000496368207765726465206A65747A74D0
:1014800020646965205A204B616C696272696572DB
:10149000756E672064757263686675656872656EDF
:1014A0002E00576C61637A616D206B616C696272AA
:1014B00061636A65207A2E00566F79206120686129
:1014C0006365722043616C6962726163696F6E204B
:1014D0005A2061686F72612E0041646573736F20DA
:1014E0006176766965726F20756E612043616C6903
:1014F0006272617A696F6E65205A2E004E796E694C
:101500002070726F76656475207A206B616C6962F9
:10151000726163692E00492077696C6C2072756E68
:10152000207A2063616C6962726174696F6E206EEB
:101530006F772E00496368207765726465206A655D
:10154000747A74206469652058595A2D4B616C690E
:101550006272696572756E6720647572636866751C
:10156000656872656E2E204573207769726420630A
:10157000612E203132204D696E7574656E20646174
:101580007565726E00576C61637A616D206B616C7A
:1015900069627261636A652078797A2E205A616A7D
:1015A0006D696520746F206F6B2E203132206D695C
:1015B0006E2E0048617265206C612063616C696207
:1015C000726163696F6E2058595A2E20546172649B
:1015D000617261203132206D696E2E206170726FF0
:1015E00078696D6164616D656E74652E0041646536
:1015F00073736F206176766965726F20756E6120F6
:1016000043616C696272617A696F6E652058595ADC
:101610002E2050756F206475726172652063697247
:101620006361203132206D696E2E004E796E692023
:1016300070726F766564752078797A206B616C6959
:1016400062726163692E205A616265726520746FEF
:1016500020707269626C697A6E65203132206D6922
:101660006E2E00492077696C6C2072756E20787937
:101670007A2063616C6962726174696F6E206E6F4B
:10168000772E2049742077696C6C2074616B65201B
:10169000617070726F782E203132206D696E732EFA
:1016A000004A65747A74207765726465206963689E
:1016B00020646965204475657365206675657220D0
:1016C000504C4120766F726865697A656E2E2000F5
:1016D0004E6167727A6577616D206479737A6520EF
:1016E000646C6120504C412E00566F79206120704F
:1016F000726563616C656E74617220656C206E6FDB
:101700007A7A6C65207061726120504C412061686A
:101710006F72612E0041646573736F207072657221
:10172000697363616C6465726F206C277567656CA3
:101730006C6F2070657220504C412E004E796E699E
:101740002070726564656872656A69207472797365
:101750006B752070726F20504C412E004E6F7720B9
:10176000492077696C6C2070726568656174206EC1
:101770006F7A7A6C6520666F7220504C412E00485B
:10178000616C6C6F2C206963682062696E206465EF
:10179000696E204F726967696E616C205072757353
:1017A0006120693320447275636B65722E204D6F22
:1017B00065636874656E20536965206D65696E6543
:1017C0002048696C66652064757263682064656E84
:1017D0002053657475702D50726F7A6573733F0076
:1017E000437A6573632C206A657374656D20547742
:1017F0006F6A61206472756B61726B61204F7269F0
:1018000067696E616C2050727573612069332E2098
:10181000437A7920706F74727A6562756A65737A3B
:1018200020706F6D6F6379207A20696E7374616CBC
:1018300061636A613F00486F6C612C20736F79208F
:10184000747520696D707265736F7261204F726973
:1018500067696E616C2050727573612069332E2048
:1018600051756965726573207175652074652067AF
:1018700075696520612074726176657320646520E6
:101880006C6120636F6E66696775726163696F6E04
:101890003F004369616F2C20736F6E6F206C612075
:1018A000747561207374616D70616E7465204F7220
:1018B0006967696E616C2050727573612069332E9F
:1018C0002047726164697265737469206169757417
:1018D0006F206174747261766572736F20696C2019
:1018E00070726F636573736F20646920636F6E66D7
:1018F00069677572617A696F6E653F00446F6272E5
:10190000792064656E2C206A73656D20766173653D
:10191000207469736B61726E61204F726967696EC2
:10192000616C2050727573612069332E20436863A7
:1019300065746520616279636820566173207072F6
:101940006F7665646C61206B616C69627261636E55
:10195000696D2070726F636573656D3F0048692C17
:10196000204920616D20796F7572204F7269676917
:101970006E616C20507275736120693320707269DA
:101980006E7465722E20576F756C6420796F7520A8
:101990006C696B65206D6520746F2067756964657F
:1019A00020796F75207468726F7567682074686538
:1019B0002073657475702070726F636573733F0078
:1019C000496368207765726465206A65747A74205B
:1019D0006572737465204C696E6965206472756305
:1019E0006B656E2E205761656872656E6420646554
:1019F0007320447275636B6573206B6F656E6E65E3
:101A00006E2053696520646965204475657365209F
:101A1000616C6C6D6165686C6963682073656E6B81
:101A2000656E20696E64656D205369652064656E1E
:101A3000204B6E6F70662064726568656E2C206244
:101A400069732053696520646965206F7074696DDE
:101A5000616C6520486F65686520657272656963B1
:101A600068656E2E20556562657270727565666573
:101A70006E20536965206469652042696C646572F3
:101A800020696E20756E736572656D2048616E64A5
:101A90006275636820696D204B61706974656C20A4
:101AA0004B616C696272696572756E67005A616339
:101AB0007A6E65206472756B6F776163206C696EF6
:101AC00069652E2053746F706E696F776F206F7029
:101AD00075737A637A616A206479737A65207072AB
:101AE0007A656B726563616A61632067757A696B99
:101AF0002C20706F6B69206E696520757A79736B25
:101B000061737A206F7074796D616C6E656A20778D
:101B100079736F6B6F7363692E2053707261776492
:101B20007A206F6272617A6B692077206E61737AB6
:101B3000796D20706F7261646E696B7520772072A9
:101B40006F7A647A2E204B616C69627261636A619C
:101B500000566F79206120636F6D656E7A61722027
:101B60006120696D7072696D6972206C61206C69A9
:101B70006E656120792074752062616A617261739B
:101B800020656C206E6F7A7A6C652067726164756F
:101B9000616C6D656E746520616C20726F7461722A
:101BA00020656C206D616E646F2C206861737461B8
:101BB00020717565206C6C65677565732061206C9C
:101BC0006120616C74757261206F7074696D612E33
:101BD000204D697261206C617320696D6167656E6B
:101BE00065732064656C206361706974756C6F2027
:101BF00043616C6962726163696F6E20656E206516
:101C00006C206D616E75616C2E0041646573736F3D
:101C100020696E697A6965726F2061207374616DE5
:101C20007061726520756E61206C696E65612065FA
:101C300020747520646F76726169206162626173DD
:101C400073617265206C277567656C6C6F20706FAF
:101C5000636F2070657220766F6C74612072756F8F
:101C600074616E646F206C61206D616E6F706F6C5B
:101C7000612073696E6F2061207261676769756E9C
:101C80006765726520756E6120616C74657A7A6132
:101C9000206F7474696D616C652E205065722066CA
:101CA00061766F72652064616920756E6F2073675D
:101CB000756172646F20616C6C27696D6D61676915
:101CC0006E652064656C206E6F7374726F206D6139
:101CD0006E75616C652C206361702E43616C696266
:101CE00072617A696F6E652E005A61636E75207439
:101CF00069736B6E6F7574206C696E6B75206120F3
:101D000056792062756465746520706F73747570A0
:101D10006E6520736E697A6F766174207472797360
:101D20006B75206F746163656E696D20746C61639F
:101D300069746B6120646F6B7564206E65646F738A
:101D400061686E657465206F7074696D616C6E6931
:101D5000207679736B792E2050726F686C65646E93
:101D6000657465207369206F6272617A6B79207681
:101D7000206E617369207072697275636365207685
:101D8000206B617069746F6C65204B616C69627265
:101D900061636500492077696C6C207374617274AB
:101DA00020746F207072696E74206C696E6520619A
:101DB0006E6420796F752077696C6C20677261643E
:101DC00075616C6C79206C6F776572207468652022
:101DD0006E6F7A7A6C6520627920726F74617469B3
:101DE0006E6720746865206B6E6F622C20756E7450
:101DF000696C20796F75207265616368206F7074FB
:101E0000696D616C206865696768742E2043686538
:101E1000636B2074686520706963747572657320E4
:101E2000696E206F75722068616E64626F6F6B20DF
:101E3000696E20636861707465722043616C6962C9
:101E4000726174696F6E2E004A65747A74207765CA
:101E5000726465206963682064656E2041627374F2
:101E6000616E64207A7769736368656E2044756576
:101E700073656E737069747A6520756E6420447240
:101E800075636B62657474206B616C6962726965FD
:101E900072656E2E004B616C696272756A65206FA7
:101EA000646C65676C6F7363206D6965647A792013
:101EB0006B6F6E636F776B61206479737A792061E1
:101EC0002073746F6C696B69656D2E00566F792095
:101ED000612063616C6962726172206C6120646967
:101EE0007374616E63696120656E747265206C61E4
:101EF0002070756E74612064656C206E6F7A7A6CE8
:101F0000652079206C6120737570657266696369FC
:101F100065206465206C6120686561746265642E6B
:101F20000041646573736F2074617265726F206C19
:101F30006F2073746163636F2066726120756765DB
:101F40006C6C6F20652073757065726669636520BF
:101F500064656C2070696174746F2E004E796E69CF
:101F6000207A6B616C696272756A6920767A646145
:101F70006C656E6F7374206D657A69206B6F6E632C
:101F8000656D20747279736B79206120706F767241
:101F90006368656D2068656174626564752E004EC6
:101FA0006F7720492077696C6C2063616C6962727D
:101FB0006174652064697374616E63652062657421
:101FC0007765656E20746970206F6620746865207F
:101FD0006E6F7A7A6C6520616E64206865617462E8
:101FE000656420737572666163652E005A756E6153
:101FF00065636873742066756568726520696368D7
:102000002064656E2053656C62737474657374200C
:10201000647572636820756D206469652068616508
:10202000756669677374656E2050726F626C656D5A
:10203000652062656920646572204175666261751C
:10204000207A752075656265727072756566656E59
:102050002E004E616A706965727720776C61637AD1
:1020600065206175746F7465737420772063656C87
:1020700075206B6F6E74726F6C6C69206E616A6331
:102080007A657374737A7963682070726F626C65B5
:102090006D6F77207A206D6F6E74617A656D2E009A
:1020A0005072696D65726F2C206861726520656C75
:1020B0002053656C6674657374207061726120636F
:1020C0006F6D70726F626172206C6F732070726FCF
:1020D000626C656D6173206465206D6F6E74616AFA
:1020E00065206D617320636F6D756E65732E0041A1
:1020F0006E7A69747574746F206176766965726F33
:1021000020696C2053656C6620546573742070657B
:102110007220636F6E74726F6C6C61726520676C95
:1021200069206572726F72692064692061737365DA
:102130006D626C616767696F2070697520636F6D90
:10214000756E692E004E656A6472697620706F6DD7
:102150006F63692073656C667465737475207A6B40
:102160006F6E746F6C756A69206E656A63617374F3
:10217000656A736920636879627920767A6E696B23
:10218000616A69636920707269207365737461762E
:10219000656E69207469736B61726E792E00466991
:1021A0007273742C20492077696C6C2072756E20D4
:1021B0007468652073656C667465737420746F2031
:1021C000636865636B206D6F737420636F6D6D6FF3
:1021D0006E20617373656D626C792070726F626CD2
:1021E000656D732E00446572206C617566656E6462
:1021F0006520417373697374656E74206C6F6573C9
:102200006368742064696520616B7475656C6C65C6
:10221000204B616C69627269657265726765626E96
:102220006973736520756E64207769726420766FB8
:102230006E20416E66616E6720616E20626567691F
:102240006E6E656E2E20466F72747365747A656E5D
:102250003F00576C61637A656E69652057697A61E2
:102260007264207573756E6965206F6265636E6553
:102270002064616E65206B616C6962726163796A6A
:102280006E652069207A61637A6E6965206F6420CB
:102290006E6F77612E204B6F6E74796E756F7761FC
:1022A000633F00456A65637574617220656C2057F1
:1022B000697A61726420626F7272617261206C6F00
:1022C000732076616C6F7265732064652063616C46
:1022D0006962726163696F6E2061637475616C65B8
:1022E00073207920636F6D656E7A61726120646519
:1022F000206E7565766F2E20436F6E74696E756102
:10230000723F005365206176766920696C205769B9
:102310007A617264207065726465726169206C61B3
:102320002063616C696272617A696F6E6520707298
:10233000656573697374656E7465206520646F7676
:10234000726169207269636F6D696E63696172653C
:102350002064616C6C27696E697A696F2E20436F07
:102360006E74696E756172653F0053707573746544
:102370006E692057697A617264612076796D617A3D
:102380006520756C6F7A656E65207679736C65640F
:102390006B79207673656368206B616C696272612A
:1023A0006369206120737075737469206B616C6957
:1023B000627261636E692070726F636573206F640F
:1023C000207A616361746B752E20506F6B7261634C
:1023D0006F7661743F0052756E6E696E6720576943
:1023E0007A6172642077696C6C2064656C657465D1
:1023F0002063757272656E742063616C69627261CC
:1024000074696F6E20726573756C747320616E648D
:102410002073746172742066726F6D207468652019
:10242000626567696E6E696E672E20436F6E7469B0
:102430006E75653F004D6F65636874656E20536906
:10244000652064656E206C65747A74656E205363D4
:10245000687269747420776965646572686F6C6509
:102460006E20756D2064656E2041627374616E64C8
:10247000207A7769736368656E204475657365209B
:10248000756E6420447275636B62657474206E654A
:10249000752065696E7A757374656C6C656E3F0046
:1024A00043686365737A20706F77746F727A7963AB
:1024B000206F737461746E69206B726F6B2069207A
:1024C00070727A65737461776963206F646C656795
:1024D0006C6F7363206D6965647A79206479737AAF
:1024E0006120612073746F6C696B69656D3F005189
:1024F00075696572657320726570657469722065AF
:102500006C20756C74696D6F207061736F207061E1
:102510007261207265616A7573746172206C6120EA
:1025200064697374616E636961206E6F7A7A6C6539
:102530002D686561746265643F0044657369646514
:102540007269207269706574657265206C27756C9C
:1025500074696D6F2070617373616767696F207054
:102560006572206D69676C696F72617265206C615C
:102570002064697374616E7A612066726120756788
:10258000656C6C6F20652070696174746F3F0043E7
:102590006863657465206F70616B6F76617420701D
:1025A0006F736C65646E69206B726F6B2061207055
:1025B0006F7A6D656E697420767A64616C656E6F92
:1025C0007374206D657A6920747279736B6F7520EE
:1025D0006120686561746265643F00446F20796FB3
:1025E000752077616E7420746F20726570656174F8
:1025F000206C617374207374657020746F20726531
:1026000061646A7573742064697374616E636520B4
:102610006265747765656E206E6F7A7A6C6520618D
:102620006E6420686561746265643F00536965206B
:102630006B6F656E6E656E20696D6D657220646589
:102640006E204173697374656E74656E20696D20C8
:102650004D656E75206E657520617566727566656F
:102660006E3A204B616C696272696572756E6720A3
:102670002D3E20417373697374616E74005A6177E3
:10268000737A65206D6F7A65737A2070727A7977C4
:10269000726F6369632057697A6172642070727A1D
:1026A000657A204B616C69627261636A61202D3EBC
:1026B0002057697A6172642E005369656D70726586
:1026C000207075656465732061636365646572205D
:1026D000616C206173697374656E746520646573E1
:1026E00064652043616C6962726163696F6E202D5D
:1026F0003E2057697A617264004520706F73736978
:1027000062696C652070726F7365677569726520A8
:102710006C612067756964652057697A617264200D
:10272000696E207175616C7369617369206D6F6D7D
:10273000656E746F206174747261766572736F2058
:1027400043616C696272617A696F6E65202D3E200B
:1027500057697A6172642E0057697A6172646120E8
:102760006D757A657465206B64796B6F6C69762022
:102770007A6E6F76752073707573746974207A2021
:102780006D656E752043616C6962726174696F6E0C
:10279000202D3E2057697A61726400596F7520635D
:1027A000616E20616C7761797320726573756D65F8
:1027B000207468652057697A6172642066726F6D53
:1027C0002043616C6962726174696F6E202D3E20D6
:1027D00057697A6172642E0049737420657320779B
:1027E00069726B6C69636820504C412046696C616A
:1027F0006D656E743F00437A7920746F2066696C52
:10280000616D656E7420504C413F00457320656CCE
:102810002066696C616D656E746F20504C413F009D
:10282000452071756573746F20756E2066696C61E3
:102830006D656E746F20646920504C413F004A659D
:1028400020746F20504C412066696C616D656E7418
:102850003F00497320697420504C412066696C61C7
:102860006D656E743F004675656872656E205369CC
:102870006520626974746520504C412046696C6122
:102880006D656E7420696E2064656E204578747283
:102890007564657220756E64206265737461657419
:1028A0006967656E205369652064656E204B6E6FA5
:1028B000706620756D206573207A75206C61646583
:1028C0006E2E0050726F737A6520756D6965736343
:1028D0002066696C616D656E7420504C41207720D4
:1028E000656B737472756465727A652069206E61B8
:1028F0006369736E696A2070727A796369736B2099
:102900006279207A616C61646F7761632E00496E31
:1029100073657274612C20706F72206661766F72BD
:102920002C2066696C616D656E746F20504C41207F
:10293000656E20656C206578747275736F722E20D9
:10294000446573707565732068617A20636C696390
:102950002070617261206361726761726C6F2E001A
:10296000506572206661766F726520696E7365725C
:102970006973636920696C2066696C616D656E744A
:102980006F20646920504C41206E656C6C27657324
:10299000747275736F72652C20706F692070726528
:1029A0006D69206C61206D616E6F706F6C6120705D
:1029B00065722063617269636172652E0050726F87
:1029C00073696D20766C6F7A746520504C41206677
:1029D000696C616D656E7420646F206578747275C2
:1029E000646572752C20706F207465207374697330
:1029F0006B6E65746520746C616369746B6F2070B5
:102A0000726F207A61766564656E692066696C61B3
:102A10006D656E74752E00506C6561736520696E0E
:102A20007365727420504C412066696C616D656EEF
:102A30007420746F2074686520657874727564659D
:102A4000722C207468656E207072657373206B6ED3
:102A50006F6220746F206C6F61642069742E004275
:102A600069747465206C6164656E205369652050DB
:102A70004C412D46696C616D656E7420756E6420E5
:102A800066616872656E20536965206D69742064A3
:102A9000656D20417373697374656E74656E20662D
:102AA0006F72742C20696E64656D205369652064B3
:102AB000656E20447275636B6572206E6575207358
:102AC00074617274656E2E0050726F737A65207A2D
:102AD000616C6164756A2066696C616D656E7420F5
:102AE000504C4120692070727A7977726F63205759
:102AF000697A6172642070727A657A207265737483
:102B0000617274206472756B61726B692E0043612F
:102B10007267612066696C616D656E746F20504CE0
:102B2000412C20706F72206661766F722C207920A4
:102B30007265696E69636961206C6120696D70728C
:102B400065736F7261207061726120636F6E74696A
:102B50006E75617220636F6E20656C2057697A61B3
:102B6000726400506572206661766F7265206361E1
:102B7000726963612066696C616D656E746F206453
:102B80006920504C4120652072697072656E6469DD
:102B900020696C2057697A61726420646F706F20BD
:102BA000617665722072696176766961746F206CF6
:102BB00061207374616D70616E74652E0050726F68
:102BC00073696D207A61766564746520504C41208C
:102BD00066696C616D656E74206120706F2074652C
:102BE000206F626E6F7674652057697A61726461D6
:102BF00020737469736B6E7574696D20726573658B
:102C00007420746C616369746B612E00506C656133
:102C10007365206C6F616420504C412066696C6163
:102C20006D656E7420616E64207468656E207265D7
:102C300073756D652057697A6172642062792072BC
:102C400065626F6F74696E67207468652070726961
:102C50006E7465722E00566F726865697A656E20B3
:102C60006465722044756573652E204269747465CD
:102C70002077617274656E2E004E6167727A657797
:102C8000616E6965206479737A792E2050726F7352
:102C90007A6520637A656B61632E005072656361AB
:102CA0006C656E74616E646F206E6F7A7A6C652EDF
:102CB0002045737065726120706F72206661766F57
:102CC000722E0053746F2070726572697363616C49
:102CD00064616E646F206C277567656C6C6F2E2065
:102CE000506572206661766F726520617474656EDE
:102CF00064692E00507265646568726976616D2042
:102D0000747279736B752E2050726F73696D2063C6
:102D1000656B656A74652E005072656865617469DB
:102D20006E67206E6F7A7A6C652E20506C656173C9
:102D30006520776169742E00497374206461732083
:102D400046696C616D656E742067656C6164656E63
:102D50003F0046696C616D656E74206A657374200E
:102D60007A616C61646F77616E793F00457374615D
:102D700020656C2066696C616D656E746F2063619F
:102D8000726761646F3F00496C2066696C616D65B4
:102D90006E746F206520737461746F206361726953
:102DA0006361746F3F004A652066696C616D656E92
:102DB00074207A61766564656E3F004973206669A8
:102DC0006C616D656E74206C6F616465643F004179
:102DD0006C6C657320777572646520676574616ECD
:102DE0002E205669656C205370617373206265698B
:102DF0006D20447275636B656E2100476F746F7749
:102E0000652E205564616E65676F206472756B7501
:102E100021005465726D696E61646F212046656C96
:102E2000697A20696D70726573696F6E2100426501
:102E30006E20666174746F2E2042756F6E61207310
:102E400074616D70612100567365206A6520686F3A
:102E5000746F766F2E00416C6C20697320646F6E06
:102E6000652E204861707079207072696E74696E89
:102E70006721004269747465207265696E696765CF
:102E80006E2053696520646173204865697A6265C4
:102E9000747420756E642064727565636B656E2052
:102EA0005369652064616E6E2064656E204B6E6FA1
:102EB00070662E0050726F737A65206F637A797333
:102EC000632073746F6C696B2069206E6163697332
:102ED0006E696A2067757A696B2E004C696D70693E
:102EE00061206C6120737570657266696369652025
:102EF0006465206C6120686561746265642C207073
:102F00006F72206661766F722C20792068617A205A
:102F1000636C696300506572206661766F7265202C
:102F200070756C6973636920696C20706961747471
:102F30006F2C20706F69207072656D69206C612044
:102F40006D616E6F706F6C612E0050726F73696D82
:102F5000206F636973746574652068656174626568
:102F600064206120737469736B6E65746520746C82
:102F7000616369746B6F2E00506C656173652063CB
:102F80006C65616E206865617462656420616E6461
:102F9000207468656E207072657373207468652094
:102FA0006B6E6F622E004269747465207565626590
:102FB000727072756566656E2053696520756E73F3
:102FC00065722048616E646275636820756E642066
:102FD0006265686562656E2053696520646173206F
:102FE00050726F626C656D2E2046616872656E204E
:102FF0005369652064616E6E206D69742064656D2F
:1030000020417373697374656E74656E20666F72A8
:10301000742C20696E64656D205369652064656E4B
:1030200020447275636B6572206E657520737461E0
:103030007274656E2E0050726F737A6520737072B1
:103040006177647A206E61737A20706F7261646E4A
:10305000696B2069206E61707261772070726F6297
:103060006C656D2E20506F74656D2070727A797763
:10307000726F632057697A6172642072657374613C
:103080007274756A6163206472756B61726B652E10
:10309000004C656520656C206D616E75616C2079F2
:1030A0002072657375656C766520656C2070726F33
:1030B000626C656D612E20446573707565732C209C
:1030C0007265696E69636961206C6120696D7072F7
:1030D00065736F7261207920636F6E74696E7561BC
:1030E00020636F6E20656C2057697A6172640050AE
:1030F0006572206661766F726520636F6E73756CA2
:10310000746120696C206E6F7374726F206D616ED4
:1031100075616C6520706572207269736F6C76657D
:10312000726520696C2070726F626C656D612E2013
:10313000506F692072697072656E646920696C20D5
:1031400057697A61726420646F706F20617665726E
:103150002072696176766961746F206C6120737486
:10316000616D70616E74652E0050726F73696D20B1
:103170006E61686C65646E65746520646F206D6156
:103180006E75616C752061206F7072617674652058
:1031900070726F626C656D2E20506F207465206FA9
:1031A000626E6F7674652057697A6172646120720D
:1031B00065626F6F746F76616E696D207469736B91
:1031C00061726E792E00506C65617365206368656D
:1031D000636B206F75722068616E64626F6F6B2025
:1031E000616E6420666978207468652070726F6211
:1031F0006C656D2E205468656E20726573756D6503
:10320000207468652057697A61726420627920723F
:1032100065626F6F74696E6720746865207072698B
:103220006E7465722E0057697A617264002057616E
:10323000746368646F6720526573657400496E66D5
:103240006F726D6174696F6E00496E666F726D6149
:10325000636A65004D6F6E69746F72697A6172009E
:1032600053636865726D61746120696E666F0049B1
:103270006E666F726D61636500496E666F20736381
:103280007265656E0045727374652D53636869637A
:103290006874204B616C004B616C2E20312E2077BE
:1032A0006172737477790043616C2E207072696D5E
:1032B000657261206361702E0043616C2E20707214
:1032C000696D6F206C617965722E004B616C2E20E8
:1032D0007072766E692076727374767900466972C0
:1032E0007374206C617965722063616C2E00576184
:1032F0007274652061756620757365722E2E2E00BE
:103300004573706572616E646F206F7264656E657F
:103310007300417474656E64656E646F20757465C6
:103320006E7465005761697420666F7220757365ED
:10333000722E2E2E004265696D20447275636B20DB
:1033400062656E75747A746500557A79746520705B
:10335000727A79206472756B7500557361646F20A1
:10336000656E20696D70726573696F6E005573616B
:103370007469206E656C6C61207374616D7061009E
:10338000506F757A69746520626568656D2074692F
:10339000736B75005573656420647572696E672080
:1033A0007072696E740046696C616D656E7420653B
:1033B0006E746C6164656E0057796A61632066693A
:1033C0006C616D656E7400536F6C74617220666918
:1033D0006C616D656E746F00536361726963612027
:1033E00066696C616D656E746F0056796A6D6F7594
:1033F000742066696C616D656E7400556E6C6F61EA
:10340000642066696C616D656E740046696C616DFF
:10341000656E742061757377657266656E005779A5
:10342000737577616D2066696C616D656E740053AC
:103430006F6C74616E646F2066696C616D656E742B
:103440006F0052696C6173632E2066696C616D65F3
:103450006E746F005679736F7576616D2066696C56
:10346000616D656E7400556E6C6F6164696E672086
:1034700066696C616D656E7400556E6B6E6F776E0C
:1034800020636F6D6D616E643A2022004665696E3F
:1034900065696E7374656C6C756E67004E617374EC
:1034A000726F696300416A75737461720052656777
:1034B0006F6C61004C616469740054756E650053F3
:1034C00044204B61727465205B466C61736841698E
:1034D000725D006B617274612053445B466C73686B
:1034E0004169725D0053442063617264205B466CE5
:1034F00073684169725D005344204B6172746520AA
:103500005B6E6F726D616C5D006B617274612053F4
:1035100044205B6E6F726D616C5D0053442063618B
:103520007264205B6E6F726D616C5D0054656D70CE
:103530002E204B616C2E205B4F4E5D004369657001
:103540006C2E206B616C2E205B4F4E5D0043616CD6
:103550002E2074656D702E205B4F4E5D0043616CB4
:103560002E2074656D702E205B4F4E5D005465708B
:103570006C2E206B616C2E205B4F4E5D0054656D90
:10358000702E2063616C2E205B4F4E5D0054656D84
:10359000702E204B616C2E205B4F46465D004369C8
:1035A00065706C2E206B616C2E205B4F46465D0073
:1035B00043616C2E2074656D702E205B4F46465D16
:1035C0000043616C2E2074656D702E205B4F464663
:1035D0005D005465706C2E206B616C2E205B4F4635
:1035E000465D0054656D702E2063616C2E205B4F2C
:1035F00046465D0054656D702E204B616C696272A9
:10360000696572756E67206665727469672E204BF6
:103610006C69636B656E20756D2077656974657282
:10362000207A7520676568656E2E00436965706C49
:103630006E61206B616C69627261636A61207A619C
:103640006B6F6E637A6F6E612E204B6F6E74796E46
:1036500075756A2070727A796369736B69656D003C
:1036600043616C69627261636F6E2074656D706531
:10367000726174757261207465726D696E616461E6
:103680002E2050726573696F6E6172207061726175
:1036900020636F6E74696E7561722E005461726181
:1036A000747572612074656D706572617475726194
:1036B000207465726D696E6174612E204661726559
:1036C00020636C69636B2070657220636F6E746930
:1036D0006E756172652E005465706C6F746E692032
:1036E0006B616C69627261636520646F6B6F6E639E
:1036F000656E612E20506F6B726163756A74652010
:10370000737469736B656D20746C616369746B614C
:103710002E0054656D706572617475726520636109
:103720006C6962726174696F6E2069732066696E7C
:1037300069736865642E20436C69636B20746F2025
:10374000636F6E74696E75652E0054656D70204BE5
:10375000616C69622E202020202020202020004340
:103760006965706C2E206B616C2E2020202020203B
:103770002020200043616C2E2074656D702E202067
:1037800020202020202020200043616C2E20746502
:103790006D702E2020202020202020202000546525
:1037A000706C2E206B616C2E202020202020202089
:1037B00020200054656D702E2063616C2E20202027
:1037C000202020202020200054656D7065726174D7
:1037D00075720054656D7065726174757261005424
:1037E000656D70657261747572610054656D7065A8
:1037F000726174757261005465706C6F746100540D
:10380000656D706572617475726500506F6D6F6380
:1038100000536F706F72746500506F64706F7261E7
:1038200000537570706F727400447275636B206121
:10383000626272656368656E005A6174727A796D4E
:103840006163206472756B00446574656E657220F7
:10385000696D70726573696F6E0041727265737421
:1038600061207374616D7061005A6173746176696F
:1038700074207469736B0053746F70207072696E7A
:103880007400474553544F5050542E20005041521D
:103890004144410041525245535441544F2E00532C
:1038A000544F505045442E2000537465707261741B
:1038B0006520746F6F20686967683A20004973203B
:1038C000737465656C207368656574206F6E20681D
:1038D0006561746265643F00546F74616C65204477
:1038E0007275636B7A6569743A00437A6173206319
:1038F000616C6B6F77697479203A005469656D70FB
:103900006F20746F74616C203A0054656D706F2085
:103910007374616D706120746F743A0043656C6BF1
:103920006F767920636173203A00546F74616C2064
:103930007072696E742074696D65203A0047657312
:10394000616D7466696C616D656E743A0046696C90
:10395000616D656E74206C61637A6E6965203A00F2
:1039600046696C616D656E746F20746F74616C3A3A
:103970000046696C616D656E746F20746F743A00F7
:1039800046696C616D656E742063656C6B656D2056
:103990003A00546F74616C2066696C616D656E7479
:1039A000203A00447275636B7A6569743A2020008E
:1039B000437A6173206472756B75203A202000543D
:1039C00069656D706F20646520696D702E3A0054D2
:1039D000656D706F206469207374616D70613A0069
:1039E000436173207469736B75203A202000507214
:1039F000696E742074696D653A20200046696C61B7
:103A00006D656E747665726272617563683A0046C0
:103A1000696C616D656E74203A20200046696C61A6
:103A20006D656E746F203A20200046696C616D658B
:103A30006E746F20757361746F3A0046696C616DC6
:103A4000656E74203A20200046696C616D656E7465
:103A500020757365643A202000537461746973742F
:103A6000696B656E200053746174797374796B614E
:103A70002020004573746164697374696361202058
:103A80000053746174697374696368650053746189
:103A900074697374696B6120200053746174697375
:103AA000746963732020004572726F72202D207339
:103AB0007461746963206D656D6F727920686173DC
:103AC000206265656E206F766572777269747465C1
:103AD0006E00476573636877696E6469676B6569D3
:103AE0007400507265646B6F73630056656C6F632E
:103AF000696461640056656C6F6369746100527932
:103B000063686C6F73740053706565640020536F55
:103B1000667477617265205265736574004C6569DF
:103B2000636874657220536368722E3A004C656B4B
:103B30006B696520736369656369653A00496E6303
:103B40006C2E206C6567676572613A004C65686B26
:103B500065207A6B6F73656E693A00536C696768AC
:103B60007420736B65773A004D6F646520202020C8
:103B7000205B6C656973655D004D6F6420202020BB
:103B80002020205B63696368795D004D6F646F205E
:103B900020205B73696C656E63696F5D004D6F64B7
:103BA0006F205B73696C656E7A696F736F5D004D32
:103BB0006F64202020202020205B74696368795D79
:103BC000004D6F646520202020205B73696C656E5A
:103BD000745D004D6F6465205B486F6865204C65BF
:103BE0006973745D004D6F64205B77207779646141
:103BF0006A6E6F73635D004D6F646F205B72656EFC
:103C0000642E706C656E6F5D004D6F6465202020C2
:103C10002020205B666F7274655D004D6F6420200C
:103C20005B7679732E2076796B6F6E5D004D6F64D5
:103C300065205B6869676820706F7765725D004515
:103C40006E64736368616C74657220537461742E62
:103C500000506F6B617A206B72616E636F776B6976
:103C600000456E73656E6120746F70652066696EC5
:103C7000616C00537461746F2066696E65636F7266
:103C800073610053746176206B6F6E632E207370C6
:103C9000696E2E0053686F7720656E642073746FB1
:103CA000707300536368776572657220536368723E
:103CB0002E3A004F7374726520736369656369659A
:103CC0003A00496E632E2072696C6576616E746588
:103CD0003A0054657A6B65207A6B6F73656E693A4A
:103CE0000053657665726520736B65773A0054659D
:103CF0006D702E2065696E7365747A656E005573FC
:103D000074617769632074656D7065726174757232
:103D1000650045737461626C656365722074656DDE
:103D2000702E3A00496D706F7374612074656D7008
:103D300065726174757261004E6173746176746549
:103D4000207465706C6F74753A00536574207465E7
:103D50006D70657261747572653A0045696E737451
:103D6000656C6C756E67656E005573746177696517
:103D70006E696100436F6E66696775726163696F32
:103D80006E00496D706F7374617A696F6E69004E71
:103D90006173746176656E690053657474696E67EA
:103DA00073005665726472616874756E67666568E3
:103DB0006C657200426C616420706F6C61637A653F
:103DC0006E6961004572726F7220646520636F6E68
:103DD0006578696F6E004572726F7265206361620B
:103DE0006C616767696F004368796261207A61700E
:103DF0006F6A656E6900576972696E6720657272D5
:103E00006F720053656C627374746573742073749D
:103E100061727420004175746F74657374207361EE
:103E20006C696461004176766961206175746F74B4
:103E30006573740053656C662074657374207374C5
:103E40006172742020004269747465207072756517
:103E500066653A00536B6F6E74726F6C756A203AC8
:103E600000436F6E74726F6C61203A005665726920
:103E70006669636172653A005A6B6F6E74726F6C3B
:103E8000756A7465203A00506C65617365206368DB
:103E900065636B203A0053656C6273747465737468
:103EA000204F4B004175746F74657374204F4B0045
:103EB00053656C662074657374204F4B004E6963C4
:103EC000687420616E67657363686C6F7373656E89
:103ED000004E696520706F646C61637A6F6E6F204D
:103EE0002020004E6F2068617920636F6E657869CD
:103EF0006F6E2020004E6F6E20636F6E6E65737361
:103F00006F004E657A61706F6A656E6F20202020A9
:103F1000004E6F7420636F6E6E656374656400534A
:103F2000696C6E696B004D6F746F7265004D6F74D4
:103F30006F720043616C656E742E2F5465726D69EB
:103F400073746F720052697363616C642E2F5465D1
:103F5000726D6973742E004865617465722F5468C0
:103F600065726D6973746F72004C75656674657205
:103F70007465737400546573742077656E74796C1E
:103F800061746F726100546573742064656C20768F
:103F9000656E74696C61646F720050726F76612037
:103FA00064656C2076656E74696C61746F72005420
:103FB0006573742076656E74696C61746F727500D8
:103FC00046616E20746573740053656C627374741B
:103FD000657374206D6973736C756E672E0053651D
:103FE0006C6674657374206E69657564616E7900C2
:103FF0004175746F746573742066616C6C61646F75
:10400000004175746F746573742066616C6C6974BB
:104010006F0053656C66746573742073656C6861BA
:104020006C20200053656C6674657374206661694A
:104030006C65642020004C696E6B6572204C756560
:10404000667465723F004C6577792077656E7420E1
:104050006E61206479737A653F0056656E742E2018
:10406000656E206C6120697A673F0056656E74202A
:1040700053582073756C6C277567656C6C6F3F00C7
:104080004C6576792076656E74206E612074727945
:104090007363653F004C65667420686F74656E6479
:1040A0002066616E3F0053656C62746573742046D0
:1040B00065686C657221004175746F746573742056
:1040C0006572726F7221004175746F74657374202C
:1040D0006E6567617469766F0053656C66746573AD
:1040E00074206572726F72202100456E6465206EC7
:1040F0006963687420676574726F662E00546F7010
:10410000652066696E2E206E6F20746F632E0046E8
:10411000696E65632E2066756F726920706F722EEE
:1041200000456E6473746F70206E6F7420686974DC
:1041300000456E64736368616C74657200546F70DF
:1041400065732066696E616C0046696E65636F72A7
:1041500073612028322900456E6473746F70730098
:10416000546F70652066696E616C0046696E6563A8
:104170006F72736100456E6473746F7000566F7276
:104180006465726572204C7565667465723F005097
:10419000727A6F646E692077656E742E2064727512
:1041A0006B753F0056656E742E20616C20667265DB
:1041B0006E74653F0056656E742064692073746187
:1041C0006D706120616E742E3F00507265646E697F
:1041D000207469736B6F76792076656E743F004644
:1041E000726F6E74207072696E742066616E3F002B
:1041F000507275656665205A20416368736520209A
:104200002020004B6F6E74726F6C61205A206178B1
:104210006973202000436F6E74726F6C2064656C4C
:1042200020656A65205A0056657269666963612077
:1042300061737365205A004B6F6E74726F6C6120EE
:104240005A2061786973202000436865636B696E4A
:1042500067205A2061786973202000507275656666
:1042600065205920416368736520202020004B6F32
:104270006E74726F6C612059206178697320200020
:10428000436F6E74726F6C2064656C20656A652084
:1042900059005665726966696361206173736520B0
:1042A00059004B6F6E74726F6C6120592061786990
:1042B00073202000436865636B696E672059206135
:1042C000786973202000507275656665205820411A
:1042D0006368736520202020004B6F6E74726F6CD2
:1042E0006120582061786973202000436F6E7472DA
:1042F0006F6C2064656C20656A6520580056657295
:10430000696669636120617373652058004B6F6E45
:1043100074726F6C612058206178697320200043AB
:104320006865636B696E6720582061786973202027
:104330000050727565666520486F74656E64004B49
:104340006F6E74726F6C6120686F74656E6420208C
:1043500000436F6E74726F6C20686F74656E6420BA
:10436000005665726966696361207567656C6C6F7C
:10437000004B6F6E74726F6C6120686F74656E6451
:10438000202000436865636B696E6720686F746501
:104390006E6420200050727565666520456E6473FA
:1043A0006368616C7465722020004B6F6E74726F6D
:1043B0006C6120656E6473746F707300436F6E740C
:1043C0002E20746F7065732066696E616C0056658F
:1043D0007269666963612066696E65636F72736195
:1043E000004B6F6E74726F6C6120656E6473746FD6
:1043F000707300436865636B696E6720656E6473F4
:10440000746F7073005072FE20426564202020207B
:1044100020202020004B6F6E74726F6C61206265EB
:1044200064202020202000436F6E74726F6C206423
:10443000652063616D61005665726966696361201C
:104440006C6574746F004B6F6E74726F6C61206278
:104450006564202020202000436865636B696E67D7
:1044600020626564202020202000416C6C65732050
:1044700072696368746967202020200057737A7915
:1044800073746B6F204F4B20202020202000546F2E
:10449000646F2062696520004E657373756E2065D8
:1044A00072726F726500567365204F4B202020207A
:1044B0002020202020202000416C6C20636F72722D
:1044C0006563742020202020200043616D612F430C
:1044D000616C656E7461646F72004C6574746F2FEB
:1044E00052697363616C642E00426564202F20481A
:1044F00065617465720041786973206C656E6774DC
:104500006800417869730053656C627374746573F5
:104510007420202020202020004175746F74657362
:1045200074004175746F746573740053656C6674C0
:1045300065737420202020202020202000577269DD
:1045400074696E6720746F2066696C653A20007626
:104550006F6C756D652E696E6974206661696C6536
:1045600064002053697A653A2000534420656E74D4
:104570006665726E7420004B617274612077796A8F
:10458000657461005461726A657461207265746952
:10459000726164610053442072696D6F73736100CE
:1045A0004B617274612076796A6D75746100436144
:1045B00072642072656D6F7665640053442070727A
:1045C000696E74696E67206279746520006F70652A
:1045D0006E206661696C65642C2046696C653A20C2
:1045E000006F70656E526F6F74206661696C6564F0
:1045F0000053442065696E67657365747A74004B77
:104600006172746120776C6F7A6F6E6100546172B1
:104610006A65746120696E736572746164610053C8
:104620004420696E736572697461004B61727461D4
:1046300020766C6F7A656E61004361726420696EEA
:1046400073657274656400534420696E69742066F2
:1046500061696C0046696C652073656C656374659F
:10466000640046696C65206F70656E65643A200071
:104670006572726F722077726974696E6720746FE9
:104680002066696C650053442063617264206F6B1F
:104690000043616E6E6F7420656E74657220737571
:1046A000626469723A20005265636874733A00501C
:1046B000726177793A004465737472613A0050729E
:1046C0006176793A0052696768743A00447275639A
:1046D0006B20776569746572676568656E00577AE7
:1046E0006E617769616E6965206472756B750052E1
:1046F00065616E7564617220696D70726573696F52
:104700006E005374616D706120696E207269707201
:10471000657361004F626E6F766F76616E692074AB
:1047200069736B7500526573756D696E6720707281
:10473000696E7400447275636B20666F727467658E
:104740007365747A7400577A6E6F7769656E696500
:10475000206472756B7500526573756D69656E6462
:104760006F20696D70726573696F6E005269707247
:10477000656E6469207374616D7061004F626E6F65
:1047800076656E69207469736B7500526573756D1B
:10479000696E67207072696E7400466F727473651B
:1047A000747A656E004B6F6E74796E756F776163A6
:1047B000005265616E7564617220696D7072657317
:1047C0002E0052697072656E6469207374616D7039
:1047D0006100506F6B7261636F7661740052657334
:1047E000756D65207072696E7400526573656E64D4
:1047F0003A2000506C656173652072656D6F766557
:1048000020737465656C2073686565742066726FCB
:104810006D20686561746265642E00426C61636B33
:104820006F7574206F636375727265642E205265B4
:10483000636F766572207072696E743F00526563B3
:104840006F766572696E67207072696E74202020C1
:104850002000686F77746F2E707275736133642EE9
:10486000637A00686F77746F2E707275736133644A
:104870002E637A00686F77746F2E70727573613370
:10488000642E636F6D00666F72756D2E7072757336
:104890006133642E637A00666F72756D2E70727567
:1048A000736133642E637A00666F72756D2E707259
:1048B00075736133642E636F6D007072757361334D
:1048C000642E637A00707275736133642E637A00AC
:1048D000707275736133642E636F6D00447275631B
:1048E0006B207061757369657274004472756B201A
:1048F0007A6174727A796D616E7900496D70726552
:1049000073696F6E20656E207061757361005374FA
:10491000616D706120696E2070617573610054690A
:10492000736B20706F7A6173746176656E0050727C
:10493000696E742070617573656400447275636B91
:10494000206162676562726F6368656E00447275AC
:104950006B2070727A657277616E7900496D707242
:104960006573696F6E2063616E63656C616461007D
:104970005374616D70612061626F7274697461005B
:104980005469736B20707265727573656E00507236
:10499000696E742061626F72746564005072696E32
:1049A00074657220646973636F6E6E6563746564A9
:1049B00000756E64204B6E6F70662064727565635F
:1049C0006B656E004E616369736E696A2070727AFE
:1049D000796369736B0050756C73617220656C202C
:1049E0006D616E646F006520636C696363617265FD
:1049F000206D616E6F706F6C6100612073746973FC
:104A00006B6E65746520746C616369746B6F0061B3
:104A10006E6420707265737320746865206B6E6FAE
:104A20006200447565736520566F72776165726DBB
:104A3000656E004E6167727A656A206479737A6583
:104A4000210050726563616C656E746172206578D7
:104A5000747275736F72005072657269732E20756F
:104A600067656C6C6F210050726564656872656A79
:104A7000746520747279736B752100507265686576
:104A8000617420746865206E6F7A7A6C65210056B7
:104A90006F72776165726D656E0047727A616E69DB
:104AA000650050726563616C656E7461720050726E
:104AB0006572697363616C646100507265646568F6
:104AC000726576005072656865617400506F776535
:104AD0007255700042697474652077617274656EF6
:104AE0000050726F737A6520637A656B6163005062
:104AF0006F72204661766F722045737065726172C5
:104B000000417370657474610050726F73696D2039
:104B100063656B656A746500506C656173652077C9
:104B2000616974004269747465206C6164656E200B
:104B3000536965207A756572737420504C41204624
:104B4000696C616D656E742E0050726F737A652C9E
:104B5000206E616A7069657277207A616C61647534
:104B60006A2066696C616D656E7420504C412E0040
:104B7000436172676120656C2066696C616D656E6A
:104B8000746F20504C41207072696D65726F207097
:104B90006F72206661766F722E00506572206661BA
:104BA000766F7265207072696D61206361726963EE
:104BB0006172652066696C616D656E746F206469F1
:104BC00020504C412E004E656A6472697665207AE9
:104BD00061766564746520504C412066696C616D36
:104BE000656E742070726F73696D2E00506C656114
:104BF0007365206C6F616420504C412066696C6164
:104C00006D656E742066697273742E00497374202A
:104C1000504C412046696C616D656E742067656C0F
:104C20006164656E3F004669616C6D656E7420500D
:104C30004C41206A657374207A616C61646F77619E
:104C40006E793F004573746120656C2066696C6104
:104C50006D656E746F20504C4120636172676164B2
:104C60006F3F00496C20504C412065207374617483
:104C70006F20636172696361746F3F004A65205001
:104C80004C412066696C616D656E74207A61766551
:104C900064656E3F00497320504C412066696C6129
:104CA0006D656E74206C6F616465643F00202050F8
:104CB0006C616E6E65724275666665724279746586
:104CC000733A2000506C6561736520706C61636598
:104CD00020737465656C207368656574206F6E2041
:104CE000686561746265642E0050494E44412065D8
:104CF00072776165726D656E0047727A616E696583
:104D00002050494E44410043616C656E74616E648D
:104D10006F2050494E44410052697363616C642EA8
:104D20002050494E4441004E6168726976616E6957
:104D30002050494E44410050494E4441204865614D
:104D400074696E670054656D706572617475722068
:104D50007775726465206E69636874206B616C6935
:104D600062726965727400436965706C6E61206B74
:104D7000616C69627261636A61206E696520627943
:104D80006C612070727A6570726F7761647A6F6E91
:104D900061004C612074656D70657261747572613B
:104DA0002064652063616C6962726163696F6E2063
:104DB0006E6F206861207369646F20616A75737417
:104DC0006164610054617261747572612064656C24
:104DD0006C612074656D7065726174757261206EAE
:104DE0006F6E20616E636F726120657365677569B0
:104DF0007461005469736B61726E61206E656279D3
:104E00006C61207465706C6F746E65207A6B616C78
:104E10006962726F76616E610054656D7065726172
:104E2000747572652063616C6962726174696F6E1A
:104E300020686173206E6F74206265656E207275E4
:104E40006E2079657400504944204B616C69622E74
:104E5000004B616C2E205049440043616C2E205061
:104E600049442020202020202020202020004361B1
:104E70006C2E2050494400504944206B616C2E2018
:104E80002020202020202020202000504944206382
:104E9000616C2E2020202020202020202020005067
:104EA0004944204B616C69622E20666572746967A3
:104EB000004B616C2E20504944207A616B6F6E6309
:104EC0007A6F6E610043616C2E20504944207465F6
:104ED000726D696E6164610043616C2E20504944BB
:104EE00020636F6D706C65746100504944206B6184
:104EF0006C2E20756B6F6E63656E610050494420A7
:104F000063616C2E2066696E697368656400504940
:104F100044204B616C696272696572756E67004B03
:104F2000616C69627261636A612050494400436147
:104F30006C6962726163696F6E205049440043611D
:104F40006C696272617A696F6E65205049440050E5
:104F50004944206B616C6962726163650050494429
:104F60002063616C6962726174696F6E004472756E
:104F7000636B20756E74657262726563682E005093
:104F8000727A6572776163206472756B0050617527
:104F900073617220696D70726573696F6E004D6523
:104FA00074746920696E20706175736100506F7A46
:104FB00061737461766974207469736B00506175F4
:104FC0007365207072696E74004C6567656E20654C
:104FD000696E20426C617474205061706965722042
:104FE000756E74657220646965204475657365200B
:104FF0007761656872656E6420646572204B616CD0
:10500000696272696572756E672064657220657287
:105010007374656E20342050756E6B74652E205746
:10502000656E6E20646965204475657365206461F2
:1050300073205061706965722065696E6B6C656D77
:105040006D742C20447275636B657220736F666F8C
:10505000727420617573736368616C74656E00555A
:105060006D69657363206B6172746B65207061702C
:1050700069657275206E6120706F646B6C6164632A
:105080006520692074727A796D616A20706F64207E
:105090006479737A6120706F64637A617320706FD2
:1050A0006D69617275207069657277737A7963686A
:1050B00020342070756E6B746F772E204A65736C88
:1050C00069206479737A61207A616861637A7920F2
:1050D0006F207061706965722C2077796C61637ADA
:1050E000206472756B61726B652E00436F6C6F6329
:1050F000617220756E6120686F6A6120646520703E
:105100006170656C20736F627265206C61207375CD
:10511000706572666963696520646520696D707287
:105120006573696F6E20647572616E7465206C6161
:105130002063616C6962726163696F6E20646520CF
:105140006C6F73207072696D65726F73203420709C
:10515000756E746F732E205369206C6120626F71BD
:1051600075696C6C61206D7565766520656C207065
:105170006170656C2C2061706167617220696D706F
:105180007265736F726120696E6D656469617461C7
:105190006D656E74652E00506F72726520756E209D
:1051A000666F676C696F20736F74746F206C2775FE
:1051B00067656C6C6F20647572616E7465206C61DC
:1051C0002063616C696272617A696F6E65206465E3
:1051D00069207072696D6920342070756E74692E53
:1051E00020496E206361736F206C277567656C6C56
:1051F0006F206D756F766120696C20666F676C69D2
:105200006F20737065676E6572652070726F6E7463
:10521000616D656E7465206C61207374616D706181
:105220006E74652E00556D697374657465206C69C4
:10523000737420706170697275206E6120706F6484
:105240006C6F7A6B752061207564727A756A74650B
:10525000206A656A20706F6420747279736B6F7551
:1052600020626568656D206D6572656E692070727B
:10527000766E696368203420626F64752E20506FEB
:105280006B756420747279736B61207A61636879DD
:1052900074692070617069722C207679706E657403
:1052A00065207469736B61726E752E00506C61635A
:1052B000652061207368656574206F662070617079
:1052C000657220756E64657220746865206E6F7AF1
:1052D0007A6C6520647572696E67207468652063F6
:1052E000616C6962726174696F6E206F66206669B5
:1052F000727374203420706F696E74732E20496647
:1053000020746865206E6F7A7A6C652063617463BF
:10531000686573207468652070617065722C2070F8
:105320006F776572206F6666207468652070726999
:105330006E74657220696D6D6564696174656C7900
:105340002E006F6B004F6666004B65696E652042EC
:1053500065776567756E672E0053696E206D6F7691
:10536000696D69656E746F004E657373756E206D3F
:105370006F76696D656E746F2E004E6F206D6F765F
:10538000652E004B65696E65205344204B61727435
:1053900065004272616B206B617274792053440026
:1053A0004E6F20686179207461726A657461205360
:1053B00044004E657373756E61205344005A6164F6
:1053C0006E61205344206B61727461004E6F2053F4
:1053D00044206361726400447565736500447973A9
:1053E0007A6100426F7175696C6C61005567656C1C
:1053F0006C6F00547279736B61004E6F7A7A6C65D2
:105400000046696C2E206E696368742067656C6164
:1054100064656E004272616B2066696C616D656ED9
:1054200074750046696C2E206E6F20696E74726F01
:1054300064756369646F0046696C2E206E6F6E2020
:10544000636172696361746F0046696C616D656E5A
:1054500074206E657A61766564656E0046696C617C
:105460006D656E74206E6F74206C6F61646564008E
:10547000466172626520756E6B6C6172004B6F6C79
:105480006F72207A616E6965637A79737A2E004350
:105490006F6C6F72206E6F20686F6D6F67656E65E1
:1054A0006F00436F6C6F7265206E6F6E2070757247
:1054B0006F004261727661206E656E692063697368
:1054C000746100436F6C6F72206E6F7420636C6543
:1054D0006172004E65696E004E6965004E65004E52
:1054E0006F00426974746520616B7475616C6973D7
:1054F000696572656E2E0050726F737A65207A61ED
:105500006B7475616C697A6F776163004163747560
:10551000616C697A617220706F72206661766F7259
:1055200000507265676120616767696F726E612EF6
:105530000050726F73696D20616B7475616C697A6C
:10554000756A74652E00506C6561736520757067AF
:10555000726164652E004E657565204669726D77CF
:105560006172652056657273696F6E20766572662A
:105570007565676261723A005779737A6C61206E63
:105580006F776120776572736A61206669726D77E3
:105590006172653A004E7565766F206669726D7747
:1055A00061726520646973706F6E69626C653A0040
:1055B0004E756F76612076657273696F6E652064D3
:1055C000656C206669726D776172652064697370BD
:1055D0006F6E6962696C65005679736C61206E6FDD
:1055E0007661207665727A65206669726D77617280
:1055F000653A004E6577206669726D776172652045
:1056000076657273696F6E20617661696C61626C38
:10561000653A00426577656765205A0050727A6581
:1056200073756E6163205A004D6F766572205A0063
:105630004D756F7669205A00506F73756E6F757473
:10564000205A004D6F7665205A0042657765676580
:1056500020590050727A6573756E61632059004D50
:105660006F7665722059004D756F7669205900502C
:105670006F73756E6F75742059004D6F7665205984
:105680000042657765676520580050727A657375CA
:105690006E61632058004D6F7665722058004D751D
:1056A0006F7669205800506F73756E6F757420584F
:1056B000004D6F76652058004578747275697200E8
:1056C0004D756F7669204573747275736F726500DE
:1056D00045787472756465720041636873626577BA
:1056E0006567756E670052756368206F7369004D5A
:1056F0006F76657220656A6573004D756F766920F7
:105700006173736500506F73756E6F7574206F737E
:1057100075004D6F76652061786973004D6573681B
:10572000206C6976656C2E206C6574746F004D6515
:10573000736820426564204C6576656C696E67000D
:105740004B616C696272696572756E67004B616C62
:1057500069627261636A610043616C69627261636C
:10576000696F6E0043616C696272617A696F6E6520
:10577000004B616C6962726163650043616C6962D0
:10578000726174696F6E0020766F6E203900207A26
:1057900020390020646520390020737520390020ED
:1057A0007A203900206F662039004D657373656E6D
:1057B00020646572205265666572656E7A686F65F1
:1057C000686520646573204B616C696272696572FB
:1057D00070756E6B746573004F6B7265736C616D81
:1057E000207779736F6B6F7363206F646E69657375
:1057F00069656E69612070756E6B7475206B616C84
:105800006962726163796A6E65676F004D6564698C
:1058100072206C6120616C747572612064656C200B
:1058200070756E746F206465206C612063616C69B3
:1058300062726163696F6E004D6973757261726542
:10584000206C27616C74657A7A61206469207269C2
:10585000666572696D656E746F2064656C20707525
:105860006E746F2064692063616C696272617A6929
:105870006F6E65004D6572696D2072656665726553
:105880006E636E69207679736B75206B616C6962EB
:105890007261636E69686F20626F6475004D656147
:1058A000737572696E67207265666572656E636591
:1058B00020686569676874206F662063616C69623F
:1058C000726174696F6E20706F696E7400536368E3
:1058D000726165676C6175663A005A6D6965722E12
:1058E00020736369656369653A00496E636C2E20B5
:1058F0006D697375726174613A004D6572656E65AC
:10590000207A6B6F73656E693A004D6561737572CD
:10591000656420736B65773A0048617570746D65D6
:105920006E7565004D656E7520676C6F776E6500EE
:105930004D656E75207072696E636970616C004DA3
:10594000656E75207072696E636970616C65004880
:105950006C61766E69206E616269646B61004D6195
:10596000696E004D32323120496E76616C69642077
:10597000657874727564657220004D323138204943
:105980006E76616C696420657874727564657220E6
:10599000004D32303020496E76616C696420657844
:1059A00074727564657220005265706F7274696EEE
:1059B0006720656E6473746F70207374617475739F
:1059C000004D3131372045727374652D536368691A
:1059D000636874204B616C2E004D313137204B6170
:1059E0006C2E20312E2077617273747779004D31DF
:1059F00031372043616C2E207072696D65726120B1
:105A00006361702E004D3131372043616C2E207060
:105A100072696D6F206C617965722E004D3131377E
:105A2000204B616C2E207072766E692076727374D2
:105A30007679004D313137204669727374206C617C
:105A40007965722063616C2E004649524D57415270
:105A5000455F4E414D453A4D61726C696E2056313D
:105A60002E302E323B20537072696E7465722F6730
:105A700072626C206D617368757020666F7220674A
:105A8000656E36204649524D574152455F55524C3E
:105A90003A68747470733A2F2F6769746875622E50
:105AA000636F6D2F707275736133642F50727573ED
:105AB000612D69332D506C75732F2050524F544F08
:105AC000434F4C5F56455253494F4E3A312E30208A
:105AD0004D414348494E455F545950453A507275BF
:105AE0007361206933204D4B33204558545255443F
:105AF00045525F434F554E543A3120555549443A2B
:105B000030303030303030302D303030302D30309B
:105B100030302D303030302D30303030303030308B
:105B2000303030300A004D31303920496E76616CAA
:105B3000696420657874727564657220004D313037
:105B40003520496E76616C6964206578747275647D
:105B5000657220004D31303420496E76616C696485
:105B600020657874727564657220004C6F736520CF
:105B70005269656D656E73636865696265004B6F38
:105B80006C6F207061736F776500506F6C6561207A
:105B90007375656C74610050756C65676769612029
:105BA0006C656E74610055766F6C6E656E61207207
:105BB000656D656E69636B61004C6F6F7365207016
:105BC000756C6C65790046696C616D656E74206CEE
:105BD0006164656E005770726F7761647A206669E0
:105BE0006C616D656E7400496E74726F6475636983
:105BF000722066696C616D2E004361726963612079
:105C000066696C616D656E746F005A617665737458
:105C10002066696C616D656E74004C6F616420660E
:105C2000696C616D656E740046696C616D656E745A
:105C3000206C65616474005770726F772E206669FE
:105C40006C616D656E747500496E74726F64756316
:105C500069656E646F2066696C616D2E00436172C8
:105C60006963616E646F2066696C616D2E005A61B4
:105C7000766164656E692066696C616D656E7475C8
:105C8000004C6F6164696E672066696C616D656E5A
:105C900074004C61646520466172626500437A79E4
:105CA000737A637A2E206B6F6C6F72750043616D2F
:105CB0006269616E646F20636F6C6F720043617222
:105CC0006963616E646F20636F6C6F726500436916
:105CD0007374656E69206261727679004C6F6164DD
:105CE000696E6720636F6C6F72004C696E6B733AFC
:105CF000004C6577793A0053696E69737472613A42
:105D0000004C6576793A004C6566743A00576165D7
:105D1000686C652053707261636865005779626FC3
:105D200072206A657A796B610043616D62696165B1
:105D300020656C206964696F6D610053656C657ADC
:105D4000696F6E61206C696E677561005679626576
:105D500072206A617A796B610053656C65637420A7
:105D60006C616E677561676500446575747363681F
:105D700000506F6C736B6900457370616E6F6C00DF
:105D80004974616C69616E6F0043657374696E611B
:105D900000456E676C697368004142474542524F47
:105DA0004348454E2E200050415241444120444535
:105DB00020454D455247454E43494100494E2054E8
:105DC000494C542E004B494C4C45442E2000496E02
:105DD00076616C69642065787472756465720046DA
:105DE000696C616D656E742065696E6C6567656E62
:105DF000005770726F7761647A2066696C616D65B7
:105E00006E7400496E74726F64756369722066699E
:105E10006C616D656E746F00496E73657269726551
:105E20002066696C616D656E746F00566C6F7A7474
:105E3000652066696C616D656E7400496E7365728C
:105E4000742066696C616D656E74005072696E7461
:105E50002046414E3A20004E6F7A7A6C65204641CA
:105E60004E3A00457874727564657220696E666F8B
:105E70000020766F6E203400207A20340020646584
:105E8000203400207375203400207A203400206FE5
:105E900066203400566572626573736572756E674D
:105EA00020426564204B616C69627269657270752D
:105EB0006E6B7400506F7072617769616D207072E3
:105EC0006563797A796A6E6F73632070756E6B742F
:105ED00075206B616C6962726163796A6E65676F68
:105EE000004D656A6F72616E646F2063616D612041
:105EF00070756E746F2064652063616C6962726195
:105F000063696F6E0050657266657A696F6E2E20E8
:105F1000696C206C6574746F2070756E746F20648A
:105F2000692063616C696272617A2E005A6C6570D7
:105F300073756A6920707265736E6F7374206B611C
:105F40006C69627261636E69686F20626F6475006C
:105F5000496D70726F76696E672062656420636157
:105F60006C6962726174696F6E20706F696E740023
:105F70004B616C69627269657265205A004B616C95
:105F8000696272756A65205A0043616C6962726168
:105F90006E646F205A0043616C696272616E646F57
:105FA000205A004B616C696272756A69205A00431D
:105FB000616C6962726174696E67205A004B616C32
:105FC000696272696572756E67204F4B004B616C38
:105FD00069627261636A61204F4B0043616C696260
:105FE000726163696F6E204F4B0043616C6962722E
:105FF000617A696F6E65204F4B004B616C6962720C
:10600000616365204F4B0043616C69627261746922
:106010006F6E20646F6E65004B616C6962726965BA
:1060200072656E205A004B616C696272756A205A03
:106030000043616C6962726172205A0043616C694D
:10604000627261205A004B616C6962726F76617492
:10605000205A0043616C696272617465205A004184
:106060007566776165726D656E204F4B0047727A79
:10607000616E6965204F4B2E0043616C656E7461E3
:106080006D69656E746F2066696E616C2E00526971
:106090007363616C642E20636F6D706C65746F0048
:1060A0005A6168726976616E69204F4B2E004865AF
:1060B0006174696E6720646F6E652E004175667746
:1060C0006165726D656E0047727A616E69652E2E2C
:1060D0002E0043616C656E74616E646F2E2E2E000F
:1060E00052697363616C64616D656E746F2E2E2EE0
:1060F000005A6168726976616E6900486561746909
:106100006E670046696C2E2073656E736F72202077
:106110005B6F6E5D0046696C2E2073656E736F72E7
:10612000205B6F66665D002046726565204D656D7B
:106130006F72793A200044657220447275636B6512
:1061400072207775726465206E6F6368206E696374
:106150006874206B616C696272696572742E20428A
:106160006974746520666F6C67656E20536965207D
:1061700064656D2048616E64627563682C204B61B4
:10618000706974656C2046697273742073746570ED
:10619000732C2041627363686E6974742043616C70
:1061A0006962726174696F6E20666C6F772E00444D
:1061B00072756B61726B61206E6965207A6F7374A2
:1061C000616C61206A65737A637A6520736B616CB8
:1061D0006962726F77616E612E2050726F737A659B
:1061E000206B6965726F7761632073696520696EE2
:1061F000737472756B636A612C20726F7A647A694A
:10620000616C205A61637A796E616D792C20706FB0
:1062100064726F7A647A69616C2053656C66746528
:1062200073742E00496D707265736F7261206E6FAA
:1062300020657374612063616C69627261646120BE
:10624000746F64617669612E20506F72206661768A
:106250006F72207573617220656C206D616E75615F
:106260006C2C20656C206361706974756C6F2046BE
:10627000697273742073746570732C2073656C6518
:106280006363696F6E2043616C6962726174696FE8
:106290006E20666C6F772E005374616D70616E7442
:1062A0006520616E636F7261206E6F6E2063616C3A
:1062B0006962726174612E20536920707265676132
:1062C000206469207365677569726520696C206D4B
:1062D000616E75616C652C2063617069746F6C6FA1
:1062E000205052494D492050415353492C20736549
:1062F0007A696F6E652064656C6C612063616C699E
:106300006272617A696F6E652E005469736B617297
:106310006E61206E6562796C61206A6573746520B8
:106320007A6B616C6962726F76616E612E20506F5C
:1063300073747570756A74652070726F73696D20FF
:10634000706F646C65206D616E75616C752C206B6F
:10635000617069746F6C61205A6163696E616D650B
:106360002C206F6473746176656320506F7374754D
:1063700070206B616C6962726163652E0050726996
:106380006E74657220686173206E6F74206265653B
:106390006E2063616C6962726174656420796574F2
:1063A0002E20506C6561736520666F6C6C6F772072
:1063B000746865206D616E75616C2C206368617016
:1063C0007465722046697273742073746570732CDF
:1063D0002073656374696F6E2043616C69627261DA
:1063E00074696F6E20666C6F772E004475726368F7
:1063F000666C7573730050727A65706C79770046BD
:106400006C756A6F00466C7573736F0050727574AB
:106410006F6B00466C6F77004265776567756E67D6
:10642000206265656E64656E004B6F6E637A656EA3
:106430006965206472756B75005465726D2E206DF0
:106440006F76696D69656E746F7300417272657302
:10645000746F20696E20636F72736F00446F6B6F8F
:106460006E636F76616E6920706F68796275004641
:10647000696E697368696E67206D6F76656D656EAC
:1064800074730020766F6E203400207A2034002050
:106490006465203400207375203400207A20340095
:1064A000206F6620340053756368656E2042656412
:1064B000204B616C69627269657270756E6B7400F5
:1064C000537A756B616D2070756E6B7475206B619E
:1064D0006C6962726163796A6E65676F20706F6460
:1064E0006B6C61646B690042757363616E646F20ED
:1064F00063616D612070756E746F206465206361E7
:106500006C6962726163696F6E0052696365726380
:10651000612064656C206C6574746F2070756E7496
:106520006F2064692063616C696272617A2E004831
:106530006C6564616D206B616C69627261636E6928
:1065400020626F6420706F646C6F7A6B79005365A2
:1065500061726368696E67206265642063616C695B
:1065600062726174696F6E20706F696E7400497435
:10657000657261636A612000526569746572616366
:10658000696F6E2000526569746572617A696F6E19
:106590006520004974657261636520004974657205
:1065A0006174696F6E2000446F6E65207361766957
:1065B0006E672066696C652E00446F6E6520707290
:1065C000696E74696E672066696C65004973742032
:1065D0004661726265207265696E3F00437A792078
:1065E0006B6F6C6F72206A65737420637A79737451
:1065F000793F00457320656C206E7565766F20636A
:106600006F6C6F72206E697469646F3F00496C2013
:10661000636F6C6F7265206527206E697469646FA3
:106620003F004A652062617276612063697374611C
:106630003F00497320636F6C6F7220636C656172F9
:106640003F0046696C616D656E742D5765636873B4
:10665000656C0057796D69656E69632066696C6168
:106660006D656E740043616D626961722066696C6C
:10667000616D656E746F0043616D622E2066696C9A
:10668000616D656E746F0056796D656E6974206614
:10669000696C616D656E74004368616E6765206644
:1066A000696C616D656E74004C7565667465722DFC
:1066B00054656D706F00507265646B6F7363207703
:1066C000656E742E0056656C6F6369646164205654
:1066D000656E742E0056656C6F6369746120766513
:1066E0006E742E00527963686C6F73742076656ED9
:1066F000742E0046616E20737065656400656E716E
:106700007565696E67202200456B737472756465E8
:1067100072004578747275736F7200457374727588
:10672000736F7265004578747275646572002045F8
:10673000787465726E616C20526573657400507276
:10674000696E7465722073746F707065642064750F
:106750006520746F206572726F72732E204669789F
:1067600020746865206572726F7220616E64207596
:106770007365204D39393920746F207265737461E7
:1067800072742E202854656D70657261747572651F
:106790002069732072657365742E205365742069B7
:1067A00074206166746572207265737461727469B5
:1067B0006E6729004E6F204C696E65204E756D62C4
:1067C0006572207769746820636865636B73756DA3
:1067D0002C204C617374204C696E653A20004E6F1A
:1067E00020436865636B73756D2077697468206CEE
:1067F000696E65206E756D6265722C204C617374D4
:10680000204C696E653A200020746F6F206C6F6EAB
:106810006720657874727573696F6E207072657623
:10682000656E746564004C696E65204E756D6265B9
:1068300072206973206E6F74204C617374204C69F0
:106840006E65204E756D6265722B312C204C617324
:1068500074204C696E653A20005072696E746572DE
:106860002068616C7465642E206B696C6C2829202B
:1068700063616C6C6564210020636F6C64206578D3
:1068800074727573696F6E2070726576656E74656B
:106890006400636865636B73756D206D69736D610A
:1068A0007463682C204C617374204C696E653A20C7
:1068B000004645484C45523A00424C41443A004556
:1068C00052524F52453A0043485942413A004552CC
:1068D000524F523A00456E642066696C65206C69BF
:1068E0007374006F70656E005452494747455245B6
:1068F0004400656E6473746F7073206869743A2025
:106900000045696E656E204D6F6D656E742062691D
:106910007474652E00456E20657370657261005356
:106920006F7370656E73696F6E652E2E2E00536CDB
:106930006565702E2E2E004D6F746F72656E20612E
:1069400075730057796C61637A79632073696C6E33
:10695000696B6900417061676172206D6F746F725D
:106960006573004469736162696C6974206D6F744A
:106970006F7269005679706E6F7574206D6F746FE9
:1069800072790044697361626C652073746570701C
:1069900065727300446174756D00446174613A00FE
:1069A0004461746100446174756D3A0044617465BA
:1069B0003A00416B7475656C6C65730054796C6B4F
:1069C0006F20616B7475616C6E65004163747561F5
:1069D0006C0041747475616C6500506F757A652048
:1069E000616B7475616C6E690043757272656E746B
:1069F000004372617368206465742E2020205B6FF1
:106A00006E5D004372617368206465742E20205BA4
:106A10006F66665D0020436F756E7420583A2000E3
:106A20005765636873656C206F6B3F0057796D69BC
:106A3000616E61206F6B3F0043616D626961646FDD
:106A400020636F72726563742E3F0043616D6269EB
:106A500061746F20636F72722E3F0056796D656EA0
:106A600061206F6B3F004368616E67656420636FF0
:106A700072726563746C793F0041626B7565686C16
:106A8000656E00577963686C6F647A696300456E60
:106A90006672696172005261666672656464610063
:106AA0005A63686C6164697400436F6F6C646F77DC
:106AB0006E00204C61737420557064617465643A93
:106AC0002000576165686C656E20536965204578C4
:106AD000747275646572005779626965727A2065AF
:106AE0006B7374727564657200456C6567697220BA
:106AF0006578747275736F723A0053656C657A6964
:106B00006F6E61206573747275736F72653A0056AB
:106B10007962657274652065787472756465723A1D
:106B20000043686F6F736520657874727564657271
:106B30003A005765636873656C206572666F6C67B1
:106B4000722E210057796D69616E61206F6B210093
:106B500043616D62696F20636F72726563746F0069
:106B600043616D62696F20726975736369746F2127
:106B7000005A6D656E612075737065736E612100DA
:106B80004368616E67652073756363657373210085
:106B9000447275636B656E20766F6E2053440044BB
:106BA00072756B207A205344004D656E75207461B8
:106BB000726A657461205344005374616D70612082
:106BC0006461205344005469736B207A205344005D
:106BD0005072696E742066726F6D20534400546564
:106BE0006D702E206B616C696272696572656E00F2
:106BF000436965706C6E61206B616C6962722E0016
:106C000043616C6962726163696F6E2074656D7057
:106C10002E0054617261747572612074656D702EFE
:106C2000005465706C6F742E206B616C69627261C8
:106C300063650054656D702E2063616C69627261DA
:106C400074696F6E0043616C6962726174696E672A
:106C5000205A004B616C696272696572656E0053FF
:106C60006B616C6962726F7761630043616C69622A
:106C70007261720043616C696272617265005A6B85
:106C8000616C6962726F7661740043616C696272F3
:106C90006174650052657365742058595A204B61C0
:106CA0006C6962722E005265736574206B616C6949
:106CB00062722E2058595A005265736574205859D3
:106CC0005A206B616C6962722E0052657365742084
:106CD00058595A2063616C6962722E004B616C696D
:106CE0006272696572756E672058595A004B616C03
:106CF00069627261636A612058595A0043616C6924
:106D00006272612058595A0043616C696272612055
:106D100058595A004B616C69627261636520585919
:106D20005A0043616C6962726174652058595A0057
:106D30002042726F776E206F757420526573657490
:106D400000426567696E2066696C65206C697374C2
:106D50000058595A2D4B616C696272696572756E83
:106D60006720756E67656E61752E204C696E6B6568
:106D70007220766F726465726572204B616C696215
:106D80007269657270756E6B7420697374207A75A0
:106D9000207765697420766F726E652E004B616C8A
:106DA00069627261636A612058595A206E6965642C
:106DB0006F6B6C61646E612E204C65777920707208
:106DC0007A65646E692070756E6B74207A6279746E
:106DD00020777973756E6965747920646F2070729D
:106DE0007A6F64752E0043616C696272617A696FB3
:106DF0006E2058595A20636F6D70726F6D6574699B
:106E000064612E2050756E746F2064656C616E74C1
:106E100065726F20697A7175696572646F206E6F33
:106E200020616C63616E7A61626C652E0043616CF7
:106E3000696272617A696F6E652058595A20636F72
:106E40006D70726F6D657373612E2050756E746F07
:106E500020616E746572696F72652073696E697303
:106E600074726F206E6F6E207261676769756E67EE
:106E70006962696C652E004B616C69627261636561
:106E80002058595A206E65707265736E612E204CC1
:106E900065767920707265646E6920626F64206D1A
:106EA0006F63207670726564752E0058595A20639E
:106EB000616C6962726174696F6E20636F6D70726C
:106EC0006F6D697365642E204C6566742066726F01
:106ED0006E742063616C6962726174696F6E207098
:106EE0006F696E74206E6F74207265616368616291
:106EF0006C652E0058595A2D4B616C696272696538
:106F000072756E6720756E67656E61752E20566F9F
:106F10007264657265204B616C696272696572703A
:106F2000756E6B74652073696E64207A7520776561
:106F3000697420766F726E652E004B616C696272A7
:106F40002E2058595A206E6965646F6B6C61646EAF
:106F5000612E2050727A65646E69652070756E6B63
:106F60007479206B616C6962722E205A6279742088
:106F70007779732E20646F2070727A6F64752E009B
:106F800043616C696272617A696F6E2058595A2048
:106F9000636F6D70726F6D65746964612E205075DA
:106FA0006E746F2064656C616E7465726F73206EB1
:106FB0006F20616C63616E7A61626C65732E004351
:106FC000616C696272617A696F6E652058595A20E6
:106FD000636F6D70726F6D657373612E2050756E87
:106FE000746920616E746572696F7269206E6F6E6C
:106FF000207261676769756E676962696C692E00E6
:107000004B616C6962726163652058595A206E65E4
:10701000707265736E612E20507265646E69206BAC
:10702000616C69627261636E6920626F6479206D60
:107030006F63207670726564752E0058595A20630C
:10704000616C6962726174696F6E20636F6D7072DA
:107050006F6D697365642E2046726F6E7420636174
:107060006C6962726174696F6E20706F696E74739F
:10707000206E6F7420726561636861626C652E00BA
:1070800058595A204B616C696272696572756E67F6
:1070900020696E204F72646E756E672E20582F59CE
:1070A0002041636873656E2073696E642065747730
:1070B0006173207363686965662E004B616C696259
:1070C0007261636A612058595A20707261776964ED
:1070D0006C6F77612E204F73696520582F59206C93
:1070E000656B6B6F20736B6F736E652E20446F62E0
:1070F000726120726F626F7461210043616C69621A
:10710000726163696F6E2058595A20636F7272659D
:107110006374612E204C6F7320656A65732058205C
:107120002F205920657374616E206C6967657261E8
:107130006D656E746520696E636C696E61646F73F2
:107140002E204275656E2074726162616A6F210043
:1071500043616C696272617A696F6E2058595A2076
:10716000636F7272657474612E2041737369205865
:107170002F59206C65676765726D656E7465207345
:10718000746F7274692E2042656E20666174746F2C
:1071900021004B616C6962726163652058595A2005
:1071A0007620706F7261646B752E20582F59206F96
:1071B0007379206D69726E65207A6B6F73656E6589
:1071C0002E20446F627261207072616365210058E5
:1071D000595A2063616C6962726174696F6E2061D3
:1071E0006C6C2072696768742E20582F5920617862
:1071F00065732061726520736C696768746C7920AF
:10720000736B657765642E20476F6F64206A6F62C9
:10721000210058595A204B616C6962726965727518
:107220006E6720696E204F72646E756E672E2053F4
:10723000636869656668656974207769726420614E
:1072400075746F6D617469736368206B6F727269B6
:1072500067696572742E004B616C69627261636A62
:10726000612058595A207072617769646C6F776138
:107270002E20536B6F737920626564612061757491
:107280006F6D617479637A6E6965207779726F7753
:107290006E616E652070727A79206472756B752EDE
:1072A0000043616C6962726163696F6E2058595A5C
:1072B00020636F7272656374612E204C6120696E69
:1072C000636C696E6163696F6E20736520636F72B2
:1072D000726567697261206175746F6D617469634D
:1072E000616D656E74652E0043616C696272617ACE
:1072F000696F6E2058595A20636F72726574746199
:107300002E204C6120646973746F7273696F6E65AF
:1073100020766572726127206175746F6D61746982
:1073200063616D656E746520636F6D70656E73610A
:1073300074612E004B616C696272616365205859FB
:107340005A207620706F7261646B752E205A6B6FB5
:1073500073656E692062756465206175746F6D6117
:107360007469636B79207679726F766E616E6F20C7
:10737000707269207469736B752E0058595A2063B6
:10738000616C6962726174696F6E20616C6C2072ED
:10739000696768742E20536B65772077696C6C2061
:1073A000626520636F7272656374656420617574D1
:1073B0006F6D61746963616C6C792E0058595A2D38
:1073C0004B616C696272696572756E67206665688B
:1073D0006C67657363686C6167656E2E20426564D7
:1073E0002D4B616C69627269657270756E6B742089
:1073F0006E6963687420676566756E64656E2E00DD
:107400004B616C6962722E2058595A206E696575FD
:1074100064616E612E204B616C6962726163796A8E
:107420006E792070756E6B7420706F646B6C616424
:107430006B69206E69657A6E616C657A696F6E79C9
:107440002E0043616C6962726163696F6E205859E6
:107450005A2066616C6C6164612E2050756E746F89
:10746000732064652063616C6962726163696F6E29
:1074700020656E206C612063616D61206E6F2065F8
:107480006E636F6E747261646F732E0043616C691A
:107490006272617A696F6E652058595A2066616C14
:1074A0006C6974612E20496C2070756E746F206455
:1074B000692063616C696272617A696F6E652073BD
:1074C000756C206C6574746F206E6F6E206527205C
:1074D000737461746F2074726F7661746F2E004BD9
:1074E000616C6962726163652058595A2073656CDA
:1074F00068616C612E204B616C69627261636E69B8
:1075000020626F6420706F646C6F7A6B79206E6597
:107510006E616C657A656E2E0058595A2063616CF5
:107520006962726174696F6E206661696C65642E50
:10753000204265642063616C6962726174696F6E78
:1075400020706F696E7420776173206E6F7420668F
:107550006F756E642E0058595A2D4B616C696272BA
:10756000696572756E67206F6B2E20582F592D41FB
:10757000636873656E2073696E642073656E6B72E9
:1075800065636874207A7565696E616E6465722ED4
:1075900020476C7565636B77756E73636821004B6C
:1075A000616C69627261636A612058595A206F6B1D
:1075B0002E204F73696520582F59207361207072F7
:1075C0006F73746F7061646C652E2047726174759F
:1075D0006C61636A65210043616C69627261636911
:1075E0006F6E2058595A206F6B2E20456A657320A4
:1075F000582F592070657270656E646963756C618F
:107600007265732E2046656C696369746163696F86
:107610006E6573210043616C696272617A696F6E95
:10762000652058595A204F4B2E20476C69206173B2
:10763000736920582F5920736F6E6F2070657270B8
:10764000656E6469636F6C6172692E20436F6D7043
:107650006C696D656E746921004B616C6962726161
:1076600063652058595A207620706F7261646B757B
:107670002E20582F59206F7379206A736F75206BF5
:107680006F6C6D652E2047726174756C756A692127
:107690000058595A2063616C6962726174696F6E37
:1076A000206F6B2E20582F592061786573206172EE
:1076B000652070657270656E646963756C61722EA9
:1076C00020436F6E67726174756C6174696F6E735D
:1076D000210058595A2D4B616C6962726965727547
:1076E0006E67206665686C67657363686C61676563
:1076F0006E2E204269747465207363686175656ECF
:107700002053696520696E206461732048616E644E
:10771000627563682E004B616C69627261636A61B5
:107720002058595A206E6965706F776965647A6967
:107730006F6E612E205370726177647A696320776F
:1077400020696E737472756B636A692E0043616C95
:107750006962726163696F6E2058595A2066616C64
:107760006C6164612E20436F6E73756C746172205E
:10777000656C206D616E75616C20706F7220666142
:10778000766F722E0043616C696272617A696F6E06
:10779000652058595A2066616C6C6974612E2053BB
:1077A0006920707265676120646920636F6E73750C
:1077B0006C7461726520696C206D616E75616C65B9
:1077C0002E004B616C6962726163652058595A20C2
:1077D00073656C68616C612E204E61686C65646EC7
:1077E00065746520646F206D616E75616C752E0027
:1077F00058595A2063616C6962726174696F6E20B6
:107800006661696C65642E20506C656173652063E8
:107810006F6E73756C7420746865206D616E756130
:107820006C2E0058595A2D4B616C696272696572F1
:10783000756E67206665686C67657363686C616701
:10784000656E2E204C696E6B657220766F72646572
:10785000726572204B616C69627269657270756ED7
:107860006B7420697374207A75207765697420764B
:107870006F726E652E004B616C6962722E205859D2
:107880005A206E69657564616E612E204C6577794A
:107890002070727A65646E692070756E6B74207AE0
:1078A00062797420646F2070727A6F64752E20572D
:1078B00079726F776E6163206472756B61726B654C
:1078C0002E0043616C6962726163696F6E20585962
:1078D0005A2066616C6C61642E2050756E746F2046
:1078E00064656C616E7465726F20697A7175696523
:1078F00072646F206E6F20616C63616E7A61626C7E
:10790000652E0043616C696272617A696F6E6520F1
:1079100058595A2066616C6C6974612E2050756EDE
:10792000746F20616E746572696F72652073696E21
:10793000697374726F206E6F6E207261676769750C
:107940006E676962696C652E004B616C6962726179
:1079500063652058595A2073656C68616C612E20EC
:107960004C65767920707265646E6920626F642060
:107970006D6F63207670726564752E2053726F761A
:107980006E656A7465207469736B61726E752E0022
:1079900058595A2063616C6962726174696F6E2014
:1079A0006661696C65642E204C6566742066726F32
:1079B0006E742063616C6962726174696F6E2070AD
:1079C0006F696E74206E6F742072656163686162A6
:1079D0006C652E0058595A2D4B616C69627269654D
:1079E00072756E67206665686C67657363686C6145
:1079F00067656E2E20566F7264657265204B616CF0
:107A000069627269657270756E6B74652073696EF8
:107A100064207A75207765697420766F726E652EA2
:107A2000004B616C6962722E2058595A206E69654C
:107A30007564616E612E2050727A65642E207075B7
:107A40006E6B7479206B616C6962722E207A627938
:107A50007420646F2070727A6F64752E205779726B
:107A60006F776E6163206472756B61726B652E0057
:107A700043616C6962726163696F6E2058595A2064
:107A800066616C6C61642E2050756E746F20646545
:107A90006C616E7465726F73206E6F20616C6361D0
:107AA0006E7A61626C65732E0043616C696272610B
:107AB0007A696F6E652058595A2066616C6C6974DA
:107AC000612E2050756E746920616E746572696FE5
:107AD0007269206E6F6E207261676769756E676983
:107AE00062696C692E004B616C696272616365202A
:107AF00058595A2073656C68616C612E205072650C
:107B0000646E69206B616C69627261636E69206288
:107B10006F6479206D6F63207670726564752E20B6
:107B200053726F766E656A7465207469736B6172E7
:107B30006E752E0058595A2063616C6962726174C7
:107B4000696F6E206661696C65642E2046726F6E87
:107B5000742063616C6962726174696F6E20706F0A
:107B6000696E7473206E6F74207265616368616200
:107B70006C652E005A2D4B616C6962726965727575
:107B80006E67206665686C67657363686C672E2036
:107B900053656E736F72206E6963687420616E67DF
:107BA000657363686C6F7373656E2E2057617274B2
:107BB00065206175662052657365742E004B616C9B
:107BC00069627261636A61206E69657564616E6184
:107BD0002E2053656E736F72206F646C61637A6FD1
:107BE0006E79206C75622075737A6B6F647A2E20C3
:107BF0006B6162656C2E20437A656B616D206E61EE
:107C00002072657365742E004E6976656C616369D8
:107C10006F6E2066616C6C6164612E2053656E73BB
:107C20006F7220646573636F6E65637461646F2047
:107C30006F206361626C65732064616E61646F7351
:107C40002E204573706572616E646F207265736576
:107C5000742E004C6976656C6C616D656E746F2076
:107C60006C6574746F2066616C6C69746F2E205340
:107C7000656E736F726520646973636F6E2E206F1B
:107C8000204361766F2044616E6E2E20496E206124
:107C900074746573612064692072657365742E0065
:107CA0004B616C696272616365205A2073656C6810
:107CB000616C612E2053656E736F72206A65206F50
:107CC00064706F6A656E79206E65626F2070726590
:107CD000727573656E79206B6162656C2E204365E9
:107CE0006B616D206E612072657365742E00426554
:107CF00064206C6576656C696E67206661696C6589
:107D0000642E2053656E736F7220646973636F6EA7
:107D10006E6563746564206F72206361626C6520B8
:107D200062726F6B656E2E2057616974696E672091
:107D3000666F722072657365742E005A2D4B616CEC
:107D40002E206665686C67657363686C672E2053C8
:107D5000656E736F72206E696368742061757367F6
:107D6000656C6F6573742E205363686D75747A69E2
:107D700067652044756573653F205761727465209F
:107D8000617566205265736574004B616C6962723F
:107D900061636A61206E69657564616E612E20534E
:107DA000656E736F72206E696520646F746B6E61AF
:107DB0006C2E205A616E6965637A79737A2E20641D
:107DC00079737A613F20437A656B616D206E612023
:107DD00072657365742E004E6976656C6163696FB8
:107DE0006E2066616C6C6164612E2053656E736FEA
:107DF00072206E6F2066756E63696F6E612E20450E
:107E000073636F6D62726F7320656E20426F717560
:107E1000692E3F204573706572616E646F207265D4
:107E20007365742E004C6976656C6C616D656E745B
:107E30006F206C6574746F2066616C6C69746F2E52
:107E40004E6F5269737053656E736F722052657313
:107E500069647569207375207567656C6C6F3F2068
:107E6000496E206174746573612064692072657362
:107E700065742E004B616C696272616365205A20E3
:107E800073656C68616C612E2053656E736F722030
:107E90006E657365706E756C2E205A6E65636973BE
:107EA00074656E6120747279736B613F2043656BFA
:107EB000616D206E612072657365742E0042656489
:107EC000206C6576656C696E67206661696C6564B7
:107ED0002E2053656E736F72206469646E74207413
:107EE0007269676765722E20446562726973206FDC
:107EF0006E206E6F7A7A6C653F2057616974696E87
:107F00006720666F722072657365742E005A2D4B60
:107F1000616C696272696572756E67206665686C0E
:107F200067657363686C672E2053656E736F72208C
:107F30007A7520686F63682061757367656C6F651B
:107F400073742E20576172746520617566205265C6
:107F50007365742E004B616C69627261636A6120A3
:107F60005A206E69657564616E612E2053656E736B
:107F70006F7220646F746B2E207A61207779736F33
:107F80006B6F2E20437A656B616D206E6120726588
:107F90007365742E004E6976656C6163696F6E203F
:107FA00066616C6C6164612E2053656E736F722024
:107FB00066756E63696F6E612064656D617369617A
:107FC000646F2074656D7072616E6F2E20457370E2
:107FD0006572616E646F2072657365742E004C6902
:107FE00076656C6C616D656E746F206C6574746F12
:107FF0002066616C6C69746F2E52697370207365B2
:108000006E736F72652074726F70706F207072651E
:1080100073746F496E2061747465736120646920A4
:1080200072657365742E004B616C69627261636581
:10803000205A2073656C68616C612E2053656E73E5
:108040006F72207365706E756C207072696C6973E5
:10805000207679736F6B6F2E2043656B616D206E98
:10806000612072657365742E00426564206C6576CC
:10807000656C696E67206661696C65642E20536566
:108080006E736F72207472696767657265642074BD
:108090006F6F20686967682E2057616974696E6721
:1080A00020666F722072657365742E0042656420CD
:1080B000617566776165726D656E0047727A616E93
:1080C00069652073746F6C696B612E2E0043616C5F
:1080D000656E74616E646F204261736500526973EE
:1080E00063616C642E206C6574746F005A616872F1
:1080F0006976616E69206265640042656420486546
:108100006174696E6700426564204F4B0053746F61
:108110006C696B204F4B2E00426173652070726555
:108120007061726164610050696174746F2066618E
:1081300074746F2E00426564204F4B2E00426564BC
:1081400020646F6E65005265636874732020202080
:108150005B756D5D005720707261776F205B756D88
:108160005D00446572656368612020205B756D5D0C
:1081700000446573747261202020205B756D5D0082
:1081800056707261766F205B756D5D00526967682D
:108190007420736964655B756D5D00527565636B12
:1081A0007365747A656E0052657365740048696E14
:1081B00074656E202020205B756D5D00446F207417
:1081C000796C7520205B756D5D0041747261732060
:1081D000202020205B756D5D00526574726F202039
:1081E0002020205B756D5D00567A61647520205BF0
:1081F000756D5D00526561722073696465205B7501
:108200006D5D00426564206C6576656C204B6F7215
:1082100072656B74004B6F72656B746120706F6474
:108220006B6C61646B6900436F72722E2064652011
:108230006C612063616D6100436F7272657A2E20FC
:108240006C69762E6C6574746F004B6F72656B632E
:108250006520706F646C6F7A6B7900426564206C86
:108260006576656C20636F7272656374004C696E2D
:108270006B7320202020205B756D5D0057206C659E
:10828000776F20205B756D5D00497A717569657245
:108290006461205B756D5D0053696E697374726112
:1082A00020205B756D5D00566C65766F20205B75D8
:1082B0006D5D004C6566742073696465205B756D47
:1082C0005D00566F726E6520202020205B756D5D0D
:1082D00000446F2070727A6F6475205B756D5D006D
:1082E0004164656C616E746520205B756D5D004650
:1082F000726F6E7465202020205B756D5D00567076
:1083000072656475205B756D5D0046726F6E7420DA
:10831000736964655B756D5D0053746F6C696B00A8
:1083200042617365004C6574746F0042656400447B
:1083300065722041627374616E64207A7769736339
:1083400068656E2064657220537069747A65206474
:10835000657220447565736520756E64206465726E
:108360002042656420697374206E6F6368206E69B3
:108370006368742065696E67657374656C6C742ED0
:1083800020426974746520666F6C67656E2053695E
:10839000652064656D2048616E64627563682C2099
:1083A00046697273742073746570732C20736563EF
:1083B00074696F6E204669727374206C617965729E
:1083C0002063616C6962726174696F6E2E004F6424
:1083D0006C65676C6F7363206479737A79206F645E
:1083E00020706F646B6C61646B69206E6965206AD4
:1083F00065737420736B616C6962726F77616E6113
:108400002E20506F73746570756A207A676F646E82
:108410006965207A20696E737472756B636A612076
:10842000726F7A647A69616C205A61637A796E61DD
:108430006D792C20706F64726F7A647A69616C2038
:108440004B616C69627261636A6120706965727701
:10845000737A656A20776172737477792E00446944
:108460007374616E63696120656E747265206C61FE
:108470002070756E7461206465206C6120626F717C
:1084800075696C6C612079206C6120737570657200
:108490006669636965206465206C612063616D6154
:1084A000206E6F2066696A6164612061756E2E209E
:1084B000506F72206661766F722073696761206504
:1084C0006C206D616E75616C2C20636170697475D0
:1084D0006C6F2046697273742073746570732C20FE
:1084E00073656363696F6E204669727374206C6193
:1084F0007965722063616C6962726174696F6E2E56
:108500000044697374616E7A6120747261206C61D9
:108510002070756E74612064656C6C277567656C7E
:108520006C6F2065206C612073757065726669637D
:1085300069652064656C206C6574746F206E6F6E65
:1085400020616E636F726120696D706F7374612E4C
:1085500020536920707265676120646920736567C4
:108560007569726520696C206D616E75616C652C32
:108570002063617069746F6C6F2046697273742038
:1085800073746570732C2073657A696F6E6520460D
:1085900069727374206C617965722063616C6962C1
:1085A000726174696F6E2E004E656E69207A6B6120
:1085B0006C6962726F76616E6120767A64616C6557
:1085C0006E6F737420747279736B79206F6420748A
:1085D00069736B6F766520706F646C6F7A6B792E40
:1085E00020506F73747570756A74652070726F7344
:1085F000696D20706F646C65206D616E75616C755E
:108600002C206B617069746F6C61205A6163696EB4
:10861000616D652C206F64737461766563204E61B3
:1086200073746176656E69207072766E69207672F9
:10863000737476792E0044697374616E6365206289
:1086400065747765656E20746970206F6620746844
:1086500065206E6F7A7A6C6520616E64207468653F
:10866000206265642073757266616365206861735A
:10867000206E6F74206265656E2073657420796565
:10868000742E20506C6561736520666F6C6C6F771B
:1086900020746865206D616E75616C2C2063686163
:1086A0007074657220466972737420737465707398
:1086B0002C2073656374696F6E2046697273742031
:1086C0006C617965722063616C6962726174696F53
:1086D0006E2E005A2065696E7374656C6C656E0051
:1086E000446F7374726F6A656E6965206F73792069
:1086F0005A004D6963726F7061736F20456A65201F
:108700005A00436F6D70656E73617A696F6E652094
:108710005A00446F6C6164656E69206F7379205AEA
:10872000004C6976652061646A757374205A004153
:10873000646A757374696E67205A00537461727449
:10874000706F736974696F6E004C6C65766172202E
:10875000616C206F726967656E0054726F7661207C
:108760006F726967696E65004175746F20686F6D1F
:108770006500207C20417574686F723A2000416C5E
:108780006C650057737A7973746B6F00546F646F04
:10879000730054757474690056736500416C6C0005
:1087A0004163746976652045787472756465723AC0
:1087B0002000511341132C1319130513F0126513E4
:1087C0006D1375137E138613E013CB13B813E013E8
:1087D000A3138E1306140214FF13FC13F813F513DE
:1087E0000A14121460144F143D1460142B141A143C
:1087F0001615FC14D914B814A214711463162B1690
:10880000ED15B315851534155C173C171517E916CA
:10881000D016A1165D19FC1892183618E0177F17AC
:10882000941DE91C0A1C511BAD1AC0199F1F5C1F27
:10883000211FCC1E951E481E9E214521EF20A02001
:108840005220EC1FD6236A230323A3225222E521C0
:10885000DB258F253A25EF24A02435249B27582794
:10886000F926B9267D262C2652283E2820280B28BA
:10887000F627D827172ABD2960290E29C32866287C
:108880000C2CBD2B632B0E2BC82A5F2A182DF42C21
:10889000C32C9B2C792C562CBB2DA62D872D6C2DF3
:1088A000522D382D562E472E2E2E122EFB2DCF2D2B
:1088B000782F4A2F152FDB2EB42E732EC631693137
:1088C000EF3091303630A62F26322D3279326F328A
:1088D0006032543249323D32DD32CB32B932A732C6
:1088E0009732853224332433123300332433EE326B
:1088F000943380336D335A3349333533FB33EA33A2
:10890000D833C733B833A6336634543442342F34A3
:108910001E340B347934BA34B434AD34A5349C34B9
:108920008C34E534E534E534E534D334BF341B35D9
:108930001B351B351B350935F7347D356D355D35F8
:108940004D353C352C35E335D235C135B0359E3506
:108950008D351237D7369C3660362B36F435B33723
:108960009E37893774375F374A37FF37F737EB372A
:10897000DF37D337C83721381938213811380B3849
:108980002138773869385A384838393829389F3883
:108990009F3894388D389F388238A938BD382A39A5
:1089A0001C390A39FB38EA38D8389239803971399C
:1089B00060394D393D39EE39E039CF39BF39B039F9
:1089C000A339483A3B3A2A3A1C3A0F3AFC399A3AC8
:1089D0008D3A813A733A663A593AA73A073BFE3ADA
:1089E000F53AEB3AE23AD23A0D3B5B3B4C3B3D3B2E
:1089F0005B3B2D3B1D3BC13BAF3B9D3B8B3B793BE9
:108A0000683B2D3C1B3C093CF73BE53BD33B943C8E
:108A1000833C733C613C513C3F3CE13CD23CC23C1A
:108A2000E13CB33CA33C4A3D383D243D123DFE3C75
:108A3000EE3C993D8F3D823D743D693D5B3DF63D89
:108A4000E73DD63DC43DB43DA23D343E343E253ED7
:108A5000153E343E033E873E783E6C3E613E543EBA
:108A6000463EB03EB03EA43EB03EB03E963E113FC4
:108A7000023FF53EE33ED13EBD3E2D3F2D3F263F1A
:108A80002D3F1F3F2D3F573F573F453F333F573FF8
:108A9000573FC03FAF3F9A3F863F753F693F2440F5
:108AA00012400140F03FDE3FC93F954080406B409F
:108AB0005A4046403640D940D940C740B740D940D7
:108AC000A640214121410F41FD402141EA4057414B
:108AD000574149413D4157413141754175416B41D4
:108AE000604175417541DF41CA41B541A4418F41A3
:108AF0007D4149423742274215420342F041B44288
:108B0000A242924280426E425B421F430D43FD42AD
:108B1000EB42D942C64283437143614351433F43D1
:108B20003143F343E143CE43BC43AA439543584406
:108B300046443744274415440544B844A644984461
:108B40008E447C446A44E944E944DA44CA44E94432
:108B5000E944F64402452B452B45224519452B4552
:108B600007453D454F456245AE45A0459545844581
:108B700077456A45BB45CD45E14539462B461F46FD
:108B80000D46FF45F14547465446624670468646C7
:108B90009146C546BE46B646C546AF46A74625479A
:108BA00014470247EF46DE46CC468B477C476C476E
:108BB000574746473447DD47D247C247B147A547E5
:108BC0009A47EA47F3471B483D487448634874484E
:108BD000744852487448A8489748A848A848864806
:108BE000A848D048C548D048D048BA48D0482E49AF
:108BF0001E490E49FB48EB48DC488E4980497049C4
:108C00005C494D493B499C490F4AFA49E649D649D6
:108C1000C449B1497B4A674A574A424A334A224AC1
:108C2000C44ABA4AAE4AA24A9A4A8F4ACC4A184B18
:108C3000094B014BEF4AE14AD44AEC4BC64B9A4BE5
:108C4000704B494B244B954C7C4C634C444C264C0C
:108C50000C4CAD4CC44C374D274D184D074DF94CBD
:108C6000E94C194EF34DC44D924D674D454D8B4E19
:108C7000774E6E4E5A4E514E464EFC4EEA4ED84EF0
:108C8000C54EB14E9F4E5D4F4F4F3E4F2E4F1F4F23
:108C90000E4FBD4FAD4F9E4F8D4F7F4F6D4FAC521E
:108CA00025529751EB505F50C94F425345537A5369
:108CB0007A53685359537A534953CC53BD53B253E3
:108CC000A05392538353FA53F353EC53E353DD53BE
:108CD000D7535C5449543754235414540154C35447
:108CE000B254A2548F547D547054DF54DC54DF547A
:108CF000DF54D854D3544655315521550C55F754AB
:108D0000E254F355D855B0559555785556554356B8
:108D10003856305628561C5613567A566F56675694
:108D20005F5653564A56B156A6569E5696568A5682
:108D30008156D056D056C056B856D056D056125737
:108D40000557FA56EF56E656D9562E572E571C574A
:108D50002E572E572E577B577157645758574D57DC
:108D60004057A4579F57995793578E5787579D58E9
:108D7000745838580C58D857AA570A59FA58EA580C
:108D80000A59DA58CD585E594F593F59305924592C
:108D9000195963597A599159A859335A1C5A055A85
:108DA000EE59D959C159495A265B3D5B545BB95BB1
:108DB000A65B975B8A5B7E5B6B5B1A5C0A5CF95B0C
:108DC000E75BD55BC65B815C6E5C5D5C485C375C79
:108DD000285CDC5CCE5CBD5CAD5C9D5C925C075D40
:108DE000015DF75C075DF15CEA5C595D4C5D3B5DE4
:108DF000295D1C5D0D5D915D895D805D785D715DB6
:108E0000695DC55DC55DBC5DA75DC55D995DCE5DF8
:108E10003B5E2B5E185E035EF15DDF5D4B5E575E71
:108E2000635E8E5E895E835E7D5E785E715E505F9E
:108E30002C5F055FE15EB45E945EAF5FA35F965FFB
:108E4000895F7D5F705F0760FA5FEA5FDB5FCD5F20
:108E5000BD5F536046603C60316026601860AE6064
:108E6000A0608E6079606D605F60FB60F160E060C3
:108E7000D260C760BC600361156127617D630A63CE
:108E800098622462AF61366113640C640564FF6309
:108E9000F663EB636F645C644B6439642964186443
:108EA000A0649B6495648F648A6483644E652F65B7
:108EB0000A65E764C064A6649C659365856578650A
:108EC0006E659C65A765B965326622660D66F365B9
:108ED000DC65CC659866876677666566536642662C
:108EE000F366E466D566C566B666A866FD66256760
:108EF00025671B671267086725672E673E67B4679B
:108F0000DE6708682668596878689268CE68C7681E
:108F1000BF68CE68B968B168D568E368E868F26888
:108F20002E692E691F6915692E6901698369746943
:108F30006369546943693769AC69A569A069AC691B
:108F40009A699469E969DA69D269CB69BC69B269DD
:108F5000F169036A156A666A5B6A4B6A386A2C6A49
:108F6000206AA96AA06A966A8E6A836A796AB26A76
:108F7000216B0F6BFA6AE96AD76AC26A806B716B00
:108F8000606B506B446B326BD06BC66BB96BA96B6B
:108F90009F6B906B336C216C126C006CF06BDE6B12
:108FA000456C8A6C7E6C746C6B6C5F6C536CCA6CB9
:108FB000B86CCA6CCA6CA66C946C226D146D086D8A
:108FC000FC6CED6CDC6C306D416DAB6E776E2D6EB4
:108FD000E66D9D6D516D3B700070BF6F806F3A6F95
:108FE000F46ECF7192715071FB70BB7080707B73A7
:108FF0003473E872A172577212721975DF748C742F
:1090000042740074BC73917659761576D7759F7546
:109010005675F077C27785774D771677D276907947
:1090200049790379C27876782378347BE67AA97A0D
:10903000707A217AD479EE7CA07C537C087CBD7B4D
:10904000747BBD7E747E257ED77D8A7D3B7D698065
:109050002780DE7F957F557F0D7FFA80EC80DD8055
:10906000CD80BB80AC803D813581278118810D8109
:1090700006818C8180817181628155814681A781C1
:10908000A781A781A781A7819B81F481E881D981EC
:10909000CA81BC81AD815B824A8238822782158277
:1090A0000382B382A782988289827C826D820A833E
:1090B000FE82EF82E082D182C2822B832B832583C2
:1090C000208319832B833686A88501855E84CE8311
:1090D0002F83218712870287F286E086D3862F8727
:1090E000688768875A87498768873B8772879C8724
:1090F000988792878C8783877E87A087457872655B
:109100006D65207370616E206F6620746865205AEB
:109110002076616C756573210043616C63756C61C9
:1091200074696F6E206F6620746865206D61636876
:10913000696E6520736B657720616E64206F66666B
:10914000736574206661696C65642E00203C2000A4
:109150005741524E494E473A2046726F6E74207006
:109160006F696E74206E6F742072656163686162EE
:109170006C652E205920636F6F7264696E6174652F
:109180003A0000497465726174696F6E3A20004953
:109190006E76616C69642062656420636F727265CB
:1091A0006374696F6E206D61747269782E205265E8
:1091B00073657474696E6720746F206964656E747A
:1091C0006974792E00496E76616C69642062656409
:1091D00020636F7272656374696F6E206D61747263
:1091E00069782E20582F5920617865732061726547
:1091F000206661722066726F6D206265696E6720FD
:1092000070657270656E646963756C61722E004979
:109210006E76616C69642062656420636F7272654A
:109220006374696F6E206D61747269782E20536863
:10923000696674206F7574206F662072616E676551
:109240002E005A65726F20706F696E7420636F72A2
:1092500072656374696F6E3A00496E76616C696419
:109260002062656420636F7272656374696F6E203B
:109270006D61747269782E204C656E677468206F1A
:109280006620746865205920766563746F72206F5C
:109290007574206F662072616E67652E00592076A6
:1092A0006563746F72206C656E6774683A00496E0E
:1092B00076616C69642062656420636F72726563B5
:1092C00074696F6E206D61747269782E204C656EC2
:1092D000677468206F66207468652058207665631F
:1092E000746F72206F7574206F662072616E67658F
:1092F0002E005820766563746F72206C656E6774FB
:10930000683A00556E646566696E656420626564DE
:1093100020636F7272656374696F6E206D61747221
:1093200069782E00000040410000000000005C430E
:109330000000000000005C4300004043000040418A
:109340000000404300004041000000000000E442F3
:1093500000000000000057430000000000005743D9
:109360000000C0420000E4420000C0420000404152
:109370000000C04200004041000040430000E442C1
:109380000000404300005743000040435A00205A69
:109390003A00590020593A00580020583A0024F465
:1093A000D43050C38E20C2A24017828B7011127A23
:1093B000910D816CD90AA861E108C758660761510F
:1093C00043061E4B5D05C145A7041A411104093D22
:1093D0009803713931034036DB0265339102D43092
:1093E0005402802E1D02632CEE01752AC501B0289F
:1093F000A001102781018F2564012B244B01E0225D
:109400003401AC211F018D200D01801FFC00841E42
:10941000ED00971DDF00B81CD200E61BC600201B24
:10942000BC00641AB200B219A8000A19A0006A1898
:109430009900D117910040178B00B51684003116A2
:109440007E00B31579003A157300C7146F005814E5
:109450006A00EE1366008813630025135E00C712CE
:109460005B006C12570015125400C11151007011AD
:109470004F0021114B00D61049008D1047004610B7
:10948000440002104200C00F4000800F3E00420F17
:109490003C00060F3B00CB0E3800930E37005C0EED
:1094A0003500270E3400F30D3200C10D3100900D50
:1094B0003000600D2E00320D2D00050D2C00D90C52
:1094C0002B00AE0C2900850C29005C0C2700350C04
:1094D00027000E0C2600E80B2400C40B2400A00B70
:1094E00023007D0B23005A0B2100390B2100180BA0
:1094F0002000F80A1F00D90A1E00BB0A1E009D0AA0
:109500001D00800A1D00630A1C00470A1B002C0A6C
:109510001B00110A1A00F7091A00DD091900C40915
:109520001900AB091900920917007B09180063099B
:1095300017004C09160036091600200916000A0902
:109540001500F5081500E0081400CC081400B80850
:109550001400A4081400900813007D0812006B0882
:10956000130058081200460812003408110023089E
:1095700011001208110001081100F0071000E007A7
:109580001000D0071000C0071000B0070F00A1079F
:10959000100091070E0083070F0074070F00650786
:1095A0000E0057070E0049070E003B070D002E075F
:1095B0000E0020070D0013070D0006070D00F90629
:1095C0000C00ED060D00E0060C00D4060C00C806E9
:1095D0000C00BC060C00B0060C00A4060B0099069B
:1095E0000C008D060B0082060B0077060B006C0644
:1095F0000B0061060A0057060B004C060A004206E3
:109600000A0038060A002E060A0024060A001A0676
:109610000A001006090007060A00FD050900F40506
:109620000900EB050900E2050900D9050900D0058C
:109630000900C7050900BE050900B5050800AD050C
:109640000800A50509009C050800940508008C0584
:109650000800840508007C050800740508006C05F6
:109660000700650508005D050700560508004E0562
:1096700007004705070040050800380507003105C9
:1096800007002A050700230507001C05060016052C
:1096900007000F0507000805060002050700FB0488
:1096A0000600F5040700EE040600E8040600E204E4
:1096B0000700DB040600D5040600CF040600C90439
:1096C0000600C3040600BD040600B7040600B1048A
:1096D0000500AC040600A6040600A00405009B04D7
:1096E000060095040500900406008A040500850420
:1096F0000500800406007A04050075040500700466
:1097000005006B04050066040500610405005C04A7
:10971000050057040500520405004D0405004804E7
:109720000500430405003E0404003A040500350426
:109730000500300404002C04050027040400230461
:1097400005001E0404001A04040016040500110498
:1097500004000D04040009040500040404000004CE
:109760000400FC030400F8030400F4030400F00305
:109770000400EC030400E8030400E4030400E00335
:109780000400DC030400D8030400D4030400D00365
:109790000400CC030400C8030300C503030024F441
:1097A00004D9201BC40C5C0E9804C4095F02650731
:1097B0007101F405F900FB04B30048048700C103FC
:1097C00069005803550003034500BE023A008402B5
:1097D000310053022A002902250004022000E4017E
:1097E0001C00C8011900AF01170098011400840182
:1097F0001300710110006101100051010E004301BE
:109800000D0036010B002B010B0020010B00150190
:1098100009000C01090003010800FB000800F30027
:109820000800EB000700E4000600DE000600D80098
:109830000600D2000600CC000500C7000500C200EB
:109840000500BD000400B9000400B5000400B1002B
:109850000400AD000400A9000400A5000300A2005C
:1098600003009F0004009B00030098000300950084
:10987000020093000300900003008D0002008B00A3
:1098800003008800020086000200840003008100BB
:1098900002007F0002007D0002007B0002007900D0
:1098A00002007700010076000200740002007200DE
:1098B0000100710002006F0002006D0001006C00E9
:1098C00002006A00010069000200670001006600F2
:1098D00001006500010064000200620001006100F7
:1098E0000100600001005F0002005D0001005C00FB
:1098F00001005B0001005A000100590001005800FE
:1099000001005700010056000100550001005400FD
:1099100001005300000053000100520001005100FB
:109920000100500001004F0001004E0000004E00F9
:1099300001004D0001004C0001004B0000004B00F5
:1099400001004A00010049000100480000004800F1
:1099500001004700010046000000460001004500EC
:1099600000004500010044000100430000004300E6
:1099700001004200000042000100410000004100DF
:109980000100400001003F0000003F0001003E00D8
:1099900000003E0001003D0000003D0001003C00D1
:1099A00000003C0000003C0001003B0000003B00C8
:1099B00001003A0000003A000100390000003900BF
:1099C00001003800000038000000380001003700B6
:1099D00000003700010036000000360000003600AD
:1099E00001003500000035000000350001003400A2
:1099F0000000340000003400010033000000330098
:109A0000000033000100320000003200000032008C
:109A10000100310000003100000031000100300081
:109A2000000030000000300001002F0000002F0077
:109A300000002F0000002F0001002E0000002E006B
:109A400000002E0001002D0000002D0000002D0060
:109A500000002D0001002C0000002C0000002C0054
:109A600000002C0001002B0000002B0000002B0048
:109A700000002B0001002A0000002A0000002A003C
:109A800000002A0001002900000029000000290030
:109A90000000290000002900010028000000280023
:109AA0000000280000002800000028000100270016
:109AB000000027000000270000002700000027000A
:109AC00001002600000026000000260000002600FD
:109AD00000002600010025000000250000002500F0
:109AE00000002500000025000000250001002400E2
:109AF00000002400000024000000240000002400D6
:109B000001002300000023000000230000002300C8
:109B100000002300000023000000230001002200B9
:109B200000002200000022000000220000002200AD
:109B3000000022000100210000002100000021009F
:109B40000000210000002100000021000000210091
:109B50000100200000002000000020000000200084
:109B60000000200000002000000020000000200075
:109B700001001F0000001F0000001F0000001F0068
:109B800000001F0000001F0000001F0001001E0059
:109B900000001E0000001E0000001E0000004572B4
:109BA000723A204D494E54454D5020424544005490
:109BB000656D706572617475726520686561746544
:109BC0006420626564207377697463686564206FDC
:109BD00066662E204D494E54454D5020747269677B
:109BE00067657265642021004572723A204D4158C4
:109BF00054454D50204245440054656D7065726176
:109C0000747572652068656174656420626564209E
:109C10007377697463686564206F66662E204D41B2
:109C20005854454D502074726967676572656420A9
:109C300021004572723A204D494E54454D50003A2C
:109C400020457874727564657220737769746368EF
:109C50006564206F66662E204D494E54454D502058
:109C60007472696767657265642021004572723A93
:109C7000204D415854454D50003A20457874727536
:109C8000646572207377697463686564206F6666C3
:109C90002E204D415854454D5020747269676765B8
:109CA00072656420210020484F54454E442054489A
:109CB00045524D414C2052554E4157415900204884
:109CC00045415442454420544845524D414C205250
:109CD000554E4157415900544845524D414C205230
:109CE000554E415741590042454420544845524D34
:109CF000414C2052554E415741590020544845523D
:109D00004D414C2052554E41574159202820505228
:109D1000454845415420484F54454E44290020545D
:109D20004845524D414C2052554E415741592028EB
:109D300020505245484541542048454154424544ED
:109D4000290050524548454154204552524F520037
:109D50004245442050524548454154204552524FB7
:109D600052004572723A205052494E542046414E9C
:109D7000204552524F52004552524F523A20507293
:109D8000696E742066616E20737065656420697306
:109D9000206C6F776572207468656E2065787065D9
:109DA00063746564004572723A20455854522E20FF
:109DB00046414E204552524F52004552524F523A60
:109DC0002045787472756465722066616E207370C8
:109DD000656564206973206C6F77657220746865AF
:109DE0006E20657870656374656400202D20496E6F
:109DF00076616C6964206578747275646572206E32
:109E0000756D626572202100504944204175746F60
:109E100074756E652066696E69736865642120508B
:109E2000757420746865206C617374204B702C20ED
:109E30004B6920616E64204B6420636F6E737461A4
:109E40006E74732066726F6D2061626F7665206933
:109E50006E746F20436F6E66696775726174696FA7
:109E60006E2E6800504944204175746F74756E659C
:109E7000206661696C6564212074696D656F757415
:109E80000020403A006F6B20543A006F6B20423A3A
:109E900000504944204175746F74756E6520666189
:109EA000696C6564212054656D70657261747572AA
:109EB0006520746F6F206869676800204B643A20E2
:109EC00000204B693A2000204B703A200020436C60
:109ED00061737369632050494420002054753A200F
:109EE00000204B753A2000206D61783A2000206DEB
:109EF000696E3A200020643A200020626961733A5A
:109F0000200010137D002015780060177300C01921
:109F10006E00401C6900E01E640080215F00402448
:109F20005A00F026550090295000202C4B00802E1E
:109F30004600C0304100D0323C00B03437005036CB
:109F40003200C0372D0000392800103A2300F03AC3
:109F50001E00B03B1900503C1400D03C0F00303DB7
:109F60000A00803D0500C03D0000F03DFBFF103EB3
:109F7000F6FF303EF1FF403EECFF503EE7FF603E13
:109F8000E2FF703EDDFF703ED8FF1000C9021001F5
:109F90002C014001220170011801B0010E01F001F5
:109FA00004015002FA00B002F0003003E600D003D2
:109FB000DC009004D2007005C800A006BE000008B6
:109FC000B400B009AA00D00BA000600E960060118A
:109FD0008C000015820020197800C01D6E00A022A0
:109FE0006400B0275A00902C500000314600E03445
:109FF0003C0010383200903A2800603C1E00A03D22
:10A000001400803E0A00203F000070012C019001E6
:10A010002701B0012201C0011D01F0011801100249
:10A02000130130020E016002090190020401C00216
:10A03000FF000003FA004003F5008003F000D003A6
:10A04000EB002004E6007004E100E004DC004005C1
:10A05000D700C005D2004006CD00D006C80080075A
:10A06000C3003008BE00F008B900C009B400B00A4F
:10A07000AF00B00BAA00D00CA500000EA000500F3E
:10A080009B00C01096005012910000148C00C01567
:10A090008700B0178200B0197D00D01B7800001E29
:10A0A000730040206E0090226900F0246400402775
:10A0B0005F0090295A00E02B5500102E50002030F0
:10A0C0004B0010324600E033410090353C00103721
:10A0D000370070383200A0392D00B03A2800A03B7C
:10A0E0002300603C1E00103D1900903D1400103EFE
:10A0F0000F00703E0A00C03E0500003F0000544DB6
:10A100004320445249564552204F56455254454DDE
:10A11000502000436F6E74696E75652077697468AE
:10A1200020616E6F7468657220626F7764656E3F40
:10A130000053746174653A2000473736004D34355A
:10A14000205A004D3435004738300020003E003E94
:10A150000020003E003E003E003E0020003E003E4B
:10A1600000200000002D2D2D2D2D2D2D2D2D2D2DE0
:10A170002D2D2D2D2D2D2D2D2D004E2F41004E2F0F
:10A1800041006D6D00004D373031004D37303200E9
:10A190004D353030004731205A3135204631353089
:10A1A0003000473931004731205835302059313996
:10A1B0003020453020463730303000473930004DB0
:10A1C000373032004D3730322043004D37303220A7
:10A1D00055004D373032004731205A313520463155
:10A1E000353030004739310047312058353020595B
:10A1F000313930204530204637303030004D38334B
:10A2000000473930004D3834004D31303420533060
:10A21000004D383400473120583130205931383022
:10A22000204634303030004731205A31302046311A
:10A230003330302E303030004D3134302053300048
:10A240004D313034205330004D313037004731200C
:10A25000452D302E30373530302046323130302EDB
:10A2600030303030300047312058353020593535C6
:10A270002045332E363237373300473120583230BD
:10A2800030205935352045302E34393338360047A3
:10A29000312058323030205937352045332E363270
:10A2A000373733004731205835302059373520456E
:10A2B000302E343933383600473120583530205964
:10A2C00039352045332E3632373733004731205861
:10A2D000323030205939352045302E343933383634
:10A2E0000047312058323030205931313520453344
:10A2F0002E36323737330047312058353020593128
:10A3000031352045302E3439333836004731205826
:10A31000353020593133352045332E3632373733F7
:10A320000047312058323030205931333520453004
:10A330002E363631373400473120583230302059EC
:10A340003135352045322E3632373733004731200C
:10A3500058313030205931353520453200473120D1
:10A3600058373520593135352045322E35004731A3
:10A3700020463130383000473120583530205931AF
:10A380003535004731204634303030004D323034DE
:10A39000205331303030004731205A302E313530A3
:10A3A0002046373230302E30303000473120452DB6
:10A3B000312E35303030302046323130302E303092
:10A3C000303030004D3833004739300047323100EB
:10A3D0004739322045302E30004731205831303057
:10A3E0002E30204531322E352046313030302E305F
:10A3F000004731205836302E302045392E30204647
:10A40000313030302E30004739322045302E300088
:10A4100047323800473837004D3130392053323118
:10A4200030004D31393020533535004D3134302036
:10A43000533535004D3130342053323130004D31F9
:10A44000303700473930004731204531004D383230
:10A45000004731204531004D3833004D3130362032
:10A46000532564004D32323020532564003A2000D9
:10A4700020202020202020202020202020202020DC
:10A4800020202000203A20002020202020202020F2
:10A4900020202020202020202020202000202020DC
:10A4A0002020202020202020202000257300202094
:10A4B000002D2D3A2D2D002000200020004C0020E2
:10A4C00020002046002D2D2D003E555342005344C0
:10A4D000002D2D00252020202020002020002020DD
:10A4E000000120002020202D2D2D200020205A00AA
:10A4F0002020000120004D36303000464C455820C9
:10A500002D20203233302F35300050502020202D88
:10A5100020203235342F3130300048495053202D1F
:10A5200020203232302F3130300050455420202D41
:10A5300020203234302F393000504C4120202D2043
:10A54000203231352F35350041425320202D202037
:10A550003235352F313030006661726D20202D206C
:10A56000203235302F3430004D3234004D3233201C
:10A57000257300052E2E00580059005A00457874A6
:10A580007275646572004739390044697361626CA1
:10A5900065206661726D206D6F64653F004469736C
:10A5A00061626C65206661726D206D6F6465004646
:10A5B00061726D206E756D626572004D38340050A9
:10A5C00072696E742066616E3A00457874727564C3
:10A5D00065722066616E3A0041786973206C656E21
:10A5E00067746820646966666572656E63653A00C3
:10A5F0004D656173757265642061786973206C655F
:10A600006E6774683A004D3834004731205A31354E
:10A61000004732382057005A30005A310059300074
:10A62000593100583000583100456E642073746F02
:10A6300070732064696167004D34340047323820FC
:10A6400057004175746F207265636F766572206381
:10A650007261736800436865636B2066616E732086
:10A660005B4449535D00436865636B2066616E73AC
:10A67000205B454E5D0054656D7065726174757246
:10A680006573002D2D2D2D2D2D2D2D2D2D2D2D00D6
:10A69000466C61736841697220495020416464725C
:10A6A0003A002D2D2D2D2D2D2D2D2D2D2D2D004E06
:10A6B0006F762031362032303137002D2D2D2D2D63
:10A6C0002D2D2D2D2D2D2D00453344763666756CA0
:10A6D0006C0045494E595F30346100315F37356D4C
:10A6E0006D5F4D4B33002D2D2D2D2D2D2D2D2D2D11
:10A6F0002D2D0020332E302E31322D524332206248
:10A70000313039004669726D776172653A002564AF
:10A710002E25642E25642E2564004661696C207305
:10A7200074617473004661726D206E756D6265723E
:10A7300000007263006265746100616C70686100A2
:10A740006465760050525553413344465700332ECA
:10A75000302E31322D5243320000000A0B02090C18
:10A760000D0E0807030401000000000000000000B7
:10A7700000000000000000000000000000000000D9
:10A780000000000000121110000000000000000096
:10A7900000000000000000000000000000000000B9
:10A7A00000000000000000000000000000000001A8
:10A7B00002102020080810204010204080020102D2
:10A7C000010804020101020408102040808040209A
:10A7D00010080402018004020180402010080402D5
:10A7E0000108040201010204081020408001020453
:10A7F0000810204080100804088010204004408089
:10A800001020400480050505050705080808080212
:10A810000202020A0A0808040404040101010101F9
:10A820000101010303030303030303040707070CE8
:10A830000C0C0C0C0C0C0C0202020206060606069E
:10A840000606060B0B0B0B0B0B0B0B07070A0A0A72
:10A850000A0A0A050505040404080800002000236C
:10A8600000260029002C002F003200000100000308
:10A87000010601090100002200250028002B002EFE
:10A88000003100340002010000050108010B010045
:10A89000002100240027002A002D00300033000191
:10A8A000010000040107010A01024E414E494E49D0
:10A8B0005459494E46CDCCCC3D0AD7233C17B7D18D
:10A8C0003877CC2B329595E6241FB14F0A00002033
:10A8D000410000C84200401C4620BCBE4CCA1B0EB2
:10A8E0005AAEC59D7400407A10F35A00A0724E18FB
:10A8F000090010A5D4E80000E87648170000E40B32
:10A9000054020000CA9A3B000000E1F505000080F7
:10A91000969800000040420F000000A08601000051
:10A9200000102700000000E80300000000640000A1
:10A930000000000A00000000000100000000002CE0
:10A9400076D888DC674F0823DFC1DFAE59E1B1B7A5
:10A9500096E5E3E453C63AE651997696E8E6C28472
:10A9600026EB898C9B62ED407C6FFCEFBC9C9F408A
:10A97000F2BAA56FA5F490055A2AF75C936B6CF9AF
:10A98000676DC11BFCE0E40D47FEF520E6B500D085
:10A99000ED902E0300943577050080841E0800009A
:10A9A000204E0A000000C80C333333330F986E1268
:10A9B000831141EF8D2114893BE65516CFFEE6DB6E
:10A9C00018D1844B381BF77C1D901DA4BBE42420B8
:10A9D0003284725E228100C9F124ECA1E53D27009A
:10A9E00039C2CFE89D010D024B016AC211241FBE7E
:10A9F000CFEFD1E2DEBFCDBF00E00CBF18E0A0E09A
:10AA0000B2E0ECE1F9EC03E00BBF02C007900D925D
:10AA1000A63CB107D9F72AE1A6ECB8E001C01D9227
:10AA2000A93FB207E1F719EACAEED9EA00E006C089
:10AA300022970109FE010BBF0F940DDBC03ED10729
:10AA400080E00807A9F70F94E5D40D947CE40C94FA
:10AA50000000CF92DF92EF92FF920F931F93CF935C
:10AA6000DF938C01D42EC62FD72FD60EDC1671F1B2
:10AA7000F801E080F180C990C7010F9440E1C81649
:10AA8000F1F06C2DC7010F9470E1C7010F9440E104
:10AA90008C15A9F0E2EAF7E08491882341F09091C7
:10AAA000C00095FFFCCF8093C6003196F5CF809112
:10AAB000C00085FFFCCF8AE08093C60007C0F80184
:10AAC00080819181019691838083D0CFDF91CF9156
:10AAD0001F910F91FF90EF90DF90CF900895EF922C
:10AAE000FF920F931F93CF93DF931F92CDB7DEB7E3
:10AAF0008C017B01460FF8018081918149830F947D
:10AB000040E1F70181937F01F801808191810196F5
:10AB10009183808349814E11EECF0F90DF91CF91C9
:10AB20001F910F91FF90EF900895FF920F931F9345
:10AB3000CF93DF93CDB7DEB72C970FB6F894DEBF77
:10AB40000FBECDBF8C01F62E80E390E3A0E3B0E012
:10AB50008D839E83AF83B8871C870B8744E0BE013B
:10AB60006B5F7F4FCE010B9674DF40E163E578E1C8
:10AB7000CE010B966EDF40E163E678E1CE010B96E5
:10AB800068DF40E163E478E1CE010B9662DF44E0E8
:10AB90006BE378E1CE010B965CDF44E067E378E19C
:10ABA000CE010B9656DF44E06FE378E1CE010B96C1
:10ABB00050DF44E063E278E1CE010B964ADF44E0E7
:10ABC00063E778E1CE010B9644DF44E067E278E189
:10ABD000CE010B963EDF44E06BE278E1CE010B96AE
:10ABE00038DF44E06FE278E1CE010B9632DF44E0DB
:10ABF00063E378E1CE010B962CDF4CE060E07AE075
:10AC0000CE010B9626DF44E069EF79E0CE010B968A
:10AC100020DF44E06DEA72E0CE010B961ADF44E0DB
:10AC200069EA72E0CE010B9614DF44E065EA72E057
:10AC3000CE010B960EDF44E06DE972E0CE010B967B
:10AC400008DF44E069E972E0CE010B9602DF44E0E0
:10AC500065E972E0CE010B96FCDE80E290E09A8717
:10AC6000898742E0BE01675F7F4FCE010B96F1DE20
:10AC700041E065EF79E0CE010B96EBDE44E064E263
:10AC800072E0CE010B96E5DE44E06CE172E0CE01AD
:10AC90000B96DFDE44E060EF79E0CE010B96D9DE63
:10ACA00044E06CEE79E0CE010B96D3DE44E068E13F
:10ACB00072E0CE010B96CDDE41E06CE17AE0CE0190
:10ACC0000B96C7DE44E064E472E0CE010B96C1DE71
:10ACD00089E08F1560F444E062E772E1CE010B96E3
:10ACE000B8DE44E06EE672E1CE010B96B2DE46E5D8
:10ACF00051E360E070E049835A836B837C831C8757
:10AD00000B8744E0BE016F5F7F4FCE010B96A1DE43
:10AD1000E4E5FFE08491882341F09091C00095FF25
:10AD2000FCCF8093C6003196F5CFE2E9F7E084913D
:10AD3000882341F09091C00095FFFCCF8093C6001E
:10AD40003196F5CF8091C00085FFFCCF8AE08093DB
:10AD5000C6002C960FB6F894DEBF0FBECDBFDF91B4
:10AD6000CF911F910F91FF9008951F93CF93DF9381
:10AD7000182FC4E5DFE0FE018491882341F0909113
:10AD8000C00095FFFCCF8093C6003196F5CFE2E876
:10AD9000F7E08491882341F09091C00095FFFCCFAB
:10ADA0008093C6003196F5CF8091C00085FFFCCF1F
:10ADB0008AE08093C600FE018491E4E5FFE08823E9
:10ADC00049F09091C00095FFFCCF8093C60031966A
:10ADD0008491F5CF409153185091541860915518B3
:10ADE000709156188AE797E00E94C46840915718FE
:10ADF000509158186091591870915A1887E797E048
:10AE00000E94C46840915B1850915C1860915D1875
:10AE100070915E1884E797E00E94C46840915F18C3
:10AE200050916018609161187091621881E797E005
:10AE30000E94C4688091C00085FFFCCF8AE08093A7
:10AE4000C600FE018491E4E5FFE0882349F090917B
:10AE5000C00095FFFCCF8093C60031968491F5CF5A
:10AE6000E7E5F7E08491882341F09091C00095FFD9
:10AE7000FCCF8093C6003196F5CF8091C00085FF4E
:10AE8000FCCF8AE08093C600FE018491E4E5FFE0F8
:10AE9000882349F09091C00095FFFCCF8093C600B5
:10AEA00031968491F5CF4091631850916418609168
:10AEB0006518709166188EE497E00E94C46840910E
:10AEC0006718509168186091691870916A188BE43E
:10AED00097E00E94C46840916B1850916C18609183
:10AEE0006D1870916E1888E497E00E94C4684091D4
:10AEF0006F1850917018609171187091721885E4F4
:10AF000097E00E94C4688091C00085FFFCCF8AE072
:10AF10008093C600FE018491E4E5FFE0882349F0B8
:10AF20009091C00095FFFCCF8093C600319684912C
:10AF3000F5CFE7E2F7E08491882341F09091C000DB
:10AF400095FFFCCF8093C6003196F5CF8091C0006D
:10AF500085FFFCCF8AE08093C600FE018491E4E582
:10AF6000FFE0882349F09091C00095FFFCCF8093CB
:10AF7000C60031968491F5CF409143185091441802
:10AF800060914518709146188EE197E00E94D5684F
:10AF900040914718509148186091491870914A188B
:10AFA0008BE197E00E94D56840914B1850914C1866
:10AFB00060914D1870914E1888E197E00E94D56815
:10AFC00040914F185091501860915118709152183B
:10AFD00085E197E00E94D5688091C00085FFFCCF95
:10AFE0008AE08093C600FE018491E4E5FFE08823B7
:10AFF00049F09091C00095FFFCCF8093C600319638
:10B000008491F5CFE0EEF6E08491882341F09091B1
:10B01000C00095FFFCCF8093C6003196F5CF80919C
:10B02000C00085FFFCCF8AE08093C600FE018491BA
:10B03000E4E5FFE0882349F09091C00095FFFCCF44
:10B040008093C60031968491F5CF40913B18509182
:10B050003C1860913D1870913E1887ED96E00E9473
:10B06000C468409137185091381860913918709120
:10B070003A1884ED96E00E94C4688091C00085FF74
:10B08000FCCF8AE08093C600FE018491E4E5FFE0F6
:10B09000882349F09091C00095FFFCCF8093C600B3
:10B0A00031968491F5CFE1E2F6E08491882341F076
:10B0B0009091C00095FFFCCF8093C6003196F5CFEC
:10B0C0008091C00085FFFCCF8AE08093C600FE011E
:10B0D0008491E4E5FFE0882349F09091C00095FF5A
:10B0E000FCCF8093C60031968491F5CF40913F18F4
:10B0F00050914018609141187091421888E196E093
:10B100000E94C4684091231850912418609125181A
:10B110007091261885E196E00E94C46840917318EA
:10B1200050917418609175187091761882E196E0CC
:10B130000E94D568409127185091281860912918CD
:10B1400070912A188FE096E00E94C46840912B18F5
:10B1500050912C1860912D1870912E188CE096E06B
:10B160000E94C46840912F18509130186091311896
:10B170007091321889E096E00E94C46840913318BB
:10B1800050913418609135187091361886E096E029
:10B190000E94C4688091C00085FFFCCF8AE0809344
:10B1A000C600FE018491E4E5FFE0882349F0909118
:10B1B000C00095FFFCCF8093C60031968491F5CFF7
:10B1C000E4EFF5E08491882341F09091C00095FF71
:10B1D000FCCF8093C6003196F5CF8091C00085FFEB
:10B1E000FCCF8AE08093C600FE018491E4E5FFE095
:10B1F000882349F09091C00095FFFCCF8093C60052
:10B2000031968491F5CF4091000A5091010A6091E6
:10B21000020A7091030A8BEE95E00E94C468409187
:10B22000040A5091050A6091060A7091070A88EE97
:10B2300095E00E94C4684091080A5091090A609103
:10B240000A0A70910B0A85EE95E00E94C46880910D
:10B25000C00085FFFCCF8AE08093C600FE01849188
:10B26000E4E5FFE0882349F09091C00095FFFCCF12
:10B270008093C60031968491F5CFE7EDF5E0849197
:10B28000882341F09091C00095FFFCCF8093C600C9
:10B290003196F5CF8091C00085FFFCCF8AE0809386
:10B2A000C600FE018491E4E5FFE0882349F0909117
:10B2B000C00095FFFCCF8093C60031968491F5CFF6
:10B2C0004091AD025091AE026091AF027091B00218
:10B2D0008DEC95E00E94C4686091A9027091AA0269
:10B2E0008091AB029091AC020F94DF55AB01BC0191
:10B2F0008AEC95E00E94C4686091A5027091A60254
:10B300008091A7029091A8020F94EB55AB01BC016C
:10B3100087EC95E00E94C4688091C00085FFFCCF57
:10B320008AE08093C600FE018491E4E5FFE0882373
:10B3300049F09091C00095FFFCCF8093C6003196F4
:10B340008491F5CFE1EBF5E08491882341F0909171
:10B35000C00095FFFCCF8093C6003196F5CF809159
:10B36000C00085FFFCCF8AE08093C600FE01849177
:10B37000E4E5FFE0882349F09091C00095FFFCCF01
:10B380008093C60031968491F5CF40919D025091F3
:10B390009E0260919F027091A00287EA95E00E9450
:10B3A000C4686091990270919A0280919B02909179
:10B3B0009C020F94DF55AB01BC0184EA95E00E942A
:10B3C000C468609195027091960280919702909165
:10B3D00098020F94EB55AB01BC0181EA95E00E9405
:10B3E000C4688091C00085FFFCCF8AE08093C600CE
:10B3F000FE018491E4E5FFE0882349F09091C000CC
:10B4000095FFFCCF8093C60031968491F5CFEDE691
:10B41000F5E08491882341F09091C00095FFFCCF26
:10B420008093C6003196F5CF8091C00085FFFCCF98
:10B430008AE08093C600FE018491E4E5FFE0882362
:10B4400049F09091C00095FFFCCF8093C6003196E3
:10B450008491F5CF409124025091250260912602FB
:10B460007091270283E695E00E94C46820E030E0F6
:10B4700040E752E460911C0270911D0280911E020F
:10B4800090911F020F94A2D8AB01BC0180E695E019
:10B490000E94C4684091F0095091F1096091F2094D
:10B4A0007091F3098DE595E00E94C4688091C00019
:10B4B00085FFFCCF8AE08093C600FE018491E4E51D
:10B4C000FFE0882349F09091C00095FFFCCF809366
:10B4D000C60031968491F5CFE1E3F5E084918823AD
:10B4E00041F09091C00095FFFCCF8093C60031964B
:10B4F000F5CF8091C00085FFFCCF8AE08093C60025
:10B50000FE018491E4E5FFE0882349F09091C000BA
:10B5100095FFFCCF8093C60031968491F5CF409182
:10B52000EC095091ED096091EE097091EF0987E205
:10B5300095E00E94C46820E030E040E752E460916A
:10B5400018027091190280911A0290911B020F94B7
:10B55000A2D8AB01BC0184E295E00E94C46880914E
:10B56000C00085FFFCCF8AE08093C600FE01849175
:10B57000E4E5FFE0882349F09091C00095FFFCCFFF
:10B580008093C60031968491F5CFEAECF4E0849183
:10B59000882341F09091C00095FFFCCF8093C600B6
:10B5A0003196F5CF8091C00085FFFCCF8AE0809373
:10B5B000C600FE018491E4E5FFE0882349F0909104
:10B5C000C00095FFFCCF8093C60031968491F5CFE3
:10B5D0004091F50950E060E070E080EC94E00E945A
:10B5E000D5688091C00085FFFCCF8AE08093C600BB
:10B5F000FE018491E4E5FFE0882349F09091C000CA
:10B6000095FFFCCF8093C60031968491F5CF809151
:10B610001C0A8823A1F1EDEAF4E08491882341F02B
:10B620009091C00095FFFCCF8093C6003196F5CF76
:10B630008091C00085FFFCCF8AE08093C600FE01A8
:10B640008491E4E5FFE0882349F09091C00095FFE4
:10B65000FCCF8093C60031968491F5CF409144028F
:10B6600050914502609146027091470283EA94E04E
:10B670000E94C4688091C00085FFFCCF11C0E7E83C
:10B68000F4E08491882341F09091C00095FFFCCFB5
:10B690008093C6003196F5CF8091C00085FFFCCF26
:10B6A0008AE08093C6001A3008F43EC0FE01C491BF
:10B6B000E4E5FFE0CC2349F08091C00085FFFCCF9A
:10B6C000C093C6003196C491F5CFEEE6F4E08491C4
:10B6D000882341F09091C00095FFFCCF8093C60075
:10B6E0003196F5CF8091C00085FFFCCF8AE0809332
:10B6F000C600409172125091731260917412709151
:10B70000751284E694E00E94C46840916E125091D4
:10B710006F1260917012709171128AE594E0DF915E
:10B72000CF911F910C94C468DF91CF911F91089520
:10B73000AF92BF92CF92DF92EF92FF920F931F933F
:10B74000CF93DF93CDB7DEB7E0970FB6F894DEBFA7
:10B750000FBECDBF80E1E2EEF2E0DE0191960190F6
:10B760000D928A95E1F780E1E2EFF2E0DE01519679
:10B7700001900D928A95E1F780E1E2E0F3E0DE01CD
:10B78000119601900D928A95E1F76E0181E2C80E43
:10B79000D11C83E5E82E88E1F82E8E010F5E1F4F45
:10B7A00063E678E1AE014F5F5F4F93E4A92E98E125
:10B7B000B92E20E030E0F60181919191A191B191F3
:10B7C0006F01F70181939193A193B1937F01F801E8
:10B7D00081919191A191B1918F01FB0181939193FD
:10B7E000A193B193BF01FA0181919191A191B1917E
:10B7F000AF01F50181939193A193B1935F012F5F05
:10B800003F4F24303105B9F60F94963280E090E432
:10B81000ACE9B4E480933B1890933C18A0933D1896
:10B82000B0933E188093371890933818A093391826
:10B83000B0933A1810923F18109240181092411885
:10B840001092421880E29EE4A0E0B0E0809373186A
:10B8500090937418A0937518B093761810922318CB
:10B8600010922418109225181092261880E090E06B
:10B87000A0E7B1E48093271890932818A093291883
:10B88000B0932A1880932B1890932C18A0932D18FE
:10B89000B0932E188DEC9CECACECBEE380932F188B
:10B8A00090933018A0933118B093321880E090E054
:10B8B000A0E2B0E48093331890933418A093351825
:10B8C000B09336181092080A1092090A10920A0AC8
:10B8D00010920B0A1092040A1092050A1092060A9E
:10B8E0001092070A1092000A1092010A1092020A9E
:10B8F0001092030A8DE39AE0A1E8B1E48093AD02CF
:10B900009093AE02A093AF02B093B0026DEC7CECCA
:10B9100084E99FE30F94D9556093A9027093AA021A
:10B920008093AB029093AC0265E87BEE80E692E4F4
:10B930000F94E5556093A5027093A6028093A70229
:10B940009093A8020F94054580E090E0A0E8BFE343
:10B950008093A1029093A202A093A302B093A402A9
:10B960001092F50980E090E0A0E4B0E48093240216
:10B9700090932502A0932602B093270240E050E066
:10B9800064E372E440931C0250931D0260931E0214
:10B9900070931F021092F0091092F1091092F209AF
:10B9A0001092F3091092EC091092ED091092EE0931
:10B9B0001092EF0940E050E060E071E4409318021B
:10B9C0005093190260931A0270931B0210921C0A82
:10B9D0008093440290934502A0934602B09347029D
:10B9E0000E94FF7EE4E5FFE08491882341F090917E
:10B9F000C00095FFFCCF8093C6003196F5CFEEE1F5
:10BA0000F4E08491882341F09091C00095FFFCCF31
:10BA10008093C6003196F5CF8091C00085FFFCCFA2
:10BA20008AE08093C600E0960FB6F894DEBF0FBEA2
:10BA3000CDBFDF91CF911F910F91FF90EF90DF90DD
:10BA4000CF90BF90AF9008951F93CF93DF93CDB762
:10BA5000DEB72C970FB6F894DEBF0FBECDBF162F02
:10BA60009C878B8786E591E3A0E0B0E089839A8389
:10BA7000AB83BC8344E0BE016B5F7F4FCE010B966E
:10BA80002ED843E050E0BE016B5F7F4FCE010196A0
:10BA90000F94AFDE892B09F0FFC040E163E578E148
:10BAA000CE010B961CD840E163E678E1CE010B96FF
:10BAB00016D840E163E478E1CE010B9610D80F94DC
:10BAC000963244E06BE378E1CE010B9608D844E06F
:10BAD00067E378E1CE010B9602D844E06FE378E1AA
:10BAE000CE010B960E946F5544E063E278E1CE01EF
:10BAF0000B960E946F5544E063E778E1CE010B9608
:10BB00000E946F5544E067E278E1CE010B960E94F7
:10BB10006F5544E06BE278E1CE010B960E946F55C1
:10BB200044E06FE278E1CE010B960E946F5544E04D
:10BB300063E378E1CE010B960E946F554CE060E024
:10BB40007AE0CE010B960E946F5544E069EF79E0F0
:10BB5000CE010B960E946F5544E06DEA72E0CE0173
:10BB60000B960E946F5544E069EA72E0CE010B9695
:10BB70000E946F5544E065EA72E0CE010B960E9488
:10BB80006F5544E06DE972E0CE010B960E946F554F
:10BB900044E069E972E0CE010B960E946F5544E0E3
:10BBA00065E972E0CE010B960E946F5542E0BE013E
:10BBB000675F7F4FCE010B960E946F5541E065EFA6
:10BBC00079E0CE010B960E946F5544E064E272E08A
:10BBD000CE010B960E946F5544E06CE172E0CE01FD
:10BBE0000B960E946F5544E060EF79E0CE010B9612
:10BBF0000E946F5544E06CEE79E0CE010B960E94F6
:10BC00006F5544E068E172E0CE010B960E946F55DB
:10BC100041E06CE17AE0CE010B960E946F5544E062
:10BC200064E472E0CE010B960E946F551A3070F0FA
:10BC300044E062E772E1CE010B960E946F5544E04A
:10BC40006EE672E1CE010B960E946F550E94FF7E58
:10BC50000F940545E4E5FFE08491882341F090913D
:10BC6000C00095FFFCCF8093C6003196F5CFE0E48D
:10BC7000F4E08491882341F09091C00095FFFCCFBF
:10BC80008093C6003196F5CF8091C00085FFFCCF30
:10BC90008AE08093C60001C04BDD2C960FB6F89465
:10BCA000DEBF0FBECDBFDF91CF911F910895CF931F
:10BCB000DF93EC0160E08E810F9424CF81E090E06F
:10BCC0000F9466CD61E08E810F9424CF81E090E0E7
:10BCD0000F9466CD60E08E810F9424CF84E690E0CF
:10BCE000DF91CF910D9466CDCF92DF92EF92FF92CC
:10BCF0000F931F93CF93DF937C01C0E0D0E0C62E5B
:10BD0000D12C87010C0F1D1F61E0F80187810F9472
:10BD1000EBCEB6010C2E02C0759567950A94E2F73A
:10BD20006170F80187810F9424CF2196C430D1052A
:10BD300041F7C701DF91CF911F910F91FF90EF90D5
:10BD4000DF90CF90B4CFCF92DF92EF92FF920F931C
:10BD50001F93CF93DF937C01C0E0D0E0C62ED12C9F
:10BD600087010C0F1D1F61E0F80187810F94EBCE56
:10BD7000B6010C2E02C0759567950A94E2F76170C2
:10BD8000F80187810F9424CF2196C830D10541F75F
:10BD9000C701DF91CF911F910F91FF90EF90DF903E
:10BDA000CF9085CF1F93CF93DF93EC01162F642F95
:10BDB0008C810F9424CF8D818F3F19F060E00F9418
:10BDC00024CF8F85612F84FF05C0CE01DF91CF91F5
:10BDD0001F91B9CF70E084E0759567958A95E1F77A
:10BDE000CE0182DF612FCE01DF91CF911F917CCFF9
:10BDF00040E0D8CF61E0FCDF80E496E00D9466CDB2
:10BE000062E0F6DF80E496E00D9466CDCF93DF9399
:10BE1000CDB7DEB728970FB6F894DEBF0FBECDBF03
:10BE200028E0E2E1F3E0DE01119601900D922A95FF
:10BE3000E1F7FC012389421710F04FEF420FFE019A
:10BE40003196E40FF11DE40FF11D2081260F2068CB
:10BE5000622F28960FB6F894DEBF0FBECDBFDF91DC
:10BE6000CF91C6CFFC016089262F2460208B6C60A7
:10BE7000BFCFCF93DF93EC01423018F08F858860FD
:10BE80008F874B8B1C8A222329F0413019F48F8530
:10BE900084608F8780E593EC0F9466CD60E08C81A1
:10BEA0000F9424CF60E08E810F9424CF8D818F3F3B
:10BEB00019F060E00F9424CF6F8564FD19C063E032
:10BEC000CE0112DF84E991E10F9466CD63E0CE01EB
:10BED0000BDF84E991E10F9466CD63E0CE0104DFCE
:10BEE00086E990E00F9466CD62E0CE01FDDE13C0DE
:10BEF0006062CE017DDF84E991E10F9466CD6F85AC
:10BF00006062CE0175DF86E990E00F9466CD6F85A3
:10BF10006062CE016DDF6F856062CE0169DF8CE308
:10BF200090E00F9466CD84E0888BCE019BDF8CE39C
:10BF300090E00F9466CDCE015DDF88EB9BE00F941F
:10BF400066CD82E0898B66E0CE0152DF8CE390E023
:10BF5000DF91CF910D9466CD6F927F928F92AF92C9
:10BF6000CF92EF920F931F93CF93DF93CDB7DEB7AE
:10BF70003C01162F842F5E854F8538899989F301FE
:10BF8000848325830683E782C086A18682865387C1
:10BF900044873587968761E00F94EBCEF301858166
:10BFA0008F3F19F061E00F94EBCE61E0F3018681E1
:10BFB0000F94EBCE112319F0F301178603C080E133
:10BFC000F301878720E041E060E1C301DF91CF9179
:10BFD0001F910F91EF90CF90AF908F907F906F90C7
:10BFE00048CF8F92AF92CF92EF920F93DC011396CE
:10BFF0001C921E921297EEE6F3E0ED93FC931F92D3
:10C000001F921F921F928C2CAE2CC02EE22E042F5A
:10C010002FEF462F61E0A0DF0F900F900F900F9051
:10C020000F91EF90CF90AF908F900895CF93DF93C3
:10C03000EC01423018F08F8588608F874B8B1C8A0B
:10C04000222329F0413019F48F8584608F8780E5A1
:10C0500093EC0F9466CD60E08C810F9424CF60E068
:10C060008E810F9424CF8D818F3F19F060E00F9463
:10C0700024CF6F8564FD19C063E0CE0135DE84E90D
:10C0800091E10F9466CD63E0CE012EDE84E991E16B
:10C090000F9466CD63E0CE0127DE86E990E00F9431
:10C0A00066CD62E0CE0120DE13C06062CE01A0DE6C
:10C0B00084E991E10F9466CD6F856062CE0198DED0
:10C0C00086E990E00F9466CD6F856062CE0190DEC8
:10C0D0006F856062CE018CDE8CE390E00F9466CDBC
:10C0E00084E0888BCE01BEDE8CE390E00F9466CDB9
:10C0F000CE0186DE80E496E00F9466CD82E0898BE7
:10C1000066E0CE0175DE8CE390E00F9466CD40E0F2
:10C1100068E0CE017BDE62E178E0CE010F94BFCF14
:10C1200041E068E0CE0172DE62E178E0CE010F947A
:10C13000BFCF42E066E0CE0169DE60E178E0CE018B
:10C14000DF91CF910D94BFCFCF92DF92EF92FF920C
:10C150000F931F93CF93DF931F921F92CDB7DEB73C
:10C160008C01677088E0689FB00111246064C80189
:10C1700049835A833DDE4981C42E5A81D52EE12C54
:10C18000F12CD6016D916D01D801ED91FC910190DA
:10C19000F081E02DC8011995BFEFEB1AFB0AE8E02A
:10C1A000EE16F10471F70F900F90DF91CF911F9170
:10C1B0000F91FF90EF90DF90CF90089541E0F2DD76
:10C1C00081E090E008951F920F920FB60F92112414
:10C1D0000BB60F922F933F934F935F936F938F9371
:10C1E0009F93EF93FF938091C00084FF03C08091E1
:10C1F000C60019C06091C6002091470930914809D6
:10C20000C90101968F7799274091490950914A09B0
:10C210008417950741F0F901E953F74F6083909334
:10C22000480980934709FF91EF919F918F916F91FA
:10C230005F914F913F912F910F900BBE0F900FBECA
:10C240000F901F9018951F920F920FB60F92112406
:10C250000BB60F922F933F934F935F936F938F93F0
:10C260009F93EF93FF9380914B09813001F580916B
:10C27000D00084FF03C08091D60019C06091D60021
:10C280002091470930914809C90101968F77992774
:10C290004091490950914A098417950741F0F901E5
:10C2A000E953F74F60839093480980934709FF91C2
:10C2B000EF919F918F916F915F914F913F912F914E
:10C2C0000F900BBE0F900FBE0F901F901895CF923E
:10C2D000DF92EF92FF926A017B01411581EE5807D0
:10C2E0006105710509F463C082E08093C00060E0DD
:10C2F00079E08DE390E0A70196010F94C6DA215012
:10C30000310941095109CA01B90122E030E040E098
:10C3100050E00F94C6DA91E03093C5002093C4003A
:10C320008091C10080618093C1008091C1008860CC
:10C330008093C1008091C10080688093C10080918A
:10C340004B098130D1F5992341F082E08093D000F0
:10C3500060E079E08DE390E006C01092D00060E8E4
:10C3600074E88EE190E0A70196010F94C6DA21509F
:10C37000310941095109CA01B90122E030E040E028
:10C3800050E00F94C6DA3093D5002093D40080910A
:10C39000D10080618093D1008091D100886080932A
:10C3A000D1008091D10080688093D10006C01092A6
:10C3B000C00090E020E130E0AFCFFF90EF90DF9041
:10C3C000CF9008952091490930914A0980914709F9
:10C3D000909148098217930771F0F901E953F74FDB
:10C3E00080812F5F3F4F2F77332730934A09209367
:10C3F000490990E008958FEF9FEF089580914909D2
:10C4000090914A09909348098093470908954F9263
:10C410005F926F927F928F929F92AF92BF92CF92D4
:10C42000DF92EF92FF920F931F93CF93DF93CDB7DD
:10C43000DEB7A0970FB6F894DEBF0FBECDBF5C018C
:10C440004115510561057105E9F420E030E040E354
:10C4500050E060E070E0A0960FB6F894DEBF0FBE2B
:10C46000CDBFDF91CF911F910F91FF90EF90DF90A3
:10C47000CF90BF90AF909F908F907F906F905F9084
:10C480004F905BC08E010F5F1F4FC12CD12C7601E6
:10C490004801422E512C612C712C8FEFC81AD80AFA
:10C4A000E80AF80ACB01BA01A30192010F94A4DAB9
:10C4B000CA01F80161938F01A901BC014115510521
:10C4C0006105710551F7F1E0CF1AD108E108F108D3
:10C4D000F401EC0DFD1D80818A3010F440E301C0B1
:10C4E00047E3480F552747FD5095652F752F20E0EE
:10C4F00030E0C50122D081E0C81AD108E108F10876
:10C50000EFEFCE16DE06EE06FE0611F7A0960FB68A
:10C51000F894DEBF0FBECDBFDF91CF911F910F9179
:10C52000FF90EF90DF90CF90BF90AF909F908F9053
:10C530007F906F905F904F9008952115310539F4E9
:10C540008091C00085FFFCCF4093C60008952A303B
:10C55000310509F43FC05BCF9A01462F552747FDAF
:10C560005095652F752FE9CFCF93DF93EC0120E035
:10C5700030E04DE050E060E070E0DFDF20E030E0F0
:10C580004AE050E060E070E0CE01DF91CF91D5CF7E
:10C59000FB012191BF01222339F03091C00035FF0A
:10C5A000FCCF2093C600F4CFDFCF9A01AB01662702
:10C5B00057FD6095762FC1CFCF93DF93EC019A01A1
:10C5C000AB01662757FD6095762FB7DFCE01DF916F
:10C5D000CF91CACFCF92DF92EF92FF92CF93DF93AA
:10C5E000EC016A017B0177FF0FC020E030E04DE2F3
:10C5F00050E060E070E0A1DFF094E094D094C0944B
:10C60000C11CD11CE11CF11C2AE0B701A601CE011E
:10C61000DF91CF91FF90EF90DF90CF90F8CE211572
:10C62000310539F48091C00085FFFCCF4093C600EE
:10C630000895EDCECF93DF93EC019A01462F50E0A1
:10C6400060E070E0ECDFCE01DF91CF918DCFCF9332
:10C65000DF93EC019A01AB0160E070E0E0DFCE0116
:10C66000DF91CF9181CFCF93DF93EC01D8DFCE0163
:10C67000DF91CF9179CF8F929F92AF92BF92CF925D
:10C68000DF92EF92FF921F93CF93DF93EC016A0149
:10C690007B01122F20E030E0A901C701B6010F9401
:10C6A000CDD587FF0CC020E030E04DE250E060E0E7
:10C6B00070E0CE0142DFF7FAF094F7F8F094B12C75
:10C6C00060E070E080E09FE3B11641F020E030E0F0
:10C6D00040E251E40F94D4D5B394F6CF9B01AC0162
:10C6E000C701B6010F94F4D46B017C010F9441D6BD
:10C6F0004B015C010F946DD69B01AC01C701B601E3
:10C700000F94F3D46B017C012AE0B501A401CE01A2
:10C710007EDE112361F0E0EAF5E08191882339F0B3
:10C720009091C00095FFFCCF8093C600F6CF1123F7
:10C7300019F120E030E040E251E4C701B6010F9466
:10C74000A2D86B017C010F943CD64B01AA2497FC24
:10C75000A094BA2CB501A401CE013CDFC501B401FF
:10C760000F946FD69B01AC01C701B6010F94F3D4AF
:10C770006B017C011150DBCFDF91CF911F91FF90B6
:10C78000EF90DF90CF90BF90AF909F908F900895E3
:10C7900072CFCF93DF93EC016EDFCE01DF91CF91AB
:10C7A000E3CEFC0165917591859194910895EF9286
:10C7B000FF920F931F93CF93DF93EC01CC0FDD1FFC
:10C7C000CC0FDD1FCE01805D904FEBDF9E01245F1B
:10C7D000354F79018E010050164FF80120813181CB
:10C7E000428153810F94F4D4F70160837183828373
:10C7F0009383CE01885B904FD4DF9E012C5C3D4F2C
:10C800007901F80120813181428153810F94F4D460
:10C81000F7016083718382839383CE01845C904FA0
:10C82000C0DFC85DDD4FF801208131814281538135
:10C830000F94F4D4688379838A839B83DF91CF91AB
:10C840001F910F91FF90EF900895CF93C82F4091C3
:10C850000C0250910D0260910E0270910F024093F4
:10C86000C3095093C4096093C5097093C609209108
:10C870005602309157023093760A2093750A24E6C7
:10C8800030E030935702209356020F9400CD60930E
:10C89000BE097093BF098093C0099093C1098C2F82
:10C8A000CF910D943F3480E00F943F348091C309C1
:10C8B0009091C409A091C509B091C60980930C025A
:10C8C00090930D02A0930E02B0930F028091750A0F
:10C8D0009091760A90935702809356020F9400CD60
:10C8E0006093BE097093BF098093C0099093C109FA
:10C8F0000895682F772767FD70958091580F909164
:10C90000590F835A904F0F9494DE90934F0F80935A
:10C910004E0F21E0892B09F420E0822F08958091A9
:10C920004E0F90914F0F4AE050E060E070E00196AA
:10C930000F94A5DCCB01089580914E0F90914F0F7D
:10C940004AE050E060E070E001960D94A5DC209193
:10C95000580F3091590FBC01C901835A904F0F9461
:10C96000CCDE90934F0F80934E0F21E0892B09F47A
:10C9700020E0822F08950F931F93CF93DF930091B0
:10C980004E0F10914F0F65E470E0C8010F9494DED4
:10C99000EC01009751F460E070E0C8010196DF916E
:10C9A000CF911F910F910D943DDB188280914E0F16
:10C9B00090914F0F60E070E001960F943DDB25E40D
:10C9C0002883DF91CF911F910F91089580914E0F91
:10C9D00090914F0F60E070E001960D943DDB2F9237
:10C9E0003F924F925F926F927F928F929F92AF92FF
:10C9F000BF92CF92DF92EF92FF920F931F93CF934C
:10CA0000DF93CDB7DEB760970FB6F894DEBF0FBEE9
:10CA1000CDBF1C012A013B014801590120E030E053
:10CA20004CE052E4C301B2010F94F3D425E535E59F
:10CA300047E052E40F94D4D56B017C010F94AAD641
:10CA40000F943CD68B0177FF12C020E030E040E825
:10CA50005FE3C701B6010F94D0D718160CF05DC084
:10CA6000C12CD12CE0E8EE2EEFE3FE2E56C066304E
:10CA70007105DCF02AEA3AE24CE453E4C301B20166
:10CA80000F94F3D425E535E547E052E40F94D4D56F
:10CA90006B017C0120E030E0A9010F94CDD587FF28
:10CAA0003FC0C12CD12C76013BC0882777FD8095F3
:10CAB000982F0F946FD625E535E547E052E40F94A3
:10CAC000A2D820E030E04CE052E40F94F4D49B0173
:10CAD000AC01C301B2010F94F3D425E535E547E07D
:10CAE00052E40F94D4D56B017C0120E030E0A90121
:10CAF0000F94CDD587FD17C020E030E040E85FE31C
:10CB0000C701B6010F94D0D7181684F4C12CD12CCC
:10CB100070E8E72E7FE3F72E09C000E010E006C0C2
:10CB200005E010E003C0C12CD12C760120E030E0FC
:10CB300040EC50E4C501B4010F94F3D42BEA3AEA77
:10CB400042E052E40F94D4D52B013C010F94AAD6B5
:10CB50000F943CD6788B6F8777FF12C020E030E0CF
:10CB600040E85FE3C301B2010F94D0D718160CF070
:10CB70005FC0412C512C60E8662E6FE3762E58C0C2
:10CB8000AF85B8891697E4F026E535E549E253E428
:10CB9000C501B4010F94F3D42BEA3AEA42E052E41F
:10CBA0000F94D4D52B013C0120E030E0A9010F9473
:10CBB000CDD587FD40C0E5E0F0E0F88BEF8746C0BB
:10CBC000882777FD8095982F0F946FD62BEA3AEA45
:10CBD00042E052E40F94A2D820E030E040EC50E470
:10CBE0000F94F4D49B01AC01C501B4010F94F3D4AC
:10CBF0002BEA3AEA42E052E40F94D4D52B013C01EF
:10CC000020E030E0A9010F94CDD587FD1CC020E0C5
:10CC100030E040E85FE3C301B2010F94D0D71816AB
:10CC2000ACF4412C512C50E8652E5FE3752E0EC0FC
:10CC3000188A1F860BC0412C512C320125E030E0B0
:10CC4000388B2F8703C0412C512C3201A70196014C
:10CC500060E070E080E89FE30F94F3D469837A8307
:10CC60008B839C83C80101969E838D83AF85B88991
:10CC70001196BA87A987A301920160E070E080E86D
:10CC80009FE30F94F3D46B877C878D879E8747E063
:10CC90002F853889429FF001439FF00D1124F887BA
:10CCA000EF83E00FF11FEE0FFF1FEE0FFF1FE20DEE
:10CCB000F31D218132814381548169817A818B8185
:10CCC0009C810F94A2D84B015C01EF81F8858D8186
:10CCD0009E81E80FF91FEE0FFF1FEE0FFF1FE20D01
:10CCE000F31D2181328143815481C701B6010F9424
:10CCF000A2D89B01AC01C501B4010F94F4D49B01EF
:10CD0000AC016B857C858D859E850F94A2D84B01E7
:10CD10005C0127E0E985FA852E9FD0012F9FB00D99
:10CD20001124B887AF83FD01E00FF11FEE0FFF1F45
:10CD3000EE0FFF1FE20DF31D2181328143815481EB
:10CD400069817A818B819C810F94A2D869837A83CF
:10CD50008B839C83AF81B8858D819E81A80FB91F7D
:10CD6000AA0FBB1FAA0FBB1FA20DB31D11962D91B9
:10CD70003D914D915C911497C701B6010F94A2D8D3
:10CD80009B01AC0169817A818B819C810F94F4D4E1
:10CD90009B01AC01C301B2010F94A2D89B01AC016D
:10CDA000C501B4010F94F4D460960FB6F894DEBFB9
:10CDB0000FBECDBFDF91CF911F910F91FF90EF90EC
:10CDC000DF90CF90BF90AF909F908F907F906F90AB
:10CDD0005F904F903F902F9008954F925F926F9287
:10CDE0007F929F92AF92BF92CF92DF92EF92FF928B
:10CDF0000F931F93CF93DF937C015B018A01E901BD
:10CE000090908A11911014C0FC0180819181A281BF
:10CE1000B381FA0180839183A283B383FB01808174
:10CE20009181A281B38188839983AA83BB837FC0C8
:10CE300091FE55C0FC012081318142815381609176
:10CE40007A1170917B1180917C1190917D110F94DA
:10CE5000A2D82B013C01F50120813181428153810F
:10CE600060917E1170917F1180918011909181115C
:10CE70000F94A2D89B01AC01C301B2010F94F4D46A
:10CE8000F8016083718382839383F701208131816C
:10CE9000428153816091821170918311809184113C
:10CEA000909185110F94A2D86B017C01F50120812E
:10CEB00031814281538160918611709187118091F7
:10CEC0008811909189110F94A2D89B01AC01C701E0
:10CED000B6010F94F4D4688379838A839B8390FE90
:10CEE00026C02091621130916311409164115091DC
:10CEF0006511F80160817181828193810F94F4D46E
:10CF0000F80160837183828393832091661130914D
:10CF100067114091681150916911688179818A8106
:10CF20009B810F94F4D4688379838A839B83DF91F8
:10CF3000CF911F910F91FF90EF90DF90CF90BF9016
:10CF4000AF909F907F906F905F904F9008952F9239
:10CF50003F924F925F926F927F928F929F92AF9289
:10CF6000BF92CF92DF92EF92FF920F931F93CF93D6
:10CF7000DF93CDB7DEB728970FB6F894DEBF0FBEAC
:10CF8000CDBF8C011B019E012F5F3F4FAE014B5F58
:10CF90005F4F23DF20E030E0A9016D817E818F812A
:10CFA00098850F94CDD587FF07C01D821E821F82F2
:10CFB0001886FF24F39401C0F12C20E030E040E417
:10CFC00051EC69817A818B819C810F94CDD587FF4B
:10CFD0000AC080E090E0A0E4B1EC89839A83AB833F
:10CFE000BC83FF24F39420E030E04FE753E46D81ED
:10CFF0007E818F8198850F94D0D7181654F480E0E5
:10D0000090E0AFE7B3E48D839E83AF83B887FF24BE
:10D01000F39420E030E042E553E469817A818B812A
:10D020009C810F94D0D718164CF480E090E0A2E5D4
:10D03000B3E489839A83AB83BC8303C0FF2009F4E4
:10D0400083C0C980DA80EB80FC808D809E80AF80B9
:10D05000B88470908A1171100BC0F801808291829F
:10D06000A282B382F101C082D182E282F3826AC0DD
:10D0700070FE1CC0209162113091631140916411C7
:10D0800050916511C501B4010F94F3D44B015C01BB
:10D09000209166113091671140916811509169118A
:10D0A000C701B6010F94F3D46B017C0171FE4AC035
:10D0B00020916A1130916B1140916C1150916D115A
:10D0C000C501B4010F94A2D82B013C0120916E112F
:10D0D00030916F114091701150917111C701B601DB
:10D0E0000F94A2D89B01AC01C301B2010F94F4D4F8
:10D0F000F801608371838283938320917211309150
:10D1000073114091741150917511C501B4010F94C0
:10D11000A2D84B015C01209176113091771140919A
:10D12000781150917911C701B6010F94A2D89B01D3
:10D13000AC01C501B4010F94F4D4F1016083718393
:10D1400082839383FF24F3948F2D28960FB6F8944F
:10D15000DEBF0FBECDBFDF91CF911F910F91FF902A
:10D16000EF90DF90CF90BF90AF909F908F907F9087
:10D170006F905F904F903F902F900895682F87EFAA
:10D180009FE00D9452E10895FC012491222341F087
:10D190003091C00035FFFCCF2093C6000196F4CF3C
:10D1A00022E030E086EC98E0F3CAFC0124912223CF
:10D1B00041F03091C00035FFFCCF2093C6000196AE
:10D1C000F4CF2AE030E086EC98E029CACF9362E7FA
:10D1D00073E086EC98E0DCD9C1E0C093B1026FEF58
:10D1E00089E69FE00F9452E1C093DE02CF9108954B
:10D1F00062E873E086EC98E0CBD91092B10260E06F
:10D2000089E69FE00F9452E11092DE020895EF92BA
:10D21000FF920F931F93CF93DF931F92CDB7DEB78B
:10D2200089830F94CA6D8981823009F468C0B4F58E
:10D23000882309F442C0813009F0F4C09FB7F89404
:10D24000809102018460809302019FBFEFEFF1EEB5
:10D2500024E0E150F0402040E1F700C000009FB71B
:10D26000F894809102018B7F809302019FBF40E080
:10D2700050E0BA018DEE9FE00F9464E140E050E091
:10D28000BA0181EF9FE00F9464E10F90DF91CF919D
:10D290001F910F91FF90EF900D949F91833009F4AF
:10D2A0005CC0843009F0BEC00F90DF91CF911F9118
:10D2B0000F91FF90EF900D9433BA9FB7F89480913F
:10D2C00002018460809302019FBF2FEF81EE94E002
:10D2D000215080409040E1F700C000009FB7F894D3
:10D2E000809102018B7F809302019FBF0F90DF919D
:10D2F000CF911F910F91FF90EF900D94746E0F944A
:10D30000746E80EF3BDF1092941A1092931A609122
:10D31000951A84EC9FE00F9452E163E97AE181EC85
:10D320009FE00F94F86D9FB7F8948091020184609C
:10D33000809302019FBF8FEF91EEE4E08150904017
:10D34000E040E1F700C000009FB7F894809102012F
:10D350008B7F809302019FBF65C087E09FE00F94A1
:10D36000748046EF5EE062E081E00F940E969FB716
:10D37000F894809102018460809302019FBFFFEFC7
:10D3800021EE84E0F15020408040E1F700C0000031
:10D390009FB7F894809102018B7F809302019FBF19
:10D3A0001092AA091092A9094FEE5EE063E083E0B3
:10D3B0000F940E964091A9095091AA0963E083E069
:10D3C0000F94D56DE12CF12C09E210E06FEFC7014D
:10D3D0000F9470E1C701B8010F9491DA892BD9F449
:10D3E0008091A9099091AA0901969093AA09809326
:10D3F000A90948EE5EE063E083E00F940E96409149
:10D40000A9095091AA0963E083E00F94D56D86EED7
:10D410009EE00F9474809FEFE91AF90AE114E0E1AD
:10D42000FE06A1F60F90DF91CF911F910F91FF9013
:10D43000EF9008958F929F92AF92BF92CF92DF921A
:10D44000EF92FF928091951A81119DC00F9400CDAB
:10D450006B017C0120911002222309F48CC04091C1
:10D460001502509116024130510509F484C0809193
:10D47000110290911202A0911302B0911402460180
:10D480005701881A990AAA0ABB0A30E0A8EEB3E04D
:10D490000F94E8DA86169706A806B9060CF473C04E
:10D4A0004430510559F13CF4423051050CF463C04D
:10D4B000E4E5FFE00EC04530510509F05CC0E4E54D
:10D4C000FFE042C09091C00095FFFCCF8093C60062
:10D4D000319684918111F6CFECEDFDE084918823A3
:10D4E00041F09091C00095FFFCCF8093C60031962B
:10D4F000F5CF8091C00085FFFCCF3AC0E4E5FFE0A6
:10D500008491882341F09091C00095FFFCCF8093D7
:10D51000C6003196F5CFE6ECFDE08491882341F01A
:10D520009091C00095FFFCCF8093C6003196F5CF57
:10D530008091C00085FFFCCF1BC09091C00095FF7B
:10D54000FCCF8093C600319684918111F6CFEFEA2B
:10D55000FDE08491882341F09091C00095FFFCCFBD
:10D560008093C6003196F5CF8091C00085FFFCCF37
:10D570008AE08093C600C0921102D0921202E0921B
:10D580001302F0921402FF90EF90DF90CF90BF90C3
:10D59000AF909F908F90089580E1ECE0FAE0A7EDC6
:10D5A000B9E001900D928A95E1F708954F925F924C
:10D5B0006F927F928F929F92AF92BF92CF92DF92A3
:10D5C000EF92FF92CF93DF9300D01F92CDB7DEB7DB
:10D5D0000F94BA3D8BE48DD9882391F0CCD96B019F
:10D5E0007C0120E030E0A9010F94D0D787FD08C06E
:10D5F000C0927212D0927312E0927412F09275126D
:10D6000082E577D9882359F0B6D96B017C0120E0F7
:10D6100030E0A9010F94CDD587FF83C006C0C12C8F
:10D62000D12C60E8E62E6FEBF62E84E462D98823D5
:10D6300021F0A1D94B015C0106C0812C912C50E84E
:10D64000A52E5FEBB52E87E554D9882321F093D919
:10D650002B013C0106C0412C512C40E8642E4FEBBD
:10D66000742E88E446D9882331F085D969837A837A
:10D670008B839C8308C080E090E0A0E8BFEB8983A7
:10D680009A83AB83BC8320E030E0A901C501B401DB
:10D690000F94D0D787FD45C020E030E0A901C30139
:10D6A000B2010F94D0D787FD3CC020E030E0A90143
:10D6B00069817A818B819C810F94D0D787FD31C09D
:10D6C00020E030E0A901C501B4010F94CDD5882335
:10D6D00091F120E030E040E05FE3C501B4010F9438
:10D6E000A2D86B017C0129813A814B815C81C30105
:10D6F000B2010F94A2D84B015C01A7019601C701AA
:10D70000B6010F94A2D82BED3FE049E450E40F940A
:10D71000A2D89B01AC01C501B4010F94D4D56B0113
:10D720007C0120E030E0A901C701B6010F94D0D7F9
:10D7300087FF04C00BC0C12CD12C7601C0926E12A1
:10D74000D0926F12E0927012F0927112E4E5FFE055
:10D750008491882341F09091C00095FFFCCF809385
:10D76000C6003196F5CFE2E7FAE08491882341F0D4
:10D770009091C00095FFFCCF8093C6003196F5CF05
:10D7800040917212509173126091741270917512DF
:10D7900022E030E086EC98E00E94C8638091C000EF
:10D7A00085FFFCCF8AE08093C600ECE6FAE0849126
:10D7B000882341F09091C00095FFFCCF8093C60074
:10D7C0003196F5CFC0906E12D0906F12E09070122B
:10D7D000F090711220E030E0A901C701B6010F946A
:10D7E000CDD5882369F022E030E0B701A60186ECB0
:10D7F00098E00E94C8638091C00085FFFCCF11C0F3
:10D80000E7E6FAE08491882341F09091C00095FF0B
:10D81000FCCF8093C6003196F5CF8091C00085FF84
:10D82000FCCF8AE08093C6000F900F900F900F906E
:10D83000DF91CF91FF90EF90DF90CF90BF90AF90AE
:10D840009F908F907F906F905F904F9008952F9250
:10D850003F924F925F926F927F928F929F92AF9280
:10D86000BF92CF92DF92EF92FF920F931F93CF93CD
:10D87000DF931F92CDB7DEB70F94CA6DE0EAFFE8E1
:10D880004591549161E080E00F940E9681E00F94F1
:10D890003F348983E7E1FFE0E4918E2F992781955A
:10D8A0000CF490951C0184E00F941E59A4E1BAE099
:10D8B0001D921D921D921C921397E0E1FAE02081C7
:10D8C000318142815381ACE0BAE06D917D918D91BF
:10D8D0009C91E8E1CE2EEAE0DE2EE12CF12C8701CE
:10D8E0000F94B93059DE8CE29FE00E94D1632DEC99
:10D8F0003CEC4CE85FE30F94A2D84B015C01B10112
:10D90000882777FD8095982F0F946FD69B01AC01E7
:10D91000C501B4010F94A2D8EFEDF9E02081318167
:10D92000428153810F94F4D42B013C01AFEDB9E057
:10D930006D937D938D939C931397E0E6F2E0608165
:10D9400071818281938160930C0270930D028093A8
:10D950000E0290930F0220E030E040E752E40F9473
:10D96000D4D54B015C01ABEDB9E02D913D914D91CA
:10D970005C91E7EDF9E06081718182819381A8EF8C
:10D98000B9E0BF93AF93F3EECF2EF9E0DF2E830122
:10D9900072010F940B2482E00F9493560F94BA3DBA
:10D9A0000F949E5980E00F943F34A4E1BAE01D9299
:10D9B0001D921D921C921397E0E1FAE020813181C3
:10D9C00042815381ACE0BAE06D917D918D919C9143
:10D9D000A8E1CA2EAAE0DA2EE12CF12C87010F94DF
:10D9E000B930DADD8AE0829DB001839D700D11248B
:10D9F000882777FD8095982F0F946FD6EFEDF9E08B
:10DA000020813181428153810F94F4D42B013C0158
:10DA1000AFEDB9E06D937D938D939C93139720E0C8
:10DA200030E040E05FE3E0E6F2E060817181828116
:10DA300093810F94A2D860930C0270930D0280938F
:10DA40000E0290930F0220E030E040E752E40F9482
:10DA5000D4D54B015C01ABEDB9E02D913D914D91D9
:10DA60005C91E7EDF9E06081718182819381A8EF9B
:10DA7000B9E0BF93AF93B3EECB2EB9E0DB2E8301B9
:10DA800072010F940B240F94BA3D89810F943F3497
:10DA900080E090E0A4E5B3E4E4E1FAE080839183E0
:10DAA000A283B383A0E1BAE02D913D914D915C91A9
:10DAB000ECE0FAE0608171818281938118E1C12EEE
:10DAC0001AE0D12EE12CF12C04E513E40F94B930C7
:10DAD00081E00F900F900F900F900F90DF91CF91FA
:10DAE0001F910F91FF90EF90DF90CF90BF90AF907C
:10DAF0009F908F907F906F905F904F903F902F906E
:10DB000008952F923F924F925F926F927F928F92E1
:10DB10009F92AF92BF92CF92DF92EF92FF920F93BC
:10DB20001F93CF93DF93CDB7DEB729970FB6F89445
:10DB3000DEBF0FBECDBF3C0181E00F943F348F8329
:10DB400082E06816710408F081C2F301EB5EF04FC9
:10DB5000E491D301AA0FBB1FAA0FBB1FBA83A983ED
:10DB6000A85ABD4FBE83AD838D919D910D90BC9100
:10DB7000A02D80930C0290930D02A0930E02B093FF
:10DB80000F0281E0062C01C0880F0A94EAF70F9477
:10DB90001E59E981FA81E45FF54FF987E887108221
:10DBA000118212821382E090140AF090150A0091FB
:10DBB000160A1091170A2091100A3091110A40910B
:10DBC000120A5091130A60910C0A70910D0A80910B
:10DBD0000E0A90910F0AE8E1CE2EEAE0DE2E0F94B5
:10DBE000B930E981FA81E952F64F2F0180E090E0E7
:10DBF000A0E4B0E480839183A283B38320E030E08B
:10DC000040E752E460910C0270910D0280910E0287
:10DC100090910F020F94D4D54B015C01E090DF0985
:10DC2000F090E0090091E1091091E2092091DB09EF
:10DC30003091DC094091DD095091DE096091D709EE
:10DC40007091D8098091D9099091DA09F8EF2F2EB7
:10DC5000F9E03F2E3F922F92A3EECA2EA9E0DA2ED2
:10DC60000F940B240F94BA3D0F94273480E00F9447
:10DC70003F34A885B9851D921D921D921C92139761
:10DC8000E090140AF090150A0091160A1091170AF4
:10DC90002091100A3091110A4091120A5091130AF2
:10DCA00060910C0A70910D0A80910E0A90910F0AF2
:10DCB000B8E1CB2EBAE0DB2E0F94B93080E090E0D3
:10DCC000A0E8BFEBF20180839183A283B38320E0BD
:10DCD00030E040E752E460910C0270910D028091B7
:10DCE0000E0290910F020F94D4D54B015C01E0908D
:10DCF000DF09F090E0090091E1091091E20920911B
:10DD0000DB093091DC094091DD095091DE09609119
:10DD1000D7097091D8098091D9099091DA093F9279
:10DD20002F92E3EECE2EE9E0DE2E0F940B240F941B
:10DD3000BA3D81E00F943F3489819A818C5D904F88
:10DD40000E94D1632DEC3CEC4CE85FEB0F94A2D821
:10DD5000D2016D937D938D939C93139720E030E0D7
:10DD600040E752E460910C0270910D0280910E0226
:10DD700090910F020F94D4D54B015C01E090DF0924
:10DD8000F090E0090091E1091091E2092091DB098E
:10DD90003091DC094091DD095091DE096091D7098D
:10DDA0007091D8098091D9099091DA093F922F9208
:10DDB0000F940B240F94BA3D0F94273480E00F94F6
:10DDC0003F34E885F9851082118212821382E09037
:10DDD000140AF090150A0091160A1091170A209162
:10DDE000100A3091110A4091120A5091130A609161
:10DDF0000C0A70910D0A80910E0A90910F0AF8E1B9
:10DE0000CF2EFAE0DF2E0F94B93080E090E0A0E250
:10DE1000B1E4F20180839183A283B38320E030E0F8
:10DE200040E752E460910C0270910D0280910E0265
:10DE300090910F020F94D4D54B015C01E090DF0963
:10DE4000F090E0090091E1091091E2092091DB09CD
:10DE50003091DC094091DD095091DE096091D709CC
:10DE60007091D8098091D9099091DA093F922F9247
:10DE7000A3EECA2EA9E0DA2E0F940B240F94BA3D1C
:10DE80000F94273481E00F943F3480E090E0A0E7C6
:10DE9000B1ECF20180839183A283B38320E030E070
:10DEA00040E05FE3AD81BE816D917D918D919C914C
:10DEB0000F94A2D860930C0270930D0280930E020F
:10DEC00090930F0220E030E040E752E40F94D4D565
:10DED0004B015C01E090DF09F090E0090091E1095D
:10DEE0001091E2092091DB093091DC094091DD09B4
:10DEF0005091DE096091D7097091D8098091D909B4
:10DF00009091DA093F922F920F940B240F94BA3D0F
:10DF1000C3010E94D763F301E350F64F81E0808391
:10DF20000F949E590F94273480E00F943F342AE0D9
:10DF300037ED43E25FE3E885F98560817181828195
:10DF400093810F94F3D4A885B9856D937D938D93B8
:10DF50009C931397E090140AF090150A0091160A0A
:10DF60001091170A2091100A3091110A4091120A5B
:10DF70005091130A60910C0A70910D0A80910E0A5B
:10DF800090910F0AB8E1CB2EBAE0DB2E0F94B93096
:10DF90002AE037ED43E25FE3E885F985608171812E
:10DFA000828193810F94F4D4A885B9856D937D9374
:10DFB0008D939C931397F201608371838283938383
:10DFC0002AE939E949E95EE360910C0270910D029A
:10DFD00080910E0290910F020F94A2D820E030E0C1
:10DFE00040E752E40F94D4D54B015C01E090DF0987
:10DFF000F090E0090091E1091091E2092091DB091C
:10E000003091DC094091DD095091DE096091D7091A
:10E010007091D8098091D9099091DA093F922F9295
:10E02000E3EECE2EE9E0DE2E0F940B240F94BA3DE2
:10E0300010920C0210920D0210920E0210920F021A
:10E040000FB6F894DEBF0FBECDBF62C192E0691675
:10E05000710409F05DC1E7E1FFE074901092140AC9
:10E060001092150A1092160A1092170A2091100A9F
:10E070003091110A4091120A5091130A60910C0AD2
:10E0800070910D0A80910E0A90910F0AF8E1CF2E3F
:10E09000FAE0DF2EE12CF12C87010F94B9308CE2ED
:10E0A0009FE00E94D1634B015C01672D772767FDDC
:10E0B0007095872F972F0F946FD62B013C0120E08E
:10E0C00030E040EC5FE3C501B4010F94A2D8A30196
:10E0D00092010F94A2D869837A838B839C83609387
:10E0E000DF097093E0098093E1099093E209609160
:10E0F000600270916102809162029091630260936C
:10E100000C0270930D0280930E0290930F0220E098
:10E1100030E040E752E40F94D4D54B015C012091EC
:10E12000DB093091DC094091DD095091DE096091F5
:10E13000D7097091D8098091D9099091DA09A8EF8F
:10E140002A2EA9E03A2E3F922F92B3EECB2EB9E0C1
:10E15000DB2EE980FA800B811C810F940B240F9435
:10E16000BA3D1092140A1092150A1092160A1092D3
:10E17000170A2091100A3091110A4091120A509109
:10E18000130A60910C0A70910D0A80910E0A909109
:10E190000F0A18E1C12E1AE0D12EE12CF12C8701D3
:10E1A0000F94B93080E29FE00E94D1639058A301A0
:10E1B00092010F94A2D869837A838B839C836093A6
:10E1C000DF097093E0098093E1099093E20920E070
:10E1D00030E040E752E460910C0270910D028091B2
:10E1E0000E0290910F020F94D4D54B015C01209147
:10E1F000DB093091DC094091DD095091DE09609125
:10E20000D7097091D8098091D9099091DA093F9284
:10E210002F9203EEC02E09E0D02EE980FA800B8108
:10E220001C810F940B240F94BA3D80E29FE00E9462
:10E23000D1639B01AC010F94F4D4A30192010F941C
:10E24000A2D82B013C016093DF097093E009809311
:10E25000E1099093E20920E030E040E05FE3609163
:10E2600060027091610280916202909163020F944A
:10E27000A2D860930C0270930D0280930E029093CB
:10E280000F0220E030E040E752E40F94D4D54B0178
:10E290005C012091DB093091DC094091DD0950914E
:10E2A000DE096091D7097091D8098091D9099091C0
:10E2B000DA093F922F92830172010F940B240F947D
:10E2C000BA3D82E090E00E94D7638091140A909159
:10E2D000150AA091160AB091170A8093DF0990934E
:10E2E000E009A093E109B093E20910920C021092A8
:10E2F0000D0210920E0210920F020F94273481E04B
:10E300008093FF090F900F900F900F900F900F9038
:10E310008F8129960FB6F894DEBF0FBECDBFDF9177
:10E32000CF911F910F91FF90EF90DF90CF90BF9012
:10E33000AF909F908F907F906F905F904F903F90A5
:10E340002F900D943F34CF92DF92EF92FF920F9374
:10E350001F9322D980E090E0D4DB81E090E0D1DB14
:10E36000E090140AF090150A0091160A1091170A0D
:10E370002091100A3091110A4091120A5091130A0B
:10E3800060910C0A70910D0A80910E0A90910F0A0B
:10E39000F8E1CF2EFAE0DF2E0F94B9301F910F91E4
:10E3A000FF90EF90DF90CF900D9427340F9400CD25
:10E3B0006093BE097093BF098093C0099093C1090F
:10E3C000089520E030E0A90168EB71E084E50F9446
:10E3D0004ED169E170E080E090E00F942FCD84E5AC
:10E3E0000F9472D464E170E080E090E00D942FCD42
:10E3F0007F928F929F92AF92BF92CF92DF92EF92D5
:10E40000FF920F931F93CF93DF9300D01F92CDB74E
:10E41000DEB710928B1910928A19109289191092F6
:10E4200088190F94CA6D8DEE9DE00F9474808E0153
:10E430000F5F1F4F7E0125E0E20EF11C86EC98E095
:10E440000E94E2618F3FEFEF9E07C1F3F8018193D5
:10E450008F01EE15FF0591F789809A80AB80BC8013
:10E460008091C00085FFFCCF8BE28093C600C12C59
:10E47000D12C7601ABE27A2E8091400A882309F4F0
:10E4800050C008E619E0C814D904EA04FB04A1F05E
:10E4900086EC98E00E94E2618F3FFFEF9F07C1F397
:10E4A0002FEFC21AD20AE20AF20AF80181938F0111
:10E4B000F9E0083A1F0739F768E679E08FE79AE054
:10E4C0000E94CAD98091C00085FFFCCF7092C6001F
:10E4D0000F94184FC814D904EA04FB0469F671DFDD
:10E4E00060E08FE79AE00E94FDDA1092400AE4ECC7
:10E4F000FEE885919491FC012491222341F0309112
:10E50000C00035FFFCCF2093C6000196F4CF809168
:10E51000C00085FFFCCF8AE08093C60080E090E0D9
:10E5200000C00F900F900F900F90DF91CF911F912F
:10E530000F91FF90EF90DF90CF90BF90AF909F90A2
:10E540008F907F9008952F923F924F925F926F929B
:10E550007F928F929F92AF92BF92CF92DF92EF9273
:10E56000FF920F931F93CF93DF931F921F92CDB70C
:10E57000DEB7382E811112C01092891910928819B5
:10E5800010928B1910928A1910928D1910928C1971
:10E5900010928F1910928E190F941F6E80E00F94B5
:10E5A00041B28BE891E10F94F5180E945CFA0F9448
:10E5B00046181092FD091092FE091092FF0981E0A1
:10E5C0000E942564E091410AF0E0EE0FFF1FE05247
:10E5D000FF4685919491BE016F5F7F4F0F9480B28B
:10E5E000B2DE35D9882309F471C1E0DE311046C0AE
:10E5F00084E090E09093160280931502ECE9F9E82C
:10E600008591949140E060E00F9439B4882331F013
:10E61000E4ECFBE8859194910F9429BCE091410AC8
:10E62000F0E0EE0FFF1FE256F347859194910F94AF
:10E6300029BC82E090E09093160280931502E0914D
:10E64000410AF0E0EE0FFF1FE455F14785919491E8
:10E65000BE016F5F7F4F0F9480B241E050E062E0F7
:10E6600080E00F94D56DE091410AF0E0EE0FFF1FBE
:10E67000E056F147859194910F94748080E090E08A
:10E68000A0EAB0E48093140A9093150AA093160AA6
:10E69000B093170A20E030E040E252E4609160025B
:10E6A0007091610280916202909163020F94D4D5BF
:10E6B0004B015C012091100A3091110A4091120A1D
:10E6C0005091130A60910C0A70910D0A80910E0A04
:10E6D00090910F0AE8EFF9E0FF93EF93E8E1CE2E77
:10E6E000EAE0DE2EE12CF12C00EA10E40F940B247A
:10E6F0000F94BA3D86E50E9479640F900F908823AD
:10E7000061F0E0914E0FF0914F0F8181893039F027
:10E710008F7D41F00E948F6403C01A8205C081E0A2
:10E720008A8302C0A1E0AA833320B1F00E9453641F
:10E730000E94B1FA0E94CDFC0F94A111882309F424
:10E74000C1C087EF9FE00F9440E1803F09F0BAC05D
:10E7500081E00E94BE68B6C08FEF0E94BE6860E094
:10E7600070E088EF9FE00F946CE11982BE016F5F4B
:10E770007F4F8A810F94720E3C010E945364212CBA
:10E78000312C10EA412E10E4512E2092140A3092BE
:10E79000150A4092160A5092170A20E030E040E233
:10E7A00052E46091600270916102809162029091E6
:10E7B00063020F94D4D54B015C012091100A309173
:10E7C000110A4091120A5091130A60910C0A70913B
:10E7D0000D0A80910E0A90910F0AA8EFB9E0BF933D
:10E7E000AF9308E1C02E0AE0D02E820171010F9490
:10E7F0000B240F94BA3D0F900F9077FC47C01982FD
:10E800008BE891E10F94F5180E9423FA81E00E94B1
:10E81000256499DDAE014F5F5F4F6A8181E00F94FF
:10E82000C7133C010E9453642092140A3092150AC7
:10E830004092160A5092170A20E030E040E252E47B
:10E840006091600270916102809162029091630216
:10E850000F94D4D54B015C012091100A3091110A1C
:10E860004091120A5091130A60910C0A70910D0A9E
:10E8700080910E0A90910F0AA8EFB9E0BF93AF9371
:10E880000F940B240F94BA3D0F900F906981C30130
:10E890000F9493BC77FC16C086EE0E94BE688FE58D
:10E8A0009FE00F9440E1813059F0E091410AF0E09F
:10E8B000EE0FFF1FEA53FF46859194910F9429BCF8
:10E8C00011E001C010E00F949E5901C010E081E0FA
:10E8D0000F9441B2812F0F900F90DF91CF911F9134
:10E8E0000F91FF90EF90DF90CF90BF90AF909F90EF
:10E8F0008F907F906F905F904F903F902F900895F2
:10E900008F929F92AF92BF92CF92DF92EF92FF923F
:10E910000F931F93CF93DF93159881E08093350A6F
:10E9200082E090E09093330A8093320AE091410AAA
:10E93000F0E0EE0FFF1FEA53F247859194910F9498
:10E94000E36E20E030E04CE852E46091180A7091E8
:10E95000190A80911A0A90911B0A0F94F4D46093BB
:10E96000180A7093190A80931A0A90931B0AE09070
:10E97000140AF090150A0091160A1091170A2091B6
:10E98000100A3091110A4091120A5091130A6091B5
:10E990000C0A70910D0A80910E0A90910F0AC8EF2F
:10E9A000D9E0DF93CF93812C912CE0ECAE2EE0E404
:10E9B000BE2EF8E1CF2EFAE0DF2E0F940B2420E0DC
:10E9C00030E048EC51E46091180A7091190A809186
:10E9D0001A0A90911B0A0F94F4D46093180A70934A
:10E9E000190A80931A0A90931B0AE090140AF09077
:10E9F000150A0091160A1091170A2091100A3091F9
:10EA0000110A4091120A5091130A60910C0A7091F8
:10EA10000D0A80910E0A90910F0ADF93CF93812CFB
:10EA2000912CA0E8AA2EAFE3BA2E0F940B240F94DA
:10EA3000BA3D0F900F900F900F908091951A8823F8
:10EA400031F181E00F9441B282E00F947AAFE0910E
:10EA5000410AF0E0EE0FFF1FEE54F84785919491C4
:10EA60000F94E36E1092340A1092350A1092330A12
:10EA70001092320ADF91CF911F910F91FF90EF908A
:10EA8000DF90CF90BF90AF909F908F90089580912E
:10EA9000340A8823B1F2E091410AF0E0EE0FFF1F43
:10EAA000E853F1478591949141E060E00F9439B4C7
:10EAB00091E0811101C090E0C8EFD9E09111C1CF80
:10EAC00081E00F9441B282E00F947AAF20E030E011
:10EAD00048EC51E46091180A7091190A80911A0A61
:10EAE00090911B0A0F94F4D46093180A7093190A3A
:10EAF00080931A0A90931B0AE090140AF090150A6A
:10EB00000091160A1091170A2091100A3091110AEB
:10EB10004091120A5091130A60910C0A70910D0AEB
:10EB200080910E0A90910F0ADF93CF93812C912C44
:10EB3000E0E8AE2EEFE3BE2EF8E1CF2EFAE0DF2EB6
:10EB40000F940B240F94BA3DE091410AF0E0EE0FD0
:10EB5000FF1FE853F1478591949141E060E00F94E5
:10EB600039B40F900F9081116CCFAACF0F9400CDC4
:10EB70006093BE097093BF098093C0099093C10947
:10EB8000E091580FF091590FE65AF04F8081813093
:10EB9000B9F4EAEAFCE885919491FC0124912223DE
:10EBA00041F03091C00035FFFCCF2093C6000196A4
:10EBB000F4CF8091C00085FFFCCF8AE08093C6002F
:10EBC000089586EC98E00E94FE61E2ECFBE88591F6
:10EBD0009491FC012491222341F03091C00035FF33
:10EBE000FCCF2093C6000196F4CF40913E0F509188
:10EBF0003F0F6091400F7091410F4F5F5F4F6F4F1C
:10EC00007F4F2AE030E086EC98E00E949D62809180
:10EC1000C00085FFFCCF8AE08093C600A7CF8F920B
:10EC20009F92AF92BF92CF92DF92EF92FF920F939B
:10EC30001F93CF93DF93BCE4EB2EB5E0FB2E0CE0EB
:10EC40001AE0C7EDD9E087E7C82E8AE0D82EF70191
:10EC500081917F010E947964882319F10E94E66402
:10EC60004B015C01F6018081811103C06091C209F2
:10EC700001C061E070E080E090E00F946FD6F80191
:10EC800020813181428153810F94A2D89B01AC0134
:10EC9000C501B4010F94F4D4688379838A839B837C
:10ECA00009C0F80180819181A281B3818883998311
:10ECB000AA83BB830C5F1F4F2496FFEFCF1ADF0A96
:10ECC00080E5E81685E0F80611F686E40E9479648E
:10ECD0008823D9F00E94E6646B017C016093C70928
:10ECE0007093C8098093C9099093CA0920E030E065
:10ECF000A9010F94D0D7181644F4C0920C02D092F8
:10ED00000D02E0920E02F0920F02DF91CF911F915F
:10ED10000F91FF90EF90DF90CF90BF90AF909F90BA
:10ED20008F9008957CDF89E40E947964882359F0EC
:10ED30000E94E6646093CB097093CC098093CD095F
:10ED40009093CE0908C01092CB091092CC09109272
:10ED5000CD091092CE098AE40E947964882359F083
:10ED60000E94E6646093CF097093D0098093D10923
:10ED70009093D20908951092CF091092D009109261
:10ED8000D1091092D2090895CF92DF92EF92FF92AB
:10ED9000CF93DF93EC01BC016C5F7F4F0E94A767AC
:10EDA00020E030E0A90160913C0270913D02809129
:10EDB0003E0290913F020F94F4D46B017C019B01C1
:10EDC000AC01688579858A859B850F94CDD587FFB1
:10EDD00004C0C886D986EA86FB86C0903002D090EF
:10EDE0003102E0903202F0903302A701960168856B
:10EDF00079858A859B850F94D0D7181624F4C88608
:10EE0000D986EA86FB86DF91CF91FF90EF90DF9065
:10EE1000CF9008952F923F924F925F926F927F9280
:10EE20008F929F92AF92BF92CF92DF92EF92FF921A
:10EE30000F931F93CF93DF93CDB7DEB7AB970FB68A
:10EE4000F894DEBF0FBECDBF9F878E87798B688B0E
:10EE50005B8B4A8B3D8B2C8B1F8B0E8BED82DC01E9
:10EE60008D909D90AD90BC9040900C0A50900D0AF2
:10EE700060900E0A70900F0ADB018D919D910D90AC
:10EE8000BC91A02D88879987AA87BB87C090100A5C
:10EE9000D090110AE090120AF090130A2091140AFF
:10EEA0003091150A4091160A5091170AEA89FB8998
:10EEB00060817181828193810F94F3D4688F798FFF
:10EEC0008A8F9B8F80918B11811173C0AE89BF890E
:10EED0008D909D90AD90BC90EA89FB89E080F18097
:10EEE00002811381A889B9892D913D914D915C9141
:10EEF000EE85FF856081718182819381FE01359667
:10EF0000FF93EF93CC88DD880F940B24EE85FF856B
:10EF100080819181A281B38180930C0A90930D0A24
:10EF2000A0930E0AB0930F0AE889F9898081918134
:10EF3000A281B3818093100A9093110AA093120AC0
:10EF4000B093130AEA89FB8980819181A281B38100
:10EF50008093140A9093150AA093160AB093170A87
:10EF6000EC89FD8980819181A281B3818093180A07
:10EF70009093190AA0931A0AB0931B0A0F900F904E
:10EF8000AB960FB6F894DEBF0FBECDBFDF91CF9129
:10EF90001F910F91FF90EF90DF90CF90BF90AF90B7
:10EFA0009F908F907F906F905F904F903F902F90A9
:10EFB0000895A3019201C501B4010F94F3D42B016C
:10EFC0003C0120E030E0A9010F94D0D75301420169
:10EFD000181624F0B7FAB094B7F8B094A7019601C8
:10EFE000688579858A859B850F94F3D468877987AE
:10EFF0008A879B8720E030E0A9010F94D0D728852D
:10F0000039854A855B8518160CF05058C501B40146
:10F010000F94F4D46B017C0120E030E0A9010F943F
:10F02000D0D718160CF052CF20E030E040EF51E47A
:10F03000C701B6010F94D4D50F94BAD50F943CD61E
:10F040007D876C87623071050CF440CF2091180ADF
:10F050003091190A40911A0A50911B0AAC89BD8956
:10F060006D917D918D919C910F94F3D46C8F7D8FD8
:10F070008E8F9F8F22242394312C8C859D85AA27E7
:10F0800097FDA095BA2F88A799A7AAA7BBA7DE01CD
:10F090001596BF83AE83B101882777FD8095982FA1
:10F0A0000F946FD66B017C0168A579A58AA59BA5F5
:10F0B0000F946FD69B01AC01C701B6010F94D4D554
:10F0C0006B017C01EE89FF8980809180A280B380F2
:10F0D0002C8D3D8D4E8D5F8D0F94A2D89B01AC0180
:10F0E0006091180A7091190A80911A0A90911B0A6E
:10F0F0000F94F4D469837A838B839C83288D398D14
:10F100004A8D5B8DC701B6010F94A2D82091140AD5
:10F110003091150A4091160A5091170A0F94F4D4B1
:10F1200068A379A38AA39BA3288539854A855B8533
:10F13000C701B6010F94A2D82091100A3091110A8C
:10F140004091120A5091130A0F94F4D46CA37DA33A
:10F150008EA39FA3A3019201C701B6010F94A2D869
:10F1600020910C0A30910D0A40910E0A50910F0A1D
:10F170000F94F4D4FF81FF932E812F93DE0111961B
:10F180006D01E8A0F9A00AA11BA12CA13DA14EA1EF
:10F190005FA10F940B24BFEF2B1A3B0A0F900F9027
:10F1A000EC85FD852E163F0609F075CF8FCE4F9268
:10F1B0005F926F927F928F929F92AF92BF92CF9207
:10F1C000DF92EF92FF920F931F93CF93DF93CDB710
:10F1D000DEB728970FB6F894DEBF0FBECDBF87ED20
:10F1E00099E0D2DD0F9400CD6093BE097093BF0902
:10F1F0008093C0099093C1098091D7099091D80953
:10F20000A091D909B091DA098D839E83AF83B88725
:10F210009C01AD0160910C0A70910D0A80910E0A5B
:10F2200090910F0A0F94CDD5811197C04090DB09C2
:10F230005090DC096090DD097090DE09A301920115
:10F240006091100A7091110A8091120A9091130A2C
:10F250000F94CDD5811181C020E030E040E752E429
:10F2600060910C0270910D0280910E0290910F023C
:10F270000F94D4D54B015C01E090DF09F090E009D8
:10F280000091E1091091E20988EF99E09F938F9333
:10F2900023EEC22E29E0D22EA30192016D817E8140
:10F2A0008F8198850F940B240F900F908091D70930
:10F2B0009091D809A091D909B091DA0980930C0AEC
:10F2C00090930D0AA0930E0AB0930F0A8091DB0968
:10F2D0009091DC09A091DD09B091DE098093100ABC
:10F2E0009093110AA093120AB093130A8091DF0938
:10F2F0009091E009A091E109B091E2098093140A8C
:10F300009093150AA093160AB093170A8091E30907
:10F310009091E409A091E509B091E6098093180A5B
:10F320009093190AA0931A0AB0931B0A28960FB655
:10F33000F894DEBF0FBECDBFDF91CF911F910F912B
:10F34000FF90EF90DF90CF90BF90AF909F908F9005
:10F350007F906F905F904F900895E090F8096091D2
:10F36000560270915702882777FD8095982F0F9449
:10F370006FD620910C0230910D0240910E025091F7
:10F380000F020F94A2D82EE333EC4EE259E30F9410
:10F39000A2D869837A838B839C838E010F5F1F4F72
:10F3A00023EE39E04FED59E06BED79E087ED99E020
:10F3B00031DD7CCF4F925F926F927F928F929F92BE
:10F3C000AF92BF92CF92DF92EF92FF920F931F9373
:10F3D000CF93C62FE091F809F0E0882309F4D9C053
:10F3E000DF01AC50B64F8C918111AFC180910C0AF6
:10F3F00090910D0AA0910E0AB0910F0A8093D7093F
:10F400009093D809A093D909B093DA098091100A92
:10F410009091110AA091120AB091130A8093DB090E
:10F420009093DC09A093DD09B093DE098091140A62
:10F430009091150AA091160AB091170A8093DF09DE
:10F440009093E009A093E109B093E209C090180AF3
:10F45000D090190AE0901A0AF0901B0AC092E309B2
:10F46000D092E409E092E509F092E609EE0FFF1F61
:10F47000EE0FFF1FE05CFD4F2081318142815381FF
:10F48000662349F06091200270912102809122024E
:10F490009091230208C0609124027091250280910E
:10F4A0002602909127020F94D4D59B01AC01C7018D
:10F4B000B6010F94F4D46093180A7093190A8093DC
:10F4C0001A0A90931B0A88E19AE00F9464328090A4
:10F4D0000C0290900D02A0900E02B0900F0220E05E
:10F4E00030E040E752E460911C0270911D0280916F
:10F4F0001E0290911F020F94A2D860930C02709389
:10F500000D0280930E0290930F02E091F809F0E053
:10F51000EC50F64F81E080834ADE2091F009309173
:10F52000F1094091F2095091F3096091140A709128
:10F53000150A8091160A9091170A0F94F3D47B0153
:10F540008C016093140A7093150A8093160A9093A5
:10F55000170A2091100A3091110A4091120A509115
:10F56000130A60910C0A70910D0A80910E0A909115
:10F570000F0AE8E1CE2EEAE0DE2E0F94B93017DE56
:10F5800080920C0290920D02A0920E02B0920F0295
:10F59000DCC0EC50F64F8081882309F4D6C08090FF
:10F5A0000C0A90900D0AA0900E0AB0900F0A80925B
:10F5B000D7099092D809A092D909B092DA0940905F
:10F5C000100A5090110A6090120A7090130A40922B
:10F5D000DB095092DC096092DD097092DE096091CE
:10F5E000140A7091150A8091160A9091170A609377
:10F5F000DF097093E0098093E1099093E20900919B
:10F60000180A1091190A20911A0A30911B0A0093C6
:10F61000E3091093E4092093E5093093E60920916A
:10F62000F0093091F1094091F2095091F3090F94DA
:10F63000F4D47B018C016093140A7093150A8093B3
:10F64000160A9093170A38E1C32E3AE0D32EA3018D
:10F650009201C501B4010F94B9301091F809CC237F
:10F6600089F02091E8093091E9094091EA09509127
:10F67000EB09609120027091210280912202909109
:10F68000230210C02091EC093091ED094091EE0960
:10F690005091EF0960912402709125028091260219
:10F6A000909127020F94F4D424E0129FF0011124CA
:10F6B000E05CFD4F20813181428153810F94D4D58C
:10F6C0009B01AC016091180A7091190A80911A0A85
:10F6D00090911B0A0F94F3D46093180A7093190A3F
:10F6E00080931A0A90931B0A88E19AE00F9464327F
:10F6F000C0900C02D0900D02E0900E02F0900F022C
:10F7000020E030E040E752E4609118027091190265
:10F7100080911A0290911B020F94A2D860930C0260
:10F7200070930D0280930E0290930F02E091F809FE
:10F73000F0E0EC50F64F10823ADDC0920C02D0920D
:10F740000D02E0920E02F0920F02CF911F910F91E5
:10F75000FF90EF90DF90CF90BF90AF909F908F90F1
:10F760007F906F905F904F900895AF92BF92CF922D
:10F77000DF92EF92FF920F931F93CF93DF93D82FD7
:10F780002091CF093091D0094091D1095091D209EF
:10F790006091CB097091CC098091CD099091CE09EF
:10F7A0000F94DDD7C62F172F082FF92E6091560220
:10F7B00070915702882777FD8095982F0F946FD608
:10F7C00020910C0230910D0240910E0250910F02D7
:10F7D0000F94A2D820E030E040E752E40F94D4D553
:10F7E00020E030E048EC52E40F94D4D52091F809A1
:10F7F0002F93DF93FF920F931F93CF935B016C01C5
:10F80000B2E0EB2E01E020E04BEC59E067ED79E04F
:10F810008CE09AE00F94DA1A8091D7099091D80978
:10F82000A091D909B091DA0980930C0A90930D0A3E
:10F83000A0930E0AB0930F0A8091DB099091DC0926
:10F84000A091DD09B091DE098093100A9093110A0E
:10F85000A093120AB093130A8091DF099091E009F6
:10F86000A091E109B091E2098093140A9093150ADE
:10F87000A093160AB093170A8091E3099091E409C6
:10F88000A091E509B091E6098093180A9093190AAE
:10F89000A0931A0AB0931B0A0F9400CD6093BE097F
:10F8A0007093BF098093C0099093C1090F900F9086
:10F8B0000F900F900F900F90DF91CF911F910F91AC
:10F8C000FF90EF90DF90CF90BF90AF900895CF93CF
:10F8D000DF931F92CDB7DEB78C01E0E6FAE08491AA
:10F8E000882341F09091C00095FFFCCF8093C60023
:10F8F0003196F5CF70E04AE050E086EC98E00E9447
:10F90000DC62F8940F94B247179A1092FD09169A88
:10F910001092FE09149AEAE5FFE08491882341F0F1
:10F920009091C00095FFFCCF8093C6003196F5CF33
:10F93000E6E0FFE885919491FC012491222341F0B7
:10F940003091C00035FFFCCF2093C6000196F4CF64
:10F950008091C00085FFFCCF8AE08093C60001152E
:10F960001105E1F0F8018491F801882349F09091A4
:10F97000C00095FFFCCF8093C60031968491F5CFEF
:10F980008091C00085FFFCCF8AE08093C600BE0155
:10F990006F5F7F4FC8010F9480B20BC0E091410AA6
:10F9A000F0E0EE0FFF1FEE5FF147859194910F9409
:10F9B0000E6F789406E010E00150110951F068ECE8
:10F9C00070E080E090E00F942FCD80E00F947AAF4C
:10F9D000F3CFF894FFCFCF92DF92EF92FF920F9385
:10F9E0001F93CF93C82F8091540F9091550F039779
:10F9F00014F40E9457E30F9400CD0091BA091091BE
:10FA0000BB092091BC093091BD09C090BE09D090BE
:10FA1000BF09E090C009F090C1096C197D098E09F9
:10FA20009F09061717072807390740F4012B022BF7
:10FA3000032B21F064E083E697E049DF4091080260
:10FA40005091090260910A0270910B02452B462BDE
:10FA5000472B19F10F9400CD0091BE091091BF09F9
:10FA60002091C0093091C109601B710B820B930B6F
:10FA7000009108021091090220910A0230910B02B4
:10FA8000061717072807390740F4909177128091DD
:10FA90007612981302C0CC2349F0CF911F910F9199
:10FAA000FF90EF90DF90CF900D943922179A10922B
:10FAB000FD09169A1092FE09149AEFCF0F94B247DF
:10FAC0008091AC09811142C081E08093AC098091A2
:10FAD0003E0F90913F0FA091400FB091410F809346
:10FAE0003A0F90933B0FA0933C0FB0933D0FEAE584
:10FAF000FFE08491882341F09091C00095FFFCCFF6
:10FB00008093C6003196F5CFECEFFEE88591949195
:10FB1000FC012491222341F03091C00035FFFCCF3D
:10FB20002093C6000196F4CF8091C00085FFFCCFE2
:10FB30008AE08093C600E091410AF0E0EE0FFF1FDB
:10FB4000E257F647859194910D94E36E0895809164
:10FB5000AC090895CF93DF93EC018091F80980936D
:10FB6000AD0984E50E947964811102C080E084C0FF
:10FB70000E94E6640F9441D66093AD096623B1F309
:10FB8000E4E5FFE08491882341F09091C00095FF67
:10FB9000FCCF8093C6003196F5CFCD36D10509F460
:10FBA00035C064F4C836D105B1F0C936D10509F0C5
:10FBB00052C0EAEAFDE8A591B49124C0CA3DD1053E
:10FBC00009F432C0CD3DD10509F045C0E2E9FDE8B8
:10FBD000A591B4913DC0ECEAFDE885919491FC01BA
:10FBE0002491222309F437C03091C00035FFFCCFA7
:10FBF0002093C6000196F3CF9091C00095FFFCCFF3
:10FC00008093C6008D918111F7CF25C0E8EAFDE809
:10FC1000A591B4918D918823F1F09091C00095FF4A
:10FC2000FCCF8093C600F6CFE4E9FDE8A591B4913E
:10FC30008D91882381F09091C00095FFFCCF809337
:10FC4000C600F6CF9091C00095FFFCCF8093C60010
:10FC50008D918111F7CF6091AD0970E04AE050E0DD
:10FC600086EC98E00E94D5628091C00085FFFCCFB1
:10FC70008AE08093C60081E0DF91CF9108954F9292
:10FC80005F926F927F928F929F92AF92BF92CF922C
:10FC9000DF92EF92FF92CF93DF9300D01F92CDB708
:10FCA000DEB72B013C0129833A834B835C838DEEC5
:10FCB0009FE00F9440E18F3F01F58EEE9FE00F949F
:10FCC00040E18F3FD1F48FEE9FE00F9440E18F3FF2
:10FCD000A1F480EF9FE00F9440E18F3F71F440E08A
:10FCE00050E0BA018DEE9FE00F9464E140E050E0F7
:10FCF000BA0181EF9FE00F9464E181EF9FE00F94E0
:10FD000048E14B015C018DEE9FE00F9448E16B01EF
:10FD10007C0169817A818B819C812CE330E040E019
:10FD200050E00F94A4DAC20ED31EE41EF51EB701F4
:10FD3000A6018DEE9FE00F9464E1C301B20128EEAD
:10FD400033E040E050E00F94A4DABA01A901480D75
:10FD5000591D6A1D7B1D81EF9FE00F9464E1109295
:10FD60003A0A10923B0A10923C0A10923D0A0F90F8
:10FD70000F900F900F90DF91CF91FF90EF90DF9059
:10FD8000CF90BF90AF909F908F907F906F905F903B
:10FD90004F900895CF92DF92EF92FF9220911C0A2C
:10FDA0002223F1F020E030E040E05FE30F94A2D89E
:10FDB0006B017C0120E030E0A9010F94CDD58823B0
:10FDC00079F0A7019601C701B6010F94A2D82BEDD7
:10FDD0003FE049E450E40F94A2D89B01AC0104C079
:10FDE00020E030E040E85FE360E070E080E89FE31F
:10FDF0000F94D4D5FF90EF90DF90CF90089560914D
:10FE00004402709145028091460290914702C2DF00
:10FE100060934002709341028093420290934302A8
:10FE20000895CF93DF93EC010F94184F81E0D3DD59
:10FE300080E00F947AAF209799F0C233D10540F05B
:10FE400062E370E080E090E00F942FCDE297ECCF7A
:10FE5000BE0180E090E00F942FCDC0E0D0E0E4CF71
:10FE6000DF91CF9108952F923F924F925F926F92C0
:10FE70007F928F929F92AF92BF92CF92DF92EF923A
:10FE8000FF921F93CF93DF934B015C01CC24CA9464
:10FE9000DC2C760165E5262E6AE0362E78EE472EBC
:10FEA00073E0572E612C712C1AE08091E7098111C3
:10FEB00026C12FEFC216D206E206F20651F0F7FC79
:10FEC0001EC10F9400CD6C197D09683B7B4008F082
:10FED00016C10F9400CD681979098A099B09693EFA
:10FEE00073408105910508F47FC08091951A8111B6
:10FEF00077C0EDE5FAE08491882341F09091C0004D
:10FF000095FFFCCF8093C6003196F5CFE091AD0907
:10FF100024E0E29FF0011124EE57F64E408151811A
:10FF20006281738121E030E086EC98E00E94C86332
:10FF3000E9E5FAE08491882341F09091C00095FFB3
:10FF4000FCCF8093C6003196F5CF6091AD0970E08B
:10FF50004AE050E086EC98E00E94D562F10184917D
:10FF6000E5E5FAE0882349F09091C00095FFFCCFC9
:10FF70008093C60031968491F5CFF7FE03C0E0E28E
:10FF8000F8E025C00F9400CD4B015C01C701B6011C
:10FF90006854744F8F4F9F4F681979098A099B09DC
:10FFA000A30192010F94A4DABA01A9012AE030E07A
:10FFB00086EC98E00E949D628091C00085FFFCCF96
:10FFC0000DC09091C00095FFFCCF8093C600819139
:10FFD0008111F7CF8091C00085FFFCCF1093C60040
:10FFE0000F9400CD4B015C010F94184F80E0F3DCBF
:10FFF00080E00F947AAFFFEFCF16DF06EF06FF0623
:020000021000EC
:1000000009F046C08091AB09E091AD09F0E0EF0145
:10001000CC0FDD1FCC0FDD1FCE57D64EEE0FFF1FCE
:10002000E657F64E8823D1F080819181BC01882764
:1000300077FD8095982F0F946FD620E030E040E850
:100040005FE30F94F3D49B01AC01688179818A81CD
:100050009B810F94D0D787FF4DC027CF808191819E
:10006000BC01882777FD8095982F0F946FD620E0EC
:1000700030E040E85FE30F94F4D49B01AC01688169
:1000800079818A819B810F94CDD518169CF50DCF6F
:10009000F7FC0BCFE091AD09F0E0EF01CC0FDD1FD5
:1000A000CC0FDD1FCE57D64EEE0FFF1FE657F64E94
:1000B00080819181BC01882777FD8095982F0F94CE
:1000C0006FD69B01AC01688179818A819B810F94F5
:1000D000F3D40F943CD697FF07C090958095709508
:1000E00061957F4F8F4F9F4F663071058105910558
:1000F0000CF4DBCE0F9400CD6B017C01D6CEDF91EA
:10010000CF911F91FF90EF90DF90CF90BF90AF9075
:100110009F908F907F906F905F904F903F902F9027
:100120000895CF93DF931F921F92CDB7DEB7BE0124
:100130006F5F7F4F88EF9FE00F94096E89819A81EE
:100140008156904F803A9F4020F11A821982ECE24A
:10015000FAE08491882341F09091C00095FFFCCF94
:100160008093C6003196F5CF8091C00085FFFCCF0B
:100170008AE08093C600BE016F5F7F4F88EF9FE0EB
:100180000F94F86D8FEE99E00F9429BC81E00F94E5
:1001900041B20F900F90DF91CF9108952F923F922F
:1001A0004F925F926F927F928F929F92AF92BF9287
:1001B000CF92DF92EF92FF920F931F93CF93DF9333
:1001C000CDB7DEB7CA58D2400FB6F894DEBF0FBE27
:1001D000CDBFC958DD4F688379838A839B83C75716
:1001E000D240FE01E75FFD4F88E2DF011D928A9554
:1001F000E9F7E850F24080E991E0DF019C011D92AF
:1002000021503040E1F7C75ADD4F19821882C95595
:10021000D240CE01875A9D4F5C014E019FE6891A5C
:100220009EEF990ADE01AF51BE4F3D0190EBC92E02
:100230009FE0D92E23E2E22EF12C00E010E0C3591A
:10024000DD4F8882CD56D240CD58DD4F9882C357BE
:10025000D240B701882777FD8095982F0F946FD6ED
:10026000D3016D937D938D939D933D01F501619134
:1002700071915F01882777FD8095982F0F946FD635
:10028000D4016D937D938D939D934D010F5F1F4F0F
:100290000630110559F0B501C6010F94096EB5E09D
:1002A000EB0EF11CE2E0CE0ED11CD3CFCF51DE4FCE
:1002B000288139814A815B81C15ED140C958DD4FB7
:1002C000688179818A819B81C757D2400F94CDD5AF
:1002D00087FD2BC3FE01EF51FE4F7F016E01FFE250
:1002E000CF1AFEEFDF0A3E012BEB621A2DEF720AE6
:1002F000C359DD4F0881CD56D240CD58DD4F18810E
:10030000C357D24085E090E0CF58DD4F9983888372
:10031000C157D240CF58DD4FA881B981C157D240D3
:100320001197CF58DD4FB983A883C157D240F70149
:100330002089318942895389648975898689978999
:100340000F94F3D44B015C01D80150962D913D914F
:100350004D915C91539754966D917D918D919C91A7
:1003600057970F94F3D4A50194010F94D4D5F601B7
:1003700092938293729362936F01D301BE92AE9275
:100380009E928E923D0104501109B4E0EB1AF108DF
:10039000CF58DD4FE881F981C157D240EF2B09F0EA
:1003A000B9CF6E01FFECCF1AFDEFDF0A3E0127E463
:1003B000621A2EEF720A2E013DE3430E511CCE014C
:1003C00001967C0101E010E0D6018D909D90AD90EA
:1003D000BC90139714962D913D914D915C91179778
:1003E000C501B4010F94F4D49B01AC010F94F4D473
:1003F000F70164A775A786A797A70130110541F0FB
:1004000080A691A6A2A6B3A684829582A682B78270
:100410000F5F1F4FD30114962D913D914D915C912B
:10042000179718966D917D918D919C911B970F94C4
:10043000F3D420E030E040EC50E40F94A2D8F20175
:100440006083718382839383F4E0CF0ED11C2CE20E
:10045000E20EF11C34E0630E711C88E2480E511C60
:100460000530110509F0B0CF8E010B5A1F4F6E01F8
:1004700091E5C90ED11C22242394312C2C0E3D1E53
:10048000A8ED2A0E311CF801B897208131814281F4
:100490005381F80160817181828193810F94D4D559
:1004A0004B015C01E12CF12C3601F8E26F1A710866
:1004B00026014E0C5F1CF301EE0DFF1D24813581DA
:1004C00046815781C501B4010F94A2D89B01AC01AC
:1004D000D20114966D917D918D919C9117970F94F7
:1004E000F3D4F2016483758386839783F4E0EF0E7F
:1004F000F11C24E1E216F104D9F6045D1F4F38E245
:10050000C30ED11C0215130509F0BDCF1E0185EBEA
:10051000280E311C6E0191EBC90ED11C3E01A7EED5
:100520006A1AADEF7A0A14E0E12EF12C270100E0FF
:1005300010E0812C912CA12CB12CF601E00FF11FC1
:10054000D301A00FB11F2D913D914D915C91608120
:100550007181828193810F94A2D89B01AC01B40177
:10056000C5010F94F4D44B015C01BFEF4B1A5B0A39
:100570000C5F1F4FE5E04E165104F9F69B01AC01EC
:10058000D1016D917D918D919C910F94F3D4F601E1
:1005900020813181428153810F94D4D5D3016D9351
:1005A0007D938D939C931397B1E0EB1AF108E8E2E9
:1005B0002E1A3108FCE2CF1AD10824E0621A710821
:1005C000E114F10409F0B2CFCB50DE4F888199815C
:1005D000AA81BB81C55FD140C957DD4F888399830C
:1005E000AA83BB83C758D2408E01075F1D4FDE012F
:1005F000AF5CBD4FC558DD4FB983A883CB57D24000
:10060000C359DD4F2880CD56D240CD58DD4F3880BC
:10061000C357D240FE01EF51FE4FC358DD4FF9835F
:10062000E883CD57D240C358DD4FA881B981CD575B
:10063000D240CD90DD90ED90FD90C358DD4FB98351
:10064000A883CD57D240C958DD4F288139814A81CE
:100650005B81C757D240C701B6010F94CDD518169C
:10066000B4F0C358DD4FE881F981CD57D2402081E5
:10067000318142815381C958DD4F688179818A81F6
:100680009B81C757D2400F94CDD51816FCF4CF5894
:10069000DD4F28813981C157D2402430310509F01E
:1006A0001FC1C957DD4F288139814A815B81C758F5
:1006B000D240C958DD4F688179818A819B81C757B3
:1006C000D2400F94D0D718160CF00AC1D801149656
:1006D0008D919D910D90BC91A02DC158DD4F8883C7
:1006E0009983AA83BB83CF57D240F80140805180C1
:1006F00062807380C558DD4FA881B981CB57D24045
:100700008D919D910D90BC91A02DC359DD4F888393
:100710009983AA83BB83CD56D240D1018D919D91FF
:100720000D90BC91A02DCD57DD4F88839983AA836E
:10073000BB83C358D240A7019601C958DD4F6881D9
:1007400079818A819B81C757D2400F94F3D4CD58C9
:10075000DD4F688379838A839B83C357D24020E02F
:1007600030E040E450E40F9405D96B017C01A30113
:100770009201C158DD4F688179818A819B81CF5771
:10078000D2400F94F3D44B015C0120E030E040EC08
:1007900050E4C359DD4F688179818A819B81CD56B0
:1007A000D2400F94A2D89B01AC01C501B4010F94B3
:1007B000D4D5A70196010F94A2D86B017C0120E04B
:1007C00030E040E05FE3C301B2010F94A2D84B01D7
:1007D0005C01CD58DD4F288139814A815B81C35747
:1007E000D240CA01B9010F94A2D89B01AC01C50146
:1007F000B4010F94A2D89B01AC01C701B6010F94BC
:10080000F4D46B017C01CD57DD4F288139814A81B9
:100810005B81C358D240F1016481758186819781E3
:100820000F94F3D4C359DD4F288139814A815B810C
:10083000CD56D2400F94D4D54B015C01C359DD4F46
:10084000288139814A815B81CD56D240CA01B901E4
:100850000F94F4D4A30192010F94A2D82B013C0170
:10086000C359DD4F288139814A815B81CD56D24001
:10087000C158DD4F688179818A819B81CF57D240F1
:100880000F94A2D89B01AC01C301B2010F94F4D420
:1008900020E030E040EC50E40F94D4D59B01AC0153
:1008A000C501B4010F94F3D4CD58DD4F28813981AF
:1008B0004A815B81C357D2400F94A2D89B01AC01FF
:1008C000C701B6010F94F4D4CD57DD4F288139818B
:1008D0004A815B81C358D2400F94F4D44B015C0130
:1008E000CF58DD4F28813981C157D2402F5F3F4F0C
:1008F000CF58DD4F39832883C157D2400C5F1F4F3B
:10090000C558DD4F88819981CB57D2400496C55890
:10091000DD4F99838883CB57D24094E0290E311C58
:100920002530310509F07FCE04C0812C912CA12CFB
:10093000B12CB401C501C657DD4F0FB6F894DEBF28
:100940000FBECDBFDF91CF911F910F91FF90EF9020
:10095000DF90CF90BF90AF909F908F907F906F90DF
:100960005F904F903F902F900895CF92DF92EF923B
:10097000FF926B017C018091720A8823A1F086EAC4
:100980009FE00F9440E1882371F0C701B60106DCB7
:1009900020915B1830915C1840915D1850915E1861
:1009A0000F94D4D503C060E070E0CB01FF90EF90CE
:1009B000DF90CF9008954F925F926F927F928F92C7
:1009C0009F92AF92BF92CF92DF92EF92FF920F93DE
:1009D0001F93CF93DF93CDB7DEB728970FB6F89468
:1009E000DEBF0FBECDBF0F94BA3D809156029091ED
:1009F00057029093760A8093750AE091F809F0E027
:100A0000EE0FFF1FE657F64E60817181882777FD54
:100A10008095982F0F946FD66093660A7093670A3B
:100A20008093680A9093690A8091F6099091F7097A
:100A30009093650A8093640A0F9400CD60934C0AEA
:100A400070934D0A80934E0A90934F0A80910C0A3E
:100A500090910D0AA0910E0AB0910F0A89839A8392
:100A6000AB83BC838093540A9093550AA093560A93
:100A7000B093570A4090100A5090110A6090120AE1
:100A80007090130A4092580A5092590A60925A0A7A
:100A900070925B0A8091140A9091150AA091160A2F
:100AA000B091170A8D839E83AF83B88780935C0AC9
:100AB00090935D0AA0935E0AB0935F0A6091180A52
:100AC0007091190A80911A0A90911B0A6093600A2A
:100AD0007093610A8093620A9093630A20E030E089
:100AE00040E85FE30F94F3D46093180A7093190AF7
:100AF00080931A0A90931B0A88EF99E09F938F9333
:100B0000812C912CB8ECAB2EB3E4BB2E18E1C12E96
:100B10001AE0D12EED80FE800F811885A30192018D
:100B200069817A818B819C810F940B2420E030E0D5
:100B300040EA51E46091140A7091150A8091160AF6
:100B40009091170A0F94F4D42B013C010F900F9051
:100B500020E030E042E553E40F94D0D718164CF073
:100B60004092140A5092150A6092160A7092170A5F
:100B70000CC080E090E0A2E5B3E48093140A909367
:100B8000150AA093160AB093170AE090140AF09081
:100B9000150A0091160A1091170A2091100A309137
:100BA000110A4091120A5091130A60910C0A709137
:100BB0000D0A80910E0A90910F0AA8EF6A2EA9E003
:100BC0007A2E7F926F92812C912CB0E7AB2EB1E4FC
:100BD000BB2EE8E1CE2EEAE0DE2E0F940B2410921D
:100BE0008B1910928A1910928D1910928C191092EB
:100BF0008F1910928E1980E090E0A8E4B2E48093FF
:100C00000C0A90930D0AA0930E0AB0930F0A80E08D
:100C100090E0AEE3B3E48093100A9093110AA0939E
:100C2000120AB093130AE090140AF090150A00918A
:100C3000160A1091170A7F926F92812C912CF8E47A
:100C4000AF2EF2E4BF2E9C01AD01C501B4010F949B
:100C50000B241092F7091092F6090F900F900F9045
:100C60000F9028960FB6F894DEBF0FBECDBFDF9170
:100C7000CF911F910F91FF90EF90DF90CF90BF9099
:100C8000AF909F908F907F906F905F904F900D945A
:100C9000BA3DE091F80984E0E89FF0011124EE5795
:100CA000F64E4081518162817381ECEEF9E08491CE
:100CB000882341F09091C00095FFFCCF8093C6003F
:100CC0003196F5CF22E030E086EC98E00E94C863D0
:100CD000E8EEF9E08491882341F09091C00095FFFF
:100CE000FCCF8093C6003196F5CF6091F80970E093
:100CF0004AE050E086EC98E00E94D562E4EEF9E02C
:100D00008491882341F09091C00095FFFCCF80939F
:100D1000C6003196F5CF40917019509171196091CC
:100D200072197091731921E030E086EC98E00E940E
:100D3000C8638091C00085FFFCCF8AE08093C60025
:100D40000895CF93DF93CDB7DEB72A970FB6F89407
:100D5000DEBF0FBECDBF0F9400CD6F83788789872C
:100D60009A87179A1092FD09169A1092FE09EFEDD4
:100D7000F9E08491882341F09091C00095FFFCCF69
:100D80008093C6003196F5CF8091C00085FFFCCFDF
:100D90008AE08093C60083E40F943A5D1C01409082
:100DA000360F5090370F6090380F7090390F0F94B6
:100DB000FE32481A590A610871080E948EE8481AE2
:100DC000590A6108710877FE03C0412C512C320189
:100DD0009091771280917612981799F0E09176129F
:100DE00027E5E29FF0011124E858FD4E20E030E0B5
:100DF00040E752E462A173A184A195A10F94A2D807
:100E000008C060910C0270910D0280910E029091C9
:100E10000F020F943CD67E836D830F9490220E9424
:100E200035E11092810A789420E030E040E85FE3F9
:100E30006091180A7091190A80911A0A90911B0A00
:100E40000F94F3D469837A838B839C83E090140A94
:100E5000F090150A0091160A1091170A2091100AB5
:100E60003091110A4091120A5091130A60910C0AB4
:100E700070910D0A80910E0A90910F0AA8EFB9E0C7
:100E8000BF93AF93812C912CE8ECAE2EE3E4BE2E01
:100E9000DE0111966D010F940B2420E030E040E854
:100EA0005FE36091180A7091190A80911A0A909173
:100EB0001B0A0F94F3D469837A838B839C832FE876
:100EC00032EC45EF5FE36091140A7091150A80914E
:100ED000160A9091170A0F94F4D46B017C0167E015
:100EE00074E062197309F4E076956795FA95E1F775
:100EF00080E090E00F946DD620915B1830915C18E3
:100F000040915D1850915E180F94D4D59B01AC01AF
:100F1000C701B6010F94F4D47B018C012091100A13
:100F20003091110A4091120A5091130A60910C0AF3
:100F300070910D0A80910E0A90910F0AA8EFB9E006
:100F4000BF93AF93812C912CA0E2AA2EA2E4BA2EDB
:100F5000DE0111966D010F940B24B301A20181E90A
:100F60009FE00F9464E10F900F900F900F9005E7B2
:100F70001FE0F12CB3E0EB2E80918B11882341F11F
:100F80008F2D6E2D0F9470DAB5E18B02F0011124D4
:100F900023E09202E00DF11D1124EE0FFF1FEE0F72
:100FA000FF1FE557FE4E20E030E04AE754E4618140
:100FB0007281838194810F94A2D820E030E040E0D8
:100FC0005FE30F94F4D40F94AAD60F943CD602C0DA
:100FD00060E070E0C8010F946CE1F3940E5F1F4F66
:100FE00089E0F812C9CFB10183E79FE00F946CE16B
:100FF00040910C0A50910D0A60910E0A70910F0AEF
:101000008DE99FE00F9464E14091100A5091110A1C
:101010006091120A7091130A81EA9FE00F9464E1D3
:101020004091140A5091150A6091160A7091170A9E
:101030008DE89FE00F9464E1BE016B5F7F4F89E80C
:101040009FE00F94F86DE091F809F0E0EE0FFF1FBC
:10105000E657F64E60818CE89FE00F9452E1609174
:1010600088198BE89FE00F9452E16091F60988E8B7
:101070009FE00F9452E161E085EA9FE00F9452E116
:101080000F94BA3DEAEDF9E08491882341F0909104
:10109000C00095FFFCCF8093C6003196F5CF83E466
:1010A0000F943A5D4AE050E0BC0186EC98E00E9463
:1010B000276384E69FE00F9440E161E0680F84E6D7
:1010C0009FE00F9452E1EFECF9E08491882341F026
:1010D0009091C00095FFFCCF8093C6003196F5CF6C
:1010E0008091C00085FFFCCF8AE08093C6000F94FA
:1010F00000CDAB01BC018F819885A985BA85481BBD
:10110000590B6A0B7B0B2AE030E086EC98E00E94DA
:101110003363F894FFCF6F987798EAE6F0E0808128
:101120008F7B8083808180688083EF9A08951F92EF
:101130000F920FB60F9211240BB60F920F931F93BD
:101140002F933F934F935F936F937F938F939F93CF
:10115000AF93BF93EF93FF938091F6099091F709B6
:101160008B3491050CF441C080916A0086FF0BC05E
:101170000F9400CD6093480A7093490A80934A0AFD
:1011800090934B0A2CC00F9400CD0091480A109107
:10119000490A20914A0A30914B0A601B710B820B5D
:1011A000930B2091F6093091F709253631052CF083
:1011B00003E010E020E030E004C004E010E020E0B4
:1011C00030E0601771078207930748F08091230A87
:1011D0009091240A02969093240A8093230A809186
:1011E0006A0090E4892780936A00FF91EF91BF9194
:1011F000AF919F918F917F916F915F914F913F91AF
:101200002F911F910F910F900BBE0F900FBE0F905B
:101210001F9018956C987498EAE6F0E080818160E0
:10122000808380818D7F8083EC9A08951F920F9236
:101230000FB60F9211240BB60F922F933F934F933B
:101240005F936F937F938F939F93AF93BF93EF932E
:10125000FF93EC98EAECF9E08491882341F09091B7
:10126000C00095FFFCCF8093C6003196F5CF8091EA
:10127000C00085FFFCCF8AE08093C6008091810A80
:1012800081115FDDFF91EF91BF91AF919F918F91A0
:101290007F916F915F914F913F912F910F900BBE76
:1012A0000F900FBE0F901F901895BF92CF92DF92B4
:1012B000EF92FF920F931F93CF93DF93CDB7DEB7DB
:1012C000E1970FB6F894DEBF0FBECDBF88E89FE070
:1012D0000F9440E1B82EBE01605D7F4F89E89FE02A
:1012E0000F94096EE3E7F8E08491882341F0909130
:1012F000C00095FFFCCF8093C6003196F5CF68A95A
:1013000079A94AE050E086EC98E00E94DC628E0108
:10131000015E1F4F85E9E82E8FE0F82ED02EC12EFA
:10132000C7010F9440E1F80181938F01FFEFEF1A9D
:10133000FF0A8DE9E8168FE0F80691F71FA2ED2D60
:10134000FC2D8191882339F09091C00095FFFCCF4E
:101350008093C600F6CF6EE678E08D2D9C2D0F941D
:10136000EFDDCF92DF9287E698E09F938F938E0117
:101370000F5F1F4F1F930F930F9414DF0F900F9069
:101380000F900F900F900F907E0195E0E90EF11CE9
:10139000F7018081882349F0992787FD90950F9464
:1013A000DEDDF70181937F01F3CF60E0C8010E9489
:1013B000ABE181E99FE00F9448E1F62EE72ED82EAD
:1013C000C92EECE4F8E08491882341F09091C000AC
:1013D00095FFFCCF8093C6003196F5CF2AE030E030
:1013E0004F2D5E2D6D2D7C2D86EC98E00E94336391
:1013F00061E088E498E00E94ABE163E478E0C80132
:101400000F94FADD8DE99FE00F9448E16CA77DA76A
:101410008EA79FA7CE018C960F946373BC01C80161
:101420000F9489DE60E478E0C8010F94EFDD81EA73
:101430009FE00F9448E16CA77DA78EA79FA7CE01E0
:101440008C960F946373BC01C8010F9489DE69E325
:1014500078E0C8010F94EFDD60E0C8010E94ABE1C5
:1014600064E378E0C8010F94FADD8DE89FE00F9403
:1014700048E16CA77DA78EA79FA7CE018C960F94FD
:101480006373BC01C8010F9489DE60E0C8010E944B
:10149000ABE161E089E298E00E94ABE189A98F931A
:1014A00088A98F9382E298E09F938F931F930F9365
:1014B0000F9414DF60E0C8010E94ABE16BE178E0BB
:1014C000C8010F94FADD8B2D90E09DA78CA7CE016B
:1014D0008C960F943876BC01C8010F9489DE60E0C9
:1014E000C8010E94ABE1CF92DF92EF92FF9282E1BE
:1014F00098E09F938F931F930F930F9414DF60E0F6
:10150000C8010E94ABE161E08EE098E00E94ABE18F
:101510000FB6F894DEBF0FBECDBFE1960FB6F894BC
:10152000DEBF0FBECDBFDF91CF911F910F91FF9016
:10153000EF90DF90CF90BF9008954F925F926F929F
:101540007F92AF92BF92CF92DF92EF92FF920F9372
:101550001F93CF93DF93CDB7DEB7E0970FB6F89424
:10156000DEBF0FBECDBF2B013C0169017A01809126
:1015700067098111E5C0F8940F94DE328091360F2F
:101580009091370FA091380FB091390F8093630974
:1015900090936409A0936509B09366090F94FE3295
:1015A00040916309509164096091650970916609E1
:1015B000481B590B610971094093630950936409F1
:1015C00060936509709366090E948EE840916309F3
:1015D000509164096091650970916609481B590B27
:1015E0006109710940936309509364096093650927
:1015F000709366099091771280917612981799F0FE
:10160000E091761287E5E89FF0011124E858FD4E3D
:1016100020E030E040E752E462A173A184A195A1EB
:101620000F94A2D808C060910C0270910D028091B5
:101630000E0290910F0260934F09709350098093AE
:101640005109909352090F94902280E1ECE0FAE066
:10165000A3E5B9E001900D928A95E1F78091F80930
:1016600080934E098091070280934D090E9435E1D5
:101670001092810A81E080936709789420E030E03D
:10168000A901C301B2010F94CDD581110AC020E098
:1016900030E0A901C701B6010F94CDD5882309F424
:1016A0004FC069E078E0FE0131965F01CF010F94F1
:1016B000FADDF50101900020E9F78F0101501109D1
:1016C00020915B0930915C0940915D0950915E0960
:1016D000C301B2010F94F4D423E048E00F941DDB62
:1016E00066E078E0C5010F94EFDDF5010190002080
:1016F000E9F78F010150110923E046E0C701B60167
:101700000F941DDB63E078E0C5010F94EFDDF50178
:1017100001900020E9F78F010150110960916002EA
:1017200070916102809162029091630223E048E02F
:101730000F941DDB60E0C5010E94ABE10E944AE30B
:10174000E0960FB6F894DEBF0FBECDBFDF91CF910C
:101750001F910F91FF90EF90DF90CF90BF90AF90CF
:101760007F906F905F904F90089520E030E0A90146
:1017700060E070E080E291E4E0CE8F929F92AF92C1
:10178000BF92CF92DF92EF92FF920F931F93CF936E
:10179000DF9300D01F92CDB7DEB79B01AC018091E3
:1017A0006709882309F497C080914E098093F8094E
:1017B00080914F0990915009A0915109B09152091F
:1017C00080930C0290930D02A0930E02B0930F022F
:1017D00060915F097091600980916109909162093F
:1017E0000F94F3D469837A838B839C83CE01019613
:1017F0000F94643220E030E040E551E460916002F3
:101800007091610280916202909163020F94D4D52D
:101810004B015C01E0905B09F0905C0900915D096F
:1018200010915E092091570930915809409159094A
:1018300050915A096091530970915409809155094A
:1018400090915609E8EFF9E0FF93EF93EFE5CE2E84
:10185000E9E0DE2E0F940B240F94BA3D80E1E3E51E
:10186000F9E0ACE0BAE001900D928A95E1F780E1F1
:10187000ECE0FAE0A7EDB9E001900D928A95E1F76E
:1018800040916309509164096091650970916609FE
:1018900040931D0D50931E0D60931F0D7093200DEE
:1018A00088E69CE00E941FC98091630990916409B9
:1018B000A0916509B09166098093360F9093370F18
:1018C000A093380FB093390F81E08093810A109272
:1018D00067090F900F900F900F900F900F90DF916E
:1018E000CF911F910F91FF90EF90DF90CF90BF901D
:1018F000AF909F908F900895EEEEF7E0849188234B
:1019000041F09091C00095FFFCCF8093C6003196C6
:10191000F5CF40910C0A50910D0A60910E0A70911A
:101920000F0A23E030E086EC98E00E94C863EBEEFB
:10193000F7E08491882341F09091C00095FFFCCF9F
:101940008093C6003196F5CF4091100A5091110A4C
:101950006091120A7091130A23E030E086EC98E05F
:101960000E94C863E8EEF7E08491882341F09091EB
:10197000C00095FFFCCF8093C6003196F5CF409113
:10198000140A5091150A6091160A7091170A23E003
:1019900030E086EC98E00E94C863E6EEF7E08491C0
:1019A000882341F09091C00095FFFCCF8093C60042
:1019B0003196F5CF8091C00085FFFCCF8AE08093FF
:1019C000C6000895EEECF7E08491882341F09091F1
:1019D000C00095FFFCCF8093C6003196F5CF0F94E1
:1019E000293EAB01BC0123E030E086EC98E00E9488
:1019F000C863EBECF7E08491882341F09091C0003C
:101A000095FFFCCF8093C6003196F5CF81E00F940F
:101A1000293EAB01BC0123E030E086EC98E00E9457
:101A2000C863E8ECF7E08491882341F09091C0000E
:101A300095FFFCCF8093C6003196F5CF82E00F94DE
:101A4000293EAB01BC0123E030E086EC98E00E9427
:101A5000C863E6ECF7E08491882341F09091C000E0
:101A600095FFFCCF8093C6003196F5CF8091C000E2
:101A700085FFFCCF8AE08093C6000895EF92FF9225
:101A80000F931F93CF93DF93E2EBF7E084918823CA
:101A900041F09091C00095FFFCCF8093C600319635
:101AA000F5CF0BE811E1F0EBEF2EF7E0FF2EC0E0F1
:101AB000D0E0F801EC0FFD1F4181528163817481F8
:101AC00023E030E086EC98E00E94C863F70184913F
:101AD000E0EBF7E0882349F09091C00095FFFCCF40
:101AE0008093C60031968491F5CF2496CC31D105F0
:101AF00001F7045E1F4FF2E10F341F07C1F6EFEA52
:101B0000F7E08491882341F09091C00095FFFCCFCD
:101B10008093C6003196F5CF8091C00085FFFCCF41
:101B20008AE08093C600DF91CF911F910F91FF90C3
:101B3000EF9008952F923F924F925F926F927F9213
:101B40008F929F92AF92BF92CF92DF92EF92FF92CD
:101B50000F931F93CF93DF93CDB7DEB7C355D10952
:101B60000FB6F894DEBF0FBECDBF82E090E0909339
:101B700016028093150283E993E00E94A7648823EC
:101B8000B1F080914E0F90914F0F6AE270E0059690
:101B90000F9494DE009711F0DC011C9280914E0F9F
:101BA00090914F0F05960F94D66E0C9409B988E961
:101BB00093E00E94A764882309F4C4C18EE993E0EE
:101BC0000E94A764882391F08091951A882311F4CC
:101BD0000C9409B90F9400CD60937B0A70937C0A32
:101BE00080937D0A90937E0A0C9409B983EA93E06E
:101BF0000E94A764882361F060913E0A70913F0AB9
:101C00004AE050E086EC98E00E9427630C9409B902
